:020000040800F2
:1000000000C0002065BB00081104000813040008AC
:100010001504000817040008190400080000000077
:100020000000000000000000000000001B040008A9
:100030001D040008000000001F040008210400083F
:10004000B1BB0008B1BB0008B1BB0008B1BB0008E0
:10005000B1BB0008B1BB0008B1BB0008B1BB0008D0
:10006000B1BB0008B1BB0008B1BB0008B1BB0008C0
:10007000B1BB0008B1BB0008B1BB0008B1BB0008B0
:10008000B1BB0008B1BB0008B1BB0008B1BB0008A0
:10009000B1BB0008B1BB0008B1BB0008B1BB000890
:1000A000B1BB0008B1BB0008B1BB0008B1BB000880
:1000B000B9290008352A0008D52A0008B1BB000874
:1000C000B1BB0008B1BB0008B1BB0008B1BB000860
:1000D000B1BB00080D2C0008492E00085D2F000858
:1000E000B1BB0008B1BB0008B1BB0008B1BB000840
:1000F000B1BB0008B1BB0008B1BB0008B1BB000830
:10010000B1BB0008B1BB0008492B0008B1BB000817
:100110006131000811320008B1BB0008B1BB000812
:10012000B1BB0008B1BB0008B1BB0008B1BB0008FF
:100130000348044B834202D0034B03B11847704776
:10014000B80D0020B80D0020000000000548064B47
:100150001B1AD90F01EBA301491002D0034B03B1C5
:1001600018477047B80D0020B80D002000000000AF
:1001700010B5064C237843B9FFF7DAFF044B13B1EF
:100180000448AFF300800123237010BDB80D002098
:10019000000000003001000808B5054B1BB10549FF
:1001A0000548AFF30080BDE80840FFF7CFBF00BFB0
:1001B00000000000BC0D00203001000810B52C4BE1
:1001C0001A7882B901224FF496712A481A7002F007
:1001D000A3FB4FF49661284802F09EFB4FF4167182
:1001E000264802F099FB264C2278012A06D1254B9D
:1001F000197819B931201A7000F0C0FF224B1A7813
:1002000072B9224A1278012A0AD1214A1278012AA7
:1002100006D120481A700CF0C3FA672000F0AEFF38
:10022000154802F087FB40B1134802F07DFB2378AC
:10023000012B02D1312000F0A1FF0E4802F07AFB21
:1002400040B10C4802F070FB134B1B7813B96220CD
:1002500000F094FF094802F06DFB38B1074802F046
:1002600063FBBDE81040672000F088BF10BD00BFF1
:10027000F00D0020E80D0020E00D0020D80D00203A
:1002800058380020D50D0020D40D0020DE0E0020AF
:10029000DD0E00207C200108890E00204FF4A060B4
:1002A0000BF05EB808B54FF49661504802F034FB8D
:1002B0000BF004F8FFF7F2FF4FF4165002F060FC69
:1002C0004FF4164002F0F0FC4FF4165002F06AFEB4
:1002D0004FF4E13002F05AFF41F61F414FF47A70BB
:1002E00002F040FB41F61F41642002F079FB41F629
:1002F0001F4141F2883002F0C3FB41F61F416420E8
:1003000002F0F8FB3A480CF04BFA07F01DFD07F03D
:1003100061FD38480CF044FA05F08AFB01200AF030
:1003200061FB40F27121052002F0C8FA902000F034
:1003300025FF314D314C02F0B3FF03F009FA04F010
:1003400017FD07F001FE01F055F801F00FFC07F072
:100350003BFE07F055FF07F063FC05F02FFC06F0AD
:100360002DF900F013FF0AF053FE0AF045FB01F0EF
:10037000C7F908F02DFC02F059F82B782BB90AF0D8
:1003800033F901F047FB01F075FB00F04FF9FFF77F
:1003900015FF0AF0FDF802F0CBF802F059F908F069
:1003A0006FFC08F0AFFC08F0E9FC02F09BFA0F4884
:1003B00002F0C0FA10B10D4802F0B6FA2378012B12
:1003C00006D1002323700E4B0E4819880CF0E8F973
:1003D0000D4B1A78012A04BF00221A700B4B1A78B1
:1003E000012AA8D100221A70A5E700BFF40D002051
:1003F00092200108C3200108890E0020010F00206F
:10040000020F0020DC200108000E0020CD0E00208D
:100410007047FEE7FEE7FEE7FEE77047704770476C
:1004200070470000374B82B01A6842F001021A6030
:100430005968354A0A405A601A6822F0847222F4D8
:1004400080321A601A6822F480221A605A6822F4F4
:10045000FE025A604FF41F029A600022009201923D
:100460001A6842F480321A601A6802F4003201926B
:10047000009A01320092019A1AB9009AB2F5A06F5F
:10048000F2D11A6812F4003218BF01220192019AC7
:10049000012A30D11D4A116841F010011160116824
:1004A00021F003011160116841F0020111605A68E6
:1004B0005A605A685A605A6842F480625A605A68B0
:1004C00022F47C125A605A6842F4E8125A601A68A0
:1004D00042F080721A601A689201FCD55A6822F0C4
:1004E00003025A605A6842F002025A605A6802F0E7
:1004F0000C02082AFAD14FF00062054B9A6002B054
:10050000704700BF001002400000FFF800200240CA
:1005100000ED00E07FB501AC84E80E00F42250430A
:100520000D4C21184A78132A14D8561C4E701421E9
:10053000255C2A44B2FBF1F501FB15220C2101FBDD
:1005400002000444043401AA07CA84E80B00012015
:1005500004B070BD0020FBE778190020F423F0B54B
:1005600003FB00F20A4CA518697879B10C26A35C4C
:10057000101D06FB030014260133B3FBF6F706FB40
:10058000173301392044A3546970F0BD0846FCE7D5
:10059000781900200B460122002110B50BB9104636
:1005A00010BD00FB01F4A2FB0021013BDBB22144A2
:1005B000F4E7000000B5174B8DB01A8803A8A2F22B
:1005C0006C7208929A78013A0792DA7806921A7950
:1005D00005925A799B79049203930CF065FB0E4BBC
:1005E000C3E9000110F5E14041F10001CDE900014E
:1005F00068460CF07BF9094A034610601421084A4A
:1006000008480DF083FA074907480CF0C9F80DB007
:1006100000BD00BF541C0020F80E00205C1C002010
:10062000EC200108681C0020FE20010813B5194BBE
:100630001A782AB901220A2117481A7002F06CF9B7
:10064000154802F077F910B3134802F06DF9134B17
:100650001B7813B912480CF0A3F81249D1E9003203
:100660005C1C42F10000C1E9004047F281015B18C7
:1006700042F100026846CDE900320CF037F90A4A2F
:10068000034610601421094A09480DF03FFA02B0F0
:1006900010BD00BFF40E0020EC0E0020000F002063
:1006A0000F210108F80E00205C1C0020EC2001083E
:1006B000681C002041F23113984264D02FD840F6D4
:1006C000A173984256D014D840F2D173984208D002
:1006D0000CD840F2E933984248D040F2EB339842CC
:1006E00014D1814214BF00200120704740F2D3731F
:1006F000F5E741F26903984242D009D840F6AB735E
:1007000098423AD041F20F0398423FD00020704700
:1007100041F2CD039842F9D141F2CE0328E041F2F3
:100720008A339842DDD012D841F225339842D8D08E
:100730000AD841F25D2398422ED041F2C12398425B
:10074000E4D141F2C22313E041F28933C7E741F219
:100750007B7398421DD041F285739842C1D041F21B
:1007600074739842D2D14EF6892301E042F21B7392
:100770009942B7E740F6A273FAE740F6B673F7E797
:1007800041F26A03F4E741F23213F1E741F27E03EA
:10079000EEE74EF66B23EBE741F25E23E8E700005D
:1007A00030B503780246482B89B03AD14378452BBF
:1007B00037D18378522B34D1C3784F2B31D10125D7
:1007C000814BC48981481D7063BA038099B2804B04
:1007D0001888FFF76FFF08B17E4B1D7041F6273375
:1007E0009C427BD042F21B7399422FD84CF6106387
:1007F0009C4200F0A18041F2CE03994219D84AF2FE
:100800000F239C4271D040F6A173994209D94BF253
:100810000F639C4200F0908046F610239C4200F04B
:100820008B804FF4806200216B480BF0CBFF09B046
:1008300030BD43F211239C427ED045F612639C42A8
:10084000EFD1664B127C1A70654B4BE046F6EA33EB
:100850009C4200F0B38048F6EA139C42E1D1137C3D
:1008600060490B70591E0329DBD8507C5E49012B6F
:100870000870907C5D490870D07C5D490870107DDF
:100880005C49087028D0507D5B49022B0870907D30
:100890005A490870D07D5A490870107E594908702D
:1008A0001AD0507E5849042B0870907E5749087022
:1008B000D07E57490870107F564908700CD1517F7F
:1008C000554B1970917F554B1970D17F544B92F84D
:1008D00020201970534B1A70534B03E0534B127C7A
:1008E0001A70534B01221A709BE7117C514B02F195
:1008F0001A041970D2F811304F491BBA0B60D2F8A4
:100900001530527E4D494E4D1BBA402A0B602A705D
:1009100003D94C480BF044FF402221464A480DF0D1
:100920000BFC2B784949E218E35812791BBA0B608B
:10093000474B1A70474BD5E7117C3E4B02F11A0426
:100940001970D2F811303C491BBA0B60D2F815303F
:10095000527E3A493A4D1BBA402A0B602A7003D99D
:1009600038480BF01DFF4022214637480DF0E4FBCC
:100970002A783649A318A2589D1D12BA0A6019791F
:10098000334A354C5B791170684620220021237070
:100990000BF018FF2278202A03D92A480BF000FF19
:1009A0002022294668460DF0C7FB6A462B492C4891
:1009B0000BF06AFD237806332370BBE71369294ADD
:1009C0001BBA1360284B8DE7010F0020020F002097
:1009D000040F0020A9100020502800208A0E0020BB
:1009E0008B0E0020300E00202F0E00201D0E002048
:1009F0001C0E00201B0E00202E0E00201A0E0020C0
:100A0000190E0020180E00202D0E0020170E0020B9
:100A1000160E0020150E00202C0E0020140E0020B3
:100A2000130E0020120E0020990E0020010E00204F
:100A3000980E002045190020281600204819002093
:100A400078160020232101088B160020940E002028
:100A50008A1600209C0E00208C0E002035210108F3
:100A6000EC170020900E00209A0E00206821F0B5AF
:100A7000184BC1B000938DF8051003784178847845
:100A80008DF804300B448DF80610303B10F8031F2E
:100A900023448DF807408DF808100B446A4641EA5C
:100AA0000421092401F10A06B6B225460134A4B294
:100AB000B44209D1535516230B31104689B2135550
:100AC00002F0C0FA41B0F0BD10F8017F57553B4429
:100AD000EBE700BFFEFEFE68F7B500230546A14C1C
:100AE00001466070A0482370A370E3700BF058FEBD
:100AF000312D4DD81F2D08D8013DEBB2082B2FD931
:100B00009A480BF04DFE04256FE0203D112DF7D8DB
:100B100001A353F825F000BF750C0008FD0C000878
:100B2000C10D0008470E0008010B0008010B00086A
:100B3000010B0008010B0008010B0008010B000865
:100B4000010B0008010B0008010B0008010B000855
:100B5000010B0008010B0008530E00086F0E00087F
:100B6000082DCDD801A353F825F000BFCF0B000806
:100B7000010C00085D0C0008650C0008010B000862
:100B8000010B0008010B0008070B0008070B000809
:100B9000672D10D85F2DB3D90120613D2071062D3E
:100BA00000F26F81DFE815F07201FB014D02550282
:100BB00058029802BA02902DA2D101236C482371E9
:100BC0000DF0C8FA6A4982B2451D601D4BE1012350
:100BD000684D2371684B2A781B78684968486371AF
:100BE000A2710DF0A9FA2D78073529462B1F5D4813
:100BF0001A0AA270E37003B0BDE8F040FFF736BFF9
:100C00000122604B22711B78FF2B15D1A2715E4A25
:100C1000042312786371E271022222725B4A237309
:100C200012785B4B62720322A2725A4A1278E27205
:100C30001B780E256373D8E7A371013B6271032B08
:100C400014D8DFE803F0020507094F4B1B780EE0CC
:100C50004E4BFBE74F4BF9E74D4BF7E70123237171
:100C60000525C2E7012323716371A37100230825C1
:100C7000E371BAE70123484A23711278042A09D89C
:100C8000002AEDD0023A6371022A23D8DFE802F08D
:100C90002A2E3200FF2AE3D1A371404B04221B8885
:100CA0006271190A2372022363723D4BE1711B8842
:100CB000E273190AE372032323733A4BA1721B8870
:100CC0001225190AA373384B61731B881A0A227400
:100CD00063748AE7A371314B1B8809251A0AE271F4
:100CE000237282E70223A3712D4BF5E70323A3713F
:100CF0002C4BF1E70423A3712B4BEDE701232B4A87
:100D000023711278042A09D8002AA9D0023A637103
:100D1000022A18D8DFE802F01A1E2200FF2A9FD10B
:100D2000A371234B04221B786271E37102232372A7
:100D3000204B22731B7863720323A3721E4B1B7814
:100D4000E3721E4B74E7A371194B7FE70223A37173
:100D5000184B7BE70323A371174B77E70423A37199
:100D6000164B73E77C1D00203E210108B0210108CD
:100D7000A8210108A60E0020A70E00200D180020B3
:100D8000831D0020A30E0020CB0E0020CA0E0020E1
:100D9000C80E0020C90E0020A20E0020A0100020C6
:100DA0009E1000209C1000209A100020A10E002010
:100DB000840B0020830B0020820B0020810B00207D
:100DC0000123A74A23711278042A0BD8002A3FF482
:100DD00047AF023AA3496371022A24D8DFE802F040
:100DE000222F3100FF2A7FF43BAF0225002104208F
:100DF000A5720325A3719B4BA5731B78162503EBE6
:100E00008303DA095B006071E17122726372E1723F
:100E100022736373E17322746374A074E1742275A6
:100E20006375E2E60223A3710023E3710B780A25C0
:100E300003EB83035A00DB0923726272D5E60323B6
:100E4000F1E70423EFE7012323716371A371864B5C
:100E5000FCE60123854823710DF07CF9834960711C
:100E600082B2851D82480DF067F9ADB2BDE601235F
:100E70000F2280497E482371627115250DF05CF9BF
:100E8000B3E67D4B06251B786371AEE67B4B7C4E4B
:100E90001D787C4B022D19787B4B36781A787B4B6A
:100EA0001B7807D0052D2AD00525794800960BF030
:100EB00077FC9AE6A071774865710088A573070AE8
:100EC00020727548E77100886173070AA072734841
:100ED000677200886275070A20737148E77200889C
:100EE000050A20746F48E5730088050AA0746E48EF
:100EF00065740088050AE57420751625D5E7A0718C
:100F00006448042500886571070A20726248E77109
:100F100000886173070AA072604867720088627572
:100F2000070A20730220A0735D48E7720088070A51
:100F300020745C48E7730088070AA0745A486774F5
:100F40000088070A20750320A0755848E7740088B8
:100F5000070A20765648E7750088070AA0765548A4
:100F600067760088070AE77620775348A5770088D8
:100F70006377050A84F820005048E577008884F8F4
:100F80002560050A84F822004D4884F82150008825
:100F9000050A84F8235084F82400262585E7374B7A
:100FA000374E1D78374B022D1978374B37781A7822
:100FB000364B1B7805D0052D1AD0052541480097E2
:100FC00075E74FF0000CA071264865710078E57256
:100FD00000EB8000C6094000102584F807C0267287
:100FE0006072A17284F80CC06673A073E273E5E7C7
:100FF0001C4DA0712D784FF0000C05EB8505EE0916
:10100000680002254FF0040EE572032584F805E020
:10101000257484F807C01A2526726072A17284F8BC
:101020000CC06673A073E27384F811C0A674E074F8
:10103000237584F815E084F816C0E6752076677687
:10104000BCE7214B1B786371204B1B780725A371EC
:10105000CBE51F4B6071F8E71E4B6071A071F5E5A1
:10106000A00E0020F4110020E20E00205021010803
:10107000821D002059380020700E00201D00002025
:10108000810B0020840B0020830B0020820B0020AA
:1010900060210108C60E0020BE0E0020BC0E0020FC
:1010A000C40E0020BA0E0020B80E0020C20E002090
:1010B000B60E0020B40E0020C00E0020B20E00209C
:1010C000B00E00208B21010808100020071000201E
:1010D00005100020E10E002000221F490B78012B93
:1010E00005BF0A701D4A1346127804BF0825E27135
:1010F0001B4A18BF0625117808BFA37101290BD11F
:101100000021117002216A1C61550D44154992B2EB
:101110000978ADB2A1540133637166E5124B102515
:101120001B786371114B1B78A371114B1B681A0E4E
:10113000E2711A0C2272A3721A0A0E4B62721B78A9
:10114000E3720D4B1B681A0E22731A0C62731A0A93
:10115000A273E37349E500BFE50E0020E00E002016
:10116000E40E0020DF0E0020DD0E0020DC0E00204B
:10117000D80E0020D40E0020D00E0020024B188084
:101180000ECB0220FFF7C6B96019002070B5774E6C
:101190003378FD2B19D1764D76486C7821460BF0CB
:1011A000FFFA312C4ED81F2C22D8032C00F08C8053
:1011B000042C00F08E80022C55D04FF48072002158
:1011C0006B480BF0FFFA002333706B4B1A782AB987
:1011D0000122022169481A7001F09EFB684C2378B5
:1011E000002B00F0AE80012B00F0B8800023B3E0AC
:1011F000203C112CE1D801A353F824F0D7120008A9
:10120000E7120008F712000807130008BB110008D6
:10121000BB110008BB110008BB110008BB1100087E
:10122000BB110008BB110008BB110008BB1100086E
:10123000BB110008BB110008BB1100080B1300080C
:101240000F130008912C64D0922CB6D1B5F805305C
:10125000B3F5807F6FD0B3F5007FAED1B5F807301E
:10126000484A5BBA6BE06B794749484A0B70ABB9A7
:10127000FF230B701370464B1B7843B1454B1B7813
:101280002BB1454B1B7813B1444B1B7813B901228A
:10129000434B1A700220FFF771FF8EE71370013B7A
:1012A000032BF7D801A252F823F000BFBD120008AB
:1012B000C1120008C512000889120008344BE4E787
:1012C000344BE2E7344BE0E7364B012220461A70FC
:1012D000E1E7354BF9E76B79344A002B08BFFF2370
:1012E00020201370D7E76B79314A002B08BFFF230A
:1012F00021201370CFE76B792E4A002B08BFFF2304
:1013000022201370C7E72320C5E73020C3E7312030
:10131000C1E7AB7969791B0443EA0163E979287A6B
:10132000254A43EA0123D9170343C2E900310122C8
:10133000224B1A7041E7B5F80730214A5BBA138097
:101340003BE70220FFF70AF970B10078FFF7C4FB12
:101350000A4801F0E9FA0123237005E0074801F08B
:10136000E9FA00287FF442AF70BD00BFD60F00201D
:101370004C270020BF210108100F0020080F00207B
:10138000060F0020FC0D0020A40E0020A30E00205C
:10139000CB0E0020CA0E0020C90E0020C80E00206F
:1013A000A50E00209F0E0020610E0020A20E00203E
:1013B000A10E0020A00E0020F80E0020000F00203B
:1013C000FE0D002038B5044608480D190BF0E8F969
:1013D000AC4204D1BDE8384004480BF0E1B914F840
:1013E000011B03480BF0DCF9F2E700BFE92001081C
:1013F000D12101082DE9F0410025304A304C137805
:101400002570012B44D12F48157023700CF0A2FEDB
:101410002D4E4FF48072294630702C480BF0D2F9D3
:101420003278284929480CF087FE2378002B43D0D6
:10143000DFF8948098F80030002B3DD00021012780
:10144000234E244D244B4FF4807224481F7031707A
:1014500029700BF0B7F9237898F800201B491F4832
:1014600033702A700CF068FE1D480BF099F9317842
:101470001C480BF095F929781B480BF091F9174996
:101480001A480BF08DF93846BDE8F041FFF776BEFB
:10149000174B1A78012A0FD11D7002232370154BA8
:1014A000094E1B784FF480722946084833700BF0C0
:1014B00089F932781049B5E7BDE8F081861100203E
:1014C000A90E002088110020A80E0020CB160020B5
:1014D000A70E0020A60E0020921000200D1800205C
:1014E000D9210108EC210108F72101080122010896
:1014F000DE110020D9110020AE380020214B1A78CF
:10150000012A03D1002204201A7070471E4B1F4984
:101510001A78012A02D00878012804D1002201207B
:101520001A700A7070471A490878012803D10023FD
:1015300002200B70704717490878012803D1002357
:1015400003200B70704714490878012803D1002349
:1015500005200B707047032A07D1104A107800222B
:101560000A2818BF07201A707047042A4FF000009D
:1015700002D1187008207047052A04BF187009208E
:10158000704700BF870E002086110020DB1100206D
:10159000DE110020DD110020DC1100208711002069
:1015A00010B5044686B01122002101A80BF00AF9FB
:1015B000601E092818D8DFE800F005191927191747
:1015C0002B17442B0924224B2246224922481C7007
:1015D0000CF0B2FD22461F4920480CF0ADFD11224F
:1015E0001F4920480CF0A8FD06B010BD1E4B1F4936
:1015F0001A78174B18481A700CF09EFD2322002110
:101600001A480BF0DFF8EFE70022114B1A70EBE7F6
:10161000174B0F4C1A7817490F4822700CF08CFDAD
:1016200023781549062219440DF10F000CF084FDB2
:1016300011220C4801A90CF07FFD212200210D4848
:10164000DFE71822024B0B4903481A70F3E700BF8B
:10165000A80E0020C9110020CB1600204E19002032
:10166000A911002058160020D9110020AE38002002
:101670008711002088110020A311002010B500243C
:10168000124B21461C70124B21221C70114B124828
:101690001C70124B1C70124B1C70124B1C70124BA6
:1016A0001C70124B1C70124B1C70124B1C700BF0F8
:1016B00089F82146092210480BF084F82146BDE83C
:1016C000104011220D480BF07DB800BF870E00209E
:1016D00086110020DB110020CB160020DE11002037
:1016E000DD110020DC11002006100020890E0020F2
:1016F000A90E0020A80E00204E1900205816002028
:1017000070B59D4B1A786AB901220A219B481A705C
:1017100001F002F964219A4801F0FEF81421994879
:1017200001F0FAF8984C2378042B08D8013B032BDE
:101730000DD8DFE813F063008900B800BE00202B4D
:1017400000F0BD80212B00F0DF8000232EE08F4BC6
:101750001A78022A3BD1002201251A708C4B8D4E3B
:101760001D708D4B32781D7073781B0243EA024363
:10177000B2781343894A1360894A126893421CD194
:1017800088480BF00DF83146092287480CF0D4FC4C
:1017900086480BF005F8844801F018F8014638B186
:1017A000834B84481D700AF0FBFF2023237003E065
:1017B00081480AF0F5FF257070BD7D4B7F481D7094
:1017C0000AF0EEFF6D4801F0AFF80423EEE77C4A23
:1017D0001378012BF0D1002111706F4A1370794BEF
:1017E0001D78012D06D178480AF0DAFF0222684BF5
:1017F0001A70E0E775480AF0D3FFE6E7644E744DCF
:101800003378012B1BD1734A624913700922724845
:101810002A700CF091FC3278704B6F491A702A785C
:101820006F4B70481A7021220CF086FC6E4B1B78AF
:10183000002BCAD0534801F077F80323B6E7022BF8
:101840001CBF04232370E6E74D4801F073F808B18C
:101850006648D0E7664B1A78012AADD11870654BFF
:101860001D78012D07D0022D0FD0002DE2D1624846
:101870000AF096FFDEE761480AF092FF444B1B78BE
:10188000022BD7D1534B1D70D4E7414B1B78012B52
:1018900005D1454800F0BCFF00F07AFFCAE7022BF3
:1018A000C8D15748E4E7374801F044F800288CD104
:1018B00082E70023354A1370464A137076E70922FF
:1018C000434D344944482A700CF036FC304B4249B1
:1018D0001A78424B43481A702A78414B1A702122D9
:1018E0000CF02AFC41F25D22464B00201A800ECB00
:1018F000FEF710FE44480AF053FF212323702048CE
:10190000BDE8704001F010B81D4801F013F8002840
:101910007FF45BAF364B1A78012A7FF44DAF187015
:10192000344B1D78012D06D0022D1AD0002D7FF4E6
:101930004CAF31485FE731480AF032FF144B1B7857
:10194000012B08D131480AF02BFF174800F084FF23
:1019500000F01EFF39E7022B7FF437AF1D4B1D70DF
:1019600033E70B4B1B78012B01D1294843E7022BAE
:101970007FF42BAF22483EE7700F0020680F002055
:10198000600F0020580F0020540F00208611002007
:10199000530F0020C911002092100020200E0020BB
:1019A0005C0E00200F220108BC2400202022010828
:1019B0008F1000202D2201084E220108612201080B
:1019C000600E0020560E0020742201088D220108AE
:1019D000A80E0020610E0020CB1600209E0E0020D5
:1019E0009D0E0020221900207B110020B02201084A
:1019F0008B0E00208A0E0020C3220108DE2201087F
:101A0000F12201086C19002006230108182301089F
:101A10002B23010838B5114B1A78012A1AD100225C
:101A20000F4C104821781A700AF0BAFE23780E4C39
:101A3000002B14BF0123002323700CD104F0EEFA15
:101A40000A4D22782B789A4204D009480AF0A8FE61
:101A500023782B7038BD04F0A5FAF1E7980E00202A
:101A6000010E002042230108050000200400002090
:101A70005323010870B5174B1A78012A28D1164C48
:101A800023789BB10F2B88BF0222144D144E88BFC0
:101A900003F00F0311202B703270FFF76FFB3278C9
:101AA000297810480AF07CFE002323700E4C23781E
:101AB000012B0DD103230A4D11202B70FFF75EFB84
:101AC000064B2A78197807480AF06AFE002323702B
:101AD00070BD00BF230000204C280020081000200B
:101AE000071000206C2301080910002010B5154BC9
:101AF000154C1978154B1A788A4207D001222270AA
:101B0000134A1448117019700AF04AFE124B1978E2
:101B1000124B1A788A4208D00120114A19701070AD
:101B2000104A114811700AF03BFE2378012B03D0B4
:101B30000B4B1B78012B04D1BDE810406620FFF74A
:101B40001DBB10BDE70E0020E50E0020520F002047
:101B5000E00E00208D230108E60E0020510F00202A
:101B6000E40E0020DF0E0020AB2301082DE9F04732
:101B70008C4B86B01A781ABB01220A218A481A7047
:101B800000F0CAFE0F21894800F0C6FE4FF4FA614A
:101B9000874800F0C1FE1E21864800F0BDFE64218A
:101BA000854800F0B9FE1421844800F0B5FE1E21DE
:101BB000834800F0B1FE40F6B831824800F0ACFE38
:101BC000814C2378112B15D8112B1DD8DFE813F089
:101BD00031006000B802E0022C032E0342031C0017
:101BE0001C001C001C001C001C001C001C001C0015
:101BF0004B034803302B00F0768307D8202B00F0EE
:101C00003D83212B00F053830023B6E2312B00F0FB
:101C10007683662BF8D1674800F08CFE002800F030
:101C20001F836A480AF0BCFD04F0BCF9FFF726FDEB
:101C3000EAE7674A1578012D40F0128300231370FC
:101C4000644A28461570644A1370644A1370644AE3
:101C50001370644A1370644A1370644A137008F076
:101C6000C1FE04F005FA62480AF09AFD614B624831
:101C70001D70624B1D700AF093FD4C4800F054FE3D
:101C80004B4800F051FE4E4800F04EFE2570E7E252
:101C9000474800F04FFE58B100232370FFF7EEFCD9
:101CA00004F080F9564806B0BDE8F0470AF078BD68
:101CB0004E4D2B786BB9424800F03CFE48B1514B79
:101CC0001B78012B0CBF0220062008F08BFE01239D
:101CD0002B704D4B1A78012A04D1002234481A7017
:101CE00000F022FE494B1A78012A0ED10022484DFD
:101CF0001A70287804F06EFA6020FFF73FFA2B780C
:101D0000062B02D1032008F06DFE424B1A78012AFF
:101D100009D100221A7005232370284806B0BDE8B7
:101D2000F04700F001BE2C4B1A78012A40F098824F
:101D3000002239481A700AF033FDFFF7D7FE612000
:101D4000FFF71CFA35480AF02BFD354B354D197855
:101D500035480AF025FD297834480AF021FD344B36
:101D60001B78012B18D133480AF01AFD2978324824
:101D7000FFF728FB314B1B78042B67D0052B00F0B5
:101D8000F7802F480AF00CFD01222E4B1A700B48E9
:101D900000F0CAFD0523F0E127492B480AF000FDB9
:101DA000E8E700BFB40F0020AC0F0020A40F002014
:101DB0009C0F0020940F00208C0F0020840F002027
:101DC0007C0F0020740F0020720F00202E260108C7
:101DD000A50E002092100020720E0020730E00202D
:101DE0009C0E00209A0E00209B0E0020710F0020F8
:101DF000C9230108880E0020EF230108890E002066
:101E00000A24010822000020750E0020710E002017
:101E1000700E0020620E00202324010844240108D3
:101E2000A70E0020A60E00206124010870240108DE
:101E3000A90E00207E2401080D1800201D0000209E
:101E40007C250108E90F00208B240108A74D288874
:101E50000FF02EFDA6490FF037FE0FF043F9A54B0A
:101E6000064618780F460FF023FD0FF03BF9CDE939
:101E70000401A14B18880FF01BFD9D490FF024FEB3
:101E80000FF030F9CDE902019C4B18880FF010FDDE
:101E900097490FF019FE0FF025F93246984E3B4650
:101EA000CDE9000197480AF07BFC30880FF000FD77
:101EB0008F490FF009FE0FF015F9934B8046187803
:101EC00089460FF0F5FC0FF00DF9CDE904018F4BB9
:101ED0008F4F18880FF0ECFC85490FF0F5FD0FF0DF
:101EE00001F9CDE902018B4B18880FF0E1FC804924
:101EF0000FF0EAFD0FF0F6F842464B46CDE900013F
:101F000085480AF04DFC38880FF0D2FC78490FF074
:101F1000DBFD0FF0E7F8814B8046187889460FF01B
:101F2000C7FC0FF0DFF8CDE904017D4B18880FF0F6
:101F3000BFFC6F490FF0C8FD0FF0D4F8CDE90201E6
:101F4000784B18880FF0B4FC69490FF0BDFD0FF015
:101F5000C9F84B46CDE90001424673480AF020FC1F
:101F6000724B1B883A883188288804F053F908E7B7
:101F70005E4DDFF8B8A128880FF09AFC5C490FF09D
:101F8000A3FD0FF0AFF85B4B064618780F460FF035
:101F90008FFC0FF0A7F8CDE90401574B18880FF01C
:101FA00087FC53490FF090FD0FF09CF8CDE902013A
:101FB000524B18880FF07CFC4D490FF085FD0FF057
:101FC00091F832464E4E3B46CDE900014D480AF0AD
:101FD000E7FB30880FF06CFC45490FF075FD0FF002
:101FE00081F8494B8046187889460FF061FC0FF064
:101FF00079F8CDE90401454B454F18880FF058FC9E
:102000003B490FF061FD0FF06DF8CDE90201414B46
:1020100018880FF04DFC36490FF056FD0FF062F8AE
:1020200042464B46CDE900013B480AF0B9FB3888EF
:102030000FF03EFC2E490FF047FD0FF053F8374BE1
:102040008046187889460FF033FC0FF04BF8CDE945
:102050000401334B18880FF02BFC25490FF034FD99
:102060000FF040F8CDE902012E4B18880FF020FC4C
:102070001F490FF029FD0FF035F842464B46CDE9D8
:10208000000129480AF08CFBBAF800000FF010FCA0
:1020900017490FF019FD0FF025F8254B80461878E9
:1020A00089460FF005FC0FF01DF8CDE90401214B26
:1020B00018880FF0FDFB0E490FF006FD0FF012F827
:1020C000CDE902011C4B18880FF0F2FB08490FF014
:1020D000FBFC0FF007F84B46CDE9000142461748DC
:1020E0000AF05EFBBAF800303CE700BFC60E0020E5
:1020F0000000C84221000020BC0E0020BE0E0020BF
:10210000C40E00209C24010820000020B80E0020EE
:10211000C20E0020BA0E0020D42401081F000020A7
:10212000B40E0020B60E00200C250108C00E0020C1
:102130001E000020B00E0020B20E00204425010831
:10214000904800F0F7FB002800F08A808E4B8F4A01
:102150001B88128813438E4A128813438D4A1288B3
:1021600013438D4A128813439BB243B18B480AF044
:1021700017FB8B4800F0D8FB0323237070E004208A
:1021800008F030FC04F040F986480AF009FBFEE54F
:10219000854B1A78012A3AD10022844D1A7028689A
:1021A0000FF086FB82490FF08FFC0EF09BFF814EF3
:1021B00002460B4680480AF0F3FA30680FF078FBCD
:1021C0007B490FF081FC0EF08DFF02460B467B48E9
:1021D0000AF0E6FA31682868814213D304F0C0F8A7
:1021E0000520FEF7CBFF2B683068C01A0FF060FBAC
:1021F0006F490FF069FC0EF075FF02460B46704800
:102200000AF0CEFA04235F48237000F08DFB644887
:1022100000F090FB20B3042008F0E4FB04F0F4F895
:1022200068480AF0BDFA76E55648F1E7664800F0DE
:1022300081FBA8B165480AF0B3FA03F0B3FE0920A8
:10224000FEF79CFFFFF71AFA0023614A1370614AF8
:10225000137092E75C4800F06DFB00287FF4D4AC6B
:1022600006B0BDE8F08700225B4B1046197804F0F9
:10227000FDF83020FEF782FF11237EE700250320C2
:102280002B462A462946009503F00EFF41F2CD0267
:10229000524B28461A800ECBFEF73CF950480AF004
:1022A0007FFA21233E48237000F03EFB35E53C4891
:1022B00000F040FB00287FF46DAD4A4B1A78012AEC
:1022C000CED11870484B1B78012B08D147480AF033
:1022D00067FA474800F0C0FA00F05AFA5AE5454854
:1022E0000AF05EFA56E541F231123C4B00201A80AA
:1022F0000ECBFEF70FF931233F4823700EE5394F1F
:102300003B78012B04D1002302203B70FEF736FFFF
:10231000FFF7F4F80546F0B10021384B384E19604C
:10232000314B092230703748197039700AF04AFA77
:102330003078FFF735F93278334B34491A70344B23
:1023400034481A78344B1A7021220BF0F5FE3023F2
:1023500032482370A7E4324E377837B931480AF053
:102360001FFAFFF78BF927707AE7234800F0E2FAAB
:1023700000283FF475AF2C480AF012FAFFF77EF9F7
:10238000357083E4940F0020C60E0020C40E002098
:10239000C20E0020C00E0020AE0E00209A250108BB
:1023A0008C0F0020BB2501089A0E0020940E0020FF
:1023B0000000C842900E0020DC250108F12501082C
:1023C000062601081B260108840F00202E2601087E
:1023D000890E0020A50E0020630E00206C1900203D
:1023E000062301089C0E002045190020182301082F
:1023F000BC2400202B230108740F00204819002062
:10240000A90E00204E190020A70E0020CB16002098
:10241000A80E00200D180020A60E00203B26010863
:102420006F0E00205026010863260108F8B52C4BDA
:102430001A7852B901224FF496712A481A7000F0A6
:102440006BFA1421284800F067FA284B284D1E78B3
:102450002B78284C1BB1012B2ED0002307E0264BF4
:102460001B78B34204D0204800F05EFA01232B70A1
:10247000224D23782A789A4208D063BB20480AF07C
:102480008FF9237823202B70FEF778FE1D4D2B78D3
:102490002BBB144800F04EFA08B301231A482B70E6
:1024A0000AF07EF92378C3B915480AF079F9BDE836
:1024B000F8402320FEF762BE0B4800F03BFA0028EC
:1024C000D6D00D4F3B78B342C7D010480AF068F918
:1024D00026703E70C1E70E48D1E70D48E5E7F8BD2C
:1024E000500F0020480F0020400F0020E30E002076
:1024F0003C0F0020E20E00203B0F00203A0F00208E
:102500008F260108390F0020B12601087626010820
:10251000A0260108054B1B685A6822B91868B0FA52
:1025200080F0400970470020704700BF5C1C00200D
:1025300070B5394B1A784AB901220A2137481A7006
:1025400000F0EAF91421364800F0E6F9354C23781A
:10255000022B50D026D843BB334B1B78012B23D101
:10256000FFF7D8FF01281FD1304B1B689A6803235F
:1025700092FBF3F303EB43039A4215D12C492D4808
:102580000AF00EF92C4B1B78022B05D02B4B1B7835
:10259000012B01D008F072FE214800F0C5F901239B
:1025A000237001E0102B2ED070BD1D4800F0C2F941
:1025B000064630B122480AF0F3F808F06FFE002317
:1025C000EEE71E4B1B78012B06D11E480AF0E8F8F7
:1025D00008F064FE0223E3E7174D2B78022BE3D1CA
:1025E00019480AF0DDF808F059FE0C482E7000F08A
:1025F0009BF91023D4E7114B1B78002BD4D113483F
:102600000AF0CEF8C6E7054800F094F90028CBD0D0
:102610000023094A1370C3E7380F0020300F002051
:10262000280F0020250F0020000F00205C1C002038
:10263000681C0020D6260108A8140020890E00205E
:10264000F326010810270108312701084E27010849
:1026500038B5364B1A7852B901220A2134481A701B
:1026600000F05AF941F27071324800F055F9324CDD
:102670002378022B46D01BD8EBB9304B1B78012BAB
:1026800018D1FFF747FF012814D12D492D480AF032
:1026900087F82D4B1B78022B05D02C4B1B78012B78
:1026A00001D008F0CBFD234800F03EF9012317E0EC
:1026B000102B31D038BD1F4800F03CF930B1244810
:1026C0000AF06EF808F0CAFD002323701F4B1B7838
:1026D000012B07D11F480AF063F808F0BFFD022361
:1026E0002370E7E7184D2B78022BE3D11A480AF044
:1026F00057F808F0B3FD00230D482B7000F014F9D3
:102700001023EDE7114B1B78002BD3D113480AF0AF
:1027100047F808F093FDC9E7054800F00BF90028D9
:10272000C8D00023084A1370DAE700BF240F002046
:102730001C0F0020140F0020110F0020000F00209C
:10274000681C00206B270108AA140020890E0020B5
:1027500086270108A1270108C0270108DB270108F7
:1027600038B5044608480D190AF01AF8AC4204D1ED
:10277000BDE8384004480AF013B814F8011B0348B8
:102780000AF00EF8F2E700BFE9200108D1210108A4
:1027900070B50A4B0A4D1A7829780A480AF000F8F1
:1027A0000024094E2B78E0B2834200D870BD10217E
:1027B00006EB0010FFF7D4FF0134F3E7B60F00205B
:1027C000B50F0020F62701087C1E0020F0B50E4B47
:1027D0001A787AB100230D494C1E451E01F10F06EF
:1027E00014F801CF15F8017FBC4505D1B442F7D1EB
:1027F0000133DAB21046F0BD0133DCB2A24201F17E
:102800001001E9D80022F5E7B50F00207C1E00205A
:1028100038B50E4C014625780D48102200EB051006
:102820000BF08AFC22780B490132D2B2632A227063
:1028300088BF00220B7888BF22700133DBB2632B84
:102840000B7084BF64230B7038BD00BFB60F00202F
:102850007C1E0020B50F0020F0B5044685B0102284
:10286000FF21684609F0AEFF2046FFF7AFFFA0B199
:1028700001380F4EC4B20F4D06EB04102B78013B0C
:10288000A3420CDC102206EB031069460BF054FC4B
:102890002B78094A013B2B70137005B0F0BD00F195
:1028A0001007102239460BF047FC01343846E5E7A3
:1028B0007C1E0020B50F0020B60F002038B505465D
:1028C0000C4645F2555009F09FF8284609F0A2F849
:1028D000204609F0A5F809F0A9F8BDE8384009F04C
:1028E000ADB8000008B50A4B1A782AB901220521B3
:1028F00008481A7000F010F8064800F01BF830B1D4
:10290000044800F011F8BDE8084009F08FB808BD90
:10291000C00F0020B80F0020024B41601B6803600D
:10292000704700BFC40F0020014B1B680360704755
:10293000C40F0020044B02681B6840689B1A834246
:1029400034BF002001207047C40F0020044B1A68D8
:10295000D0E90030184490428CBF801A00207047A4
:10296000C40F002030B50C46012185B0054608464D
:1029700008F020FE002301A94FF08040ADF80A3096
:10298000ADF80630ADF80850ADF8044008F02CFF63
:10299000012241214FF0804008F077FF01214FF0E4
:1029A000804008F069FF034B6846009308F0E2FCA2
:1029B00005B030BD1C00030108B501214FF0804077
:1029C00008F06EFF18B1054A136801331360012146
:1029D000BDE808404FF0804008F06EBFC40F0020F3
:1029E00030B5054685B00C460220012108F0E2FD15
:1029F000002301A90D48ADF80A30ADF80630ADF856
:102A00000850ADF8044008F0EFFE012241210748CC
:102A100008F03BFF0121054808F02EFF044B6846F3
:102A2000009308F0A7FC05B030BD00BF00040040D3
:102A30001D02020108B501210D4808F031FF58B10F
:102A40000C4B1B78012B07D10B4B1B7853B900F0B3
:102A50000BFD08B1094B18700121BDE8084004487E
:102A600008F02ABF012BF7D100F09AFDF1E700BF73
:102A700000040040E80E0020230000204C28002025
:102A800030B50C4685B005460121042008F092FDC2
:102A9000ADF80440002401A90C48ADF80850ADF889
:102AA0000A40ADF8064008F09FFE01224121074888
:102AB00008F0EBFE064B6846009308F05BFC2146ED
:102AC000024808F0D9FE05B030BD00BF0008004044
:102AD0001E02020108B50121054808F0E1FE28B1F7
:102AE000BDE808400121024808F0E6BE08BD00BF6D
:102AF0000008004030B50C4685B00546012108208D
:102B000008F058FDADF80440002401A90C48ADF8C8
:102B10000850ADF80A40ADF8064008F065FE012205
:102B20000748114608F0B1FE064B6846009308F0CE
:102B300021FC2146024808F09FFE05B030BD00BFD1
:102B4000000C00403203020108B501210A4808F0D8
:102B5000A7FE80B1094A0121138807486FEA434361
:102B60006FEA5343138008F0A7FEBDE80840002138
:102B7000014808F081BE08BD000C0040C80F0020CD
:102B800010B5012186B0044644F2040008F006FDA9
:102B9000194808F033FD194B69461948009308F0AD
:102BA00026FC4FF48063ADF80030042369461448D6
:102BB0008DF8033008F01BFC4FF4402302940024EE
:102BC00002A90D48CDE90343ADF8144008F064FDB7
:102BD0000C4B01A8019308F0CDFB012240F22551D6
:102BE000054808F0AEFD0121034808F0A1FD064BA1
:102BF0001C8006B010BD00BF003801400002031861
:102C00000008014025010201C80F002038B540F23C
:102C10002551114808F0C8FDB0B10F4808F0B7FDC4
:102C20000E4C054623887F2B0FD800210C4808F056
:102C300035FE23881BB90121094808F01DFE2388B1
:102C40005A1C2280074AD55438BD6FEA43436FEAC5
:102C500053432380F8E700BF00380140C80F00202D
:102C6000000C0040CC240020014608B5044808F0C0
:102C70008AFD4021024808F08EFD0128F9D108BDE7
:102C80000038014038B50D1804464021054808F0C9
:102C900088FDAC4200D138BD14F8010BFFF7E4FF0A
:102CA000F7E700BF0038014010B5012186B00446A7
:102CB000042008F073FC01214FF4003008F07AFC86
:102CC000164B69461648009308F091FB0823ADF8AF
:102CD00000300423694612488DF8033008F087FB62
:102CE00000234FF4402202A90E48CDE90332ADF88B
:102CF0001430029408F0D0FC0B4B01A8019308F0AB
:102D000039FB012240F22551064808F01AFD012145
:102D1000044808F00DFD06B010BD00BF0400031804
:102D2000000801400044004026000001014608B5AB
:102D3000044808F028FD4021024808F02CFD012835
:102D4000F9D108BD0044004038B50D1804464021B3
:102D5000054808F026FDAC4200D138BD14F8010B3F
:102D6000FFF7E4FFF7E700BF00440040F0B5304B49
:102D70001A78092A5AD8DFE802F0050A59131B24E9
:102D80002C394E54FE280AD101221A7007E0FE2881
:102D900005D068284AD103221A70264B1870F0BD5E
:102DA000254A244910700A7802440A700422ECE78C
:102DB00068283BD105221A701E4A137868331370B5
:102DC000EDE71D4A1B4950700A7802440A7006223A
:102DD000DBE7194A174990700A7802440A70174ACB
:102DE000107008B90822D0E70722CEE7134E144C22
:102DF000104D367822782978013EB2420E4E02F10B
:102E000003070144F055297002DA01322270C6E747
:102E100000222270E6E7074A1278824206D1092290
:102E2000B3E7162802BFFD21064A11700022ACE765
:102E3000CD0F0020CC0F00204C250020CB0F002010
:102E4000CA0F0020CE0F002008B540F225510648D9
:102E500008F0AAFC38B1044808F099FCBDE8084025
:102E6000C0B2FFF783BF08BD0044004030B5012168
:102E700091B00446082008F091FB01214FF4802016
:102E800008F098FB2C4808F0B9FB2C4B69462C48FD
:102E9000009308F0ACFA4FF40063ADF8003004235F
:102EA000694627488DF8033008F0A1FA4FF4402313
:102EB0000194002401A92048CDE90243ADF8104057
:102EC00008F0EAFB0121084608F05CFB052008F049
:102ED00013FA1C4808F0F4FC1B4B802505931B4B90
:102EE00005A90693102307934FF480531548CDE9A5
:102EF0000E34CDE90A54CDE90C44099408F05AFD8A
:102F0000294601220C4808F035FC114B05A8059311
:102F100008F030FA012240F22551074808F011FC70
:102F20000121054808F004FC0A4B21460A481C8090
:102F300008F0A2FC11B030BD0048004000040318A6
:102F4000000C01401C0002400448004058300020A2
:102F500027000001503000200008004008B540F272
:102F60002551064808F020FC38B1044808F00FFC51
:102F7000BDE80840C0B200F087BE08BD0048004070
:102F800010B504460021064808F030FD21460448EB
:102F900008F037FDBDE810400121014808F026BDCA
:102FA0001C00024010B5012186B00446102008F034
:102FB000F5FA01214FF4002008F0FCFA164B69469F
:102FC0001648009308F013FA4FF40063ADF8003090
:102FD0000423694611488DF8033008F008FA0023ED
:102FE0004FF4402202A90E48CDE90332ADF8143067
:102FF000029408F051FB0B4B01A8019308F0BAF9B9
:10300000012240F22551064808F09BFB01210448AB
:1030100008F08EFB06B010BD00040318001001403C
:10302000004C004034010101014608B5044808F095
:10303000AAFB4021024808F0AEFB0128F9D108BDE7
:10304000004C004038B50D1804464021054808F0F2
:10305000A8FBAC4200D138BD14F8010BFFF7E4FF28
:10306000F7E700BF004C0040F0B5384B1A78092A4A
:1030700008D8092A08D8DFE802F0090E07171E272A
:103080002E475C623E2A2DD0002202E0FE290AD1A2
:1030900001221A7007E0FE2905D06829F4D1032225
:1030A0001A702B4B1970F0BD0170294802780A4440
:1030B00002700422EDE76829E6D105221A70244A3D
:1030C000137868331370EEE74170214802780A44A0
:1030D00002700622DDE781701D4802780A44027002
:1030E0003E22D6E71A4CC17022780A4422708278B8
:1030F00041EA022217490A800AB90822C9E70021D9
:10310000154A11800722C4E7124F114E124D3F8815
:103110002A883478013F0C4402F1040CBA4200F8CA
:103120000C10347002DA01322A80BCE700222A80B7
:10313000E3E7074A12788A42A6D10922A9E71629AD
:1031400002BFFD21054A11709EE700BFD50F002088
:10315000D40F0020D20F0020D00F0020D60F002067
:1031600008B540F22551074808F01EFB40B105485C
:1031700008F00DFBBDE80840C1B20348FFF774BF7B
:1031800008BD00BF004C00404C27002010B50121B5
:1031900086B00446302008F001FA01214FF4801077
:1031A00008F008FA154B69461548009308F01FF916
:1031B000042369461348ADF800308DF8033008F059
:1031C00016F900234FF4402202A90F48CDE903323B
:1031D000ADF81430029408F05FFA0C4B01A801938B
:1031E00008F0C8F8012240F22551074808F0A9FA72
:1031F0000121054808F09CFA06B010BD0010031824
:10320000001001400014014000500040350201014F
:1032100008B540F22551054808F0C6FA20B1BDE8CE
:103220000840024808F0B3BA08BD00BF0050004093
:1032300007B50121092008F0B1F90121074808F07C
:103240002FF9074B01A90748019308F0D0F8102186
:10325000044808F021F903B000BD00BF00023000AF
:1032600010000310000C014008B51021034808F0BD
:1032700015F90122024B1A7008BD00BF000C014075
:10328000EA0F002008B51021034808F005F90022D4
:10329000024B1A7008BD00BF000C0140EA0F00206D
:1032A00010B5154B1A7842B9012114481970FFF76F
:1032B00033FB13211248FFF72FFB124C23781BB16D
:1032C000012B0DD0002309E0FFF7DCFF0C48FFF7CE
:1032D00031FB20B10948FFF727FB0123237010BD04
:1032E000FFF7C2FF0548FFF725FB0028F7D0044889
:1032F000FFF71AFBE6E700BFE80F0020E00F002011
:10330000D80F0020D70F002073B5482420250121B5
:10331000042008F043F90121042008F03FF90121BD
:10332000102008F03BF90121082008F037F90121AD
:10333000042008F033F90121042008F02FF90121BD
:10334000102008F02BF90121082008F027F90121AD
:10335000082008F023F90121082008F01FF90121B5
:10336000102008F01BF90121102008F017F901A91D
:103370003748ADF804508DF8074008F038F880233E
:1033800001A93348ADF804308DF8074008F02FF854
:10339000ADF80450022501A92E482F4E8DF80740A4
:1033A00008F025F801A92D48ADF804508DF8074024
:1033B00008F01DF801A92648019608F018F8102118
:1033C000234808F069F8264B01A92148019308F029
:1033D0000EF840211E4808F05FF801A91D4801962B
:1033E00008F005F810211B4808F056F81D4B01A9FC
:1033F0001A48019307F0FBFF0121184808F04CF828
:103400004FF4807301A91548ADF804308DF80740DA
:1034100007F0EDFF4FF4007301A91048ADF8043038
:103420008DF8074007F0E3FF012301A90948ADF833
:1034300004308DF8074007F0DAFF064801A9ADF81F
:1034400004508DF8074007F0D2FF02B070BD00BFF6
:10345000000801400010014010000310000C014062
:10346000400003100100031070B5454B1A782AB9CB
:103470000122142143481A70FFF74EFA424E347865
:10348000032C0CD8DFE804F002274D5E20213F48D2
:1034900007F0FCFF3E4C20B9012323703370002558
:1034A00039E08021394807F0F1FF18B90223237071
:1034B0000123F3E72021374807F0E8FF08B9032389
:1034C000F5E70221344807F0E1FF08B90423EEE7ED
:1034D00000232370E3E720212C4807F0D7FF88B1B1
:1034E00080212A4807F0D2FFB8B12021294807F0EF
:1034F000CDFFA0B10221284807F0C8FFB0FA80F440
:103500006409A400224B1D78A54236D102231D4830
:103510003370FFF709FA284670BD0224F2E703244E
:10352000F0E71848FFF706FA60B1194B1D786B1EDB
:10353000032B4FF0030396BF05EB05150025EDB2F5
:103540003370E8E72021114807F0A0FF0128A6D139
:1035500080210E4807F09AFF0128A0D120210D48B4
:1035600007F094FF01289AD102210B4807F08EFF43
:10357000012894D10122094B1A7000238EE700BF65
:1035800004100020FC0F0020FA0F0020000801406A
:10359000F90F002000100140000C0140091000202C
:1035A00038B5344B1A782AB90122142132481A70DE
:1035B000FFF7B2F92021314807F068FF8021054666
:1035C0002F4807F063FF202144002D4807F05EFFDD
:1035D00044EA85042B4D20432B782B4CC0B220703D
:1035E000032B13D8DFE803F002142842274A60B106
:1035F000411E042904D8DFE801F004040404040097
:103600001846012310702B7000E0107000240DE0AC
:103610001E4B68B1421E042A00D900201C78844247
:1036200008D1022314482B70FFF77EF9204638BDDD
:103630001870F2E70023E6E70F48FFF77BF960B167
:10364000124B1C78631E042B4FF0030396BF04EB50
:1036500004140024E4B22B70E8E72378002BD5D1C2
:10366000002301222B700A4B1A70CFE70028F7D0F5
:10367000CCE700BFF80F0020F00F00200010014041
:1036800000080140EC0F00200A100020EB0F002082
:1036900009100020013803280FD8DFE800F00206E7
:1036A000080B1021054807F0F9BE4021FAE7102168
:1036B0000348F8E701210348F5E770470008014097
:1036C00000100140000C0140013803280FD8DFE84A
:1036D00000F00206080B1021054807F0DDBE40216E
:1036E000FAE710210348F8E701210348F5E770479E
:1036F0000008014000100140000C01400421014875
:1037000007F0CABE000C014007B50121082007F0F0
:1037100045FF074B01A90748019307F068FE042104
:10372000044807F0BBFE0122034B1A7003B000BD32
:1037300004000310000C01409310002008B1FFF7B3
:10374000DDBF0421014807F0A9BE00BF000C014005
:1037500038B5954B1A784AB90122022193481A705C
:10376000FFF7DAF808219248FFF7D6F8914C237852
:10377000012B40D0022B53D0002B4DD18E4B1D7806
:10378000012D05D1FFF7BAFF8848FFF7CDF8257066
:103790008A4B1A7842B9012189481970FFF7BCF8A1
:1037A00002218848FFF7B8F8874C2378012B3ED0D8
:1037B000022B51D0002B4BD1844B1D78012D05D10C
:1037C000FFF79CFF7E48FFF7AFF82570804B1A7813
:1037D0002AB9012202217F481A70FFF79DF87E4C1A
:1037E0002378002B3FD0012B5CD00020FFF7A6FFF1
:1037F0000023237042E06D48FFF79CF840B10020A1
:10380000FFF79CFF6A48FFF78FF802232370BFE79A
:10381000694B1B78002BBBD10020FFF78FFF04E022
:103820006348FFF787F80028F2D00023EEE76448EA
:10383000FFF780F840B10020FFF780FF6148FFF7F5
:1038400073F802232370C1E7604B1B78002BBDD1B6
:103850000020FFF773FF04E05A48FFF76BF80028D9
:10386000F2D00023EEE75D4A1578012D06D11370E2
:10387000FFF744FF5748FFF757F82570584B1A7861
:103880002AB90122142157481A70FFF745F8564CFF
:1038900023786BB1012B35D00020FFF74FFF0023B9
:1038A000237010E04B48FFF745F80028E6D09CE76E
:1038B0004E4A1578012D06D11370FFF71FFF4948B6
:1038C000FFF732F825704A4B1A788AB90124494823
:1038D00021461C70FFF720F802214748FFF71CF82B
:1038E00021464648FFF718F802214548FFF714F82B
:1038F000444C2378052B00F2A880DFE803F00B2D61
:103900003B478D993748FFF715F80028C4D1FFF7DA
:10391000F5FED8E73C4B1D78012D07D100221A7027
:10392000FFF7ECFE3348FEF7FFFF2570374B1A78A0
:103930002AB90122052136481A70FEF7EDFF354CF1
:103940002378052B00F2EA80DFE813F08400A90059
:10395000B700C300D000DC002648FEF7EBFF0028CC
:10396000E4D00020FFF7EAFE2448FEF7DDFF022343
:103970002370DBE72148FEF7DDFF0028D6D0FFF7F4
:10398000BDFE1D48FEF7D0FF0323F1E71A48FEF7FE
:10399000D1FF0028CAD00020FFF7D0FE1848FEF75C
:1039A000C3FF0423E4E700BF8C1000208410002034
:1039B0007C100020791000208E100020781000204C
:1039C0007010002068100020651000208D1000206D
:1039D000641000205C10002059100020921000207C
:1039E00058100020501000204D1000209110002091
:1039F0004C100020441000203C1000203410002007
:103A00002C100020291000209310002028100020E6
:103A1000201000201D1000208248FEF78BFF002898
:103A200084D0FFF76BFE8048FEF77EFF05239FE7FB
:103A30007D48FEF77FFF00283FF478AF0020FFF7B6
:103A40007DFE0023794A137092E70020FFF776FE8F
:103A500000238DE7764B1D78012D07D100221A70C7
:103A6000FFF74CFE7348FEF75FFF2570724B1A7824
:103A70004AB90122022171481A70FEF74DFF022156
:103A80006F48FEF749FF6F4C2378092B00F2C28084
:103A9000DFE803F0495664707D8996A2AFBB6548A4
:103AA000FEF748FF0028E1D00020FFF747FE6148FD
:103AB000FEF73AFF02232370D8E75E48FEF73AFF8D
:103AC0000028D3D0FFF71AFE5A48FEF72DFF032334
:103AD000F1E75848FEF72EFF0028C7D00020FFF777
:103AE0002DFE5448FEF720FF0423E4E75148FEF77B
:103AF00021FF0028BAD0FFF701FE4E48FEF714FF61
:103B00000523D8E74B48FEF715FF0028AED000206C
:103B1000FFF714FE0023464A1370CCE70020FFF79E
:103B20000DFE0023C7E7484B1D78012D07D1002269
:103B30001A70FFF7E3FD4148FEF7F6FE257038BD29
:103B40003E48FEF7F7FE0028F9D00020FFF7F6FD0B
:103B50003A48FEF7E9FE02232370F0E73748FEF704
:103B6000E9FE0028EBD0FFF7C9FD3448FEF7DCFE84
:103B70000323F1E73148FEF7DDFE0028DFD0002007
:103B8000FFF7DCFD2D48FEF7CFFE0423E4E72B48CA
:103B9000FEF7D0FE0028D2D0FFF7B0FD2748FEF791
:103BA000C3FE0523D8E72548FEF7C4FE0028C6D08B
:103BB0000020FFF7C3FD2148FEF7B6FE0623CBE742
:103BC0001E48FEF7B7FE0028B9D0FFF797FD1B4847
:103BD000FEF7AAFE0723BFE71848FEF7ABFE002852
:103BE000ADD00020FFF7AAFD1448FEF79DFE082384
:103BF000B2E71248FEF79EFE0028A0D0FFF77EFD38
:103C00000E48FEF791FE0923A6E70C48FEF792FE48
:103C1000002894D00020FFF791FD00230A4A13707A
:103C20009AE700BF2C1000203C10002093100020C9
:103C300090100020201000201C10002014100020E4
:103C40000C1000200B1000208F1000204FF4E130EA
:103C5000FFF70CB90846FFF793B900000FB407B59A
:103C600004AA52F8041B0748019208F0EBFC05482F
:103C70000AF070FA80B2FFF783F903B05DF804EB45
:103C800004B0704758300020F8B5234D234E2B88E0
:103C9000B3F5806F38D2224C591C327889B2298012
:103CA000E05422BB631813F8013C0A2B0DD11D48C8
:103CB0000329037803F10103037004D962542046F9
:103CC000C9B201F0B5F800232B80174B1B78102BDD
:103CD0000CD12988631813F8013C3E2B06D100262D
:103CE0000F486654C9B201F0A3F82E80F8BD0F4BFF
:103CF0001B888B42FAD8002720466754C9B2FCF7CC
:103D00004FFD2F803770F1E700232B803370084878
:103D1000BDE8F84008F044BDA6100020A81000201F
:103D200050280020A21000207E110020A4100020A6
:103D30001A28010801220C4B0C491A700C4B1A70FE
:103D400000230B700B490B700B490A700B4A137060
:103D50000B4A13700B4A13700B4A13700B4A137003
:103D60000B4A1370704700BF7211002073110020BE
:103D700070110020711100206F1100207B110020B4
:103D80005838002074110020751100207611002091
:103D90007A11002007B50121082007F0FFFB094B2D
:103DA00001A90948019307F022FB4FF4805106480E
:103DB00007F074FBFFF74AFF0022044B1A7003B0B0
:103DC00000BD00BF00100310000C01405838002057
:103DD0000123024A1370024A1370704772110020C7
:103DE0007011002010B51D4B1A784AB901221E210E
:103DF0001B481A70FEF790FD50211A48FEF78CFD03
:103E0000194C2378012B11D0022B1ED063B917480F
:103E100008F0C6FC4FF48051154807F03DFB1048F0
:103E2000FEF782FD01232370002010BD0C48FEF731
:103E300081FD0028F8D04FF480510D4807F02EFB8B
:103E40000848FEF771FD0223EDE70648FEF772FD14
:103E50000028E9D0002301202370E6E76C11002040
:103E6000641100205C11002059110020272801084E
:103E7000000C014038B5594B1A782AB90122642147
:103E800057481A70FEF748FD564C23780A2B13D872
:103E9000DFE803F006131D7780353E555E969E00E1
:103EA000514A1578012D07D1002313704F4A50480D
:103EB000137008F075FC257038BD0B214D4800F0DB
:103EC00073FF4748FEF730FD02232370F4E74A4BA7
:103ED00093F81F34012B04D1484808F061FC0523F6
:103EE000F3E7642B04D1464808F05AFC0A23ECE7B8
:103EF0003B48FEF71FFD0028DED04248F4E71321BF
:103F0000414800F051FF3648FEF70EFD0623DCE77E
:103F1000394B93F81F37012B04D13C4808F040FC83
:103F20000723D2E7642B03D1394808F039FC1BE0A2
:103F30002B48FEF7FFFC0028BED03648F5E71421D9
:103F4000354800F031FF2648FEF7EEFC0823BCE7B9
:103F5000294B93F87F37012B08D13048FCF72AFB17
:103F60002F49304808F01CFC0323AEE7642B01D135
:103F70002D48DAE71A48FEF7DDFC00289CD02B48D4
:103F8000D3E70C212A4800F00FFF1548FEF7CCFCC0
:103F900004239AE7184B93F87F34012B04D125486A
:103FA00008F0FEFB092390E7642B01D122489BE730
:103FB0000B48FEF7BFFC00283FF47EAF1F4893E795
:103FC00000250122084B1E481D70084B1A7070E72F
:103FD0000023054A1370054A137076E75811002034
:103FE000501100204D1100206E1100206D11002095
:103FF00091280108A728010824000020B228010800
:10400000C1280108D3280108ED2801080B2901085F
:104010001A2901082D29010848290108541C0020EB
:10402000681C0020512901085D2901087029010838
:104030008B29010898290108A9290108BD2901082F
:10404000D9290108F8B59D4B1A784AB90122642193
:104050009B481A70FEF760FC14219A48FEF75CFC3E
:10406000994C9A4D2378172B1BD8013B162B1CD843
:10407000DFE813F02A0036004900550063006C00A9
:104080008300A400BF00C800DA00EF000E016C013D
:104090008B01A001BC01C501E001EB01FF0107029A
:1040A0000C02FF2B7ED016230CE0FFF79BFE0028AE
:1040B00078D00023864A1370864A1370864A82F8A5
:1040C0004230012323706DE0844808F069FB012130
:1040D000834800F069FE7A48FEF726FC0223F1E7E8
:1040E000804B93F85F30012B04D17F4808F058FBD8
:1040F0000323E7E77248FEF71DFC002852D07B48F7
:1041000008F04EFBCFE77A4808F04AFB02217948D5
:1041100000F04AFE6A48FEF707FC0423D2E7714B21
:1041200093F8BF30012B01D10523CBE76448FEF79C
:1041300001FC002836D07048E2E703216F4800F008
:1041400033FE5F48FEF7F0FB0623BBE7654B93F8B1
:104150001F71012F0BD16A4E6A48314608F020FBCF
:104160000022694B06F8017C1A70FF23AAE7544825
:10417000FEF7E0FBB0B16548C2E7634B1A78052A49
:1041800007D900221A700422534B614883F8422059
:10419000B6E76048042100F007FE08234948237071
:1041A000FEF7C2FB2B78012B07D10026484B5A485B
:1041B0002E701E7008F0F4FA2670F8BD494B93F883
:1041C0007F31012B0AD1554808F0EAFA544808F02B
:1041D000E7FA00224C4B1A70092373E73948FEF7BF
:1041E000A9FB0028DED0484A137801331370072357
:1041F00068E705214B4800F0D7FD3148FEF794FBF6
:104200000A235FE7374B93F8DF31012B05D146498D
:10421000464808F0C5FA0B2354E72948FEF78AFB05
:104220000028BFD042486BE7374B1A780A2A07D9D3
:1042300000221A700222284B3E4883F842205FE792
:1042400006213D4800F0B0FD1E48FEF76DFB0C2333
:1042500038E7244B93F83F32012B0FD11D4B1978CF
:1042600061B163290AD0354808F09AFA344808F059
:1042700097FA0022244B1A700D2323E71148FEF70A
:1042800059FB00288ED0204A137801331370C2E7FF
:104290001D4B1A78142A07D900221A7002220E4BDD
:1042A000284883F842202BE70721274800F07CFDAF
:1042B0000448FEF739FB0E2304E700BF4C11002031
:1042C000441100203C1100203A11002072110020FE
:1042D000731100209B38002058380020F129010874
:1042E000FE29010824000020012A01080E2A0108E5
:1042F000232A0108302A0108352A01084C2A01081E
:1043000059380020542A010839110020622A010876
:10431000772A01089E2A0108352C0108A72A0108DE
:10432000B92A0108C92A010882380020D22A0108C6
:10433000E12A0108FA2A01083B280108152B010887
:104340002B2B0108402B0108612B0108564B93F8D9
:104350009F32012B0AD1554808F022FA544808F040
:104360001FFA0022534B1A700F23ABE65248FEF798
:10437000E1FA00283FF416AF4E4B5048197801314E
:10438000C9B2197008F00CFA76E74A4B1A780A2A73
:1043900007D900221A700322494B4A4883F8422069
:1043A000AEE60821484800F0FFFC4348FEF7BCFA9F
:1043B000102387E63C4B93F8FF32012B07D1404A8C
:1043C000424882F8423008F0EBF911237AE63A4885
:1043D000FEF7B0FA00283FF4E5AE364B37481978BF
:1043E0000131C9B2197008F0DBF9BDE7092138487D
:1043F00000F0DAFC3748FEF797FA122362E62A4B00
:1044000093F85F33012B0DD12D4B93F82930012BFD
:1044100004D1314808F0C4F9132353E6022BFBD131
:104420002E48F7E72B48FEF785FA00283FF4BAAE8E
:104430002B48EFE701222B4B26481A7000222A4B0B
:104440001A70FEF771FA14233CE6FFF713FD264BB2
:104450001A78012A03D100221A70152332E61D486A
:10446000FEF768FA00283FF49DAE204808F098F95E
:10447000F3E700220F4B1A7001221D4B1A7017230D
:1044800020E61C4808F08CF900231BE62B78012B52
:104490007FF488AE0026164B17482E701E7008F069
:1044A0007FF926707EE600BF240000206A2B0108F9
:1044B0007B2B0108391100203C110020962B0108AC
:1044C00058380020A32B0108BE2B0108C82B010877
:1044D000DD2B010844110020E62B0108F32B010815
:1044E000002C01086E1100206D1100200F2C010816
:1044F00073110020222C0108352C010870B59F4B48
:104500001A78CAB901221E219D481A70FEF704FAD2
:104510001E219C48FEF700FA64219B48FEF7FCF937
:1045200064219A48FEF7F8F914219948FEF7F4F946
:10453000C8219848FEF7F0F9974C984E23780D2B38
:1045400000F21681DFE813F00E00170040007B0038
:1045500087005800640091009E00B400BF00D500A1
:10456000F30000018E4B1D78012D19D18D4808F004
:1045700017F9257014E08C4808F012F98B4B0A21CA
:1045800093F82930022B14BF89488A4800F00CFCAC
:104590007B48FEF7C9F97F48FEF7C6F9022323706E
:1045A0003378012B0FD100258348357008F0F8F8D7
:1045B000824B25701D70824B1D707C4B1D70814B92
:1045C0001D70814B1D7070BD804B93F8BF33012B64
:1045D00004D17F4808F0E4F80523E0E7642B04D118
:1045E0007C4808F0DDF80C23D9E76548FEF7A2F90E
:1045F0000028D5D07848F4E7784808F0D1F80C21A5
:10460000774800F0D1FB5E48FEF78EF90623C6E737
:104610006E4B93F87F24012A04D1724808F0C0F849
:104620000323BCE793F81F34642B01D16E48D8E70D
:104630005348FEF77FF90028B2D06C48D1E76C48A8
:1046400008F0AEF80B216B4800F0AEFB4C48FEF7CB
:104650006BF90423A3E75D4B93F81F34012BE3D1DF
:10466000654808F09DF8072399E7644808F098F832
:1046700063480D2100F098FB082341482370FEF7A2
:1046800053F98DE7514B93F8DF34012B04D15D488A
:1046900008F086F8092382E7642B01D15A48A0E785
:1046A0003748FEF747F900283FF47AAF574898E7B4
:1046B000574808F075F857480E2100F075FB0A239B
:1046C00031482370DBE7414B93F83F35012B04D190
:1046D000514808F065F80B2361E7642B01D14F487E
:1046E0007FE72948FEF726F900283FF459AF4C48E8
:1046F00077E70123314A4B481370314A13704A4A15
:10470000118819444FF6FF7389B299420ABF0223F8
:104710000B461946138008F043F80023294A13700A
:10472000294A13700122214B1A700D2337E73F48A5
:1047300008F036F8244B3E4819780131C9B2197097
:1047400008F02EF800232AE73378012B7FF43BAFE3
:1047500000251948357008F023F8184B1D70184BC8
:104760001D70124B1D70174B1D70174B1D7000E70D
:10477000304808F015F8FFF72BFB11E7381100203F
:1047800030110020281100202011002018110020D5
:1047900010110020081100200511002070110020C8
:1047A000731100204C2C0108672C01085838002098
:1047B0007D2C0108972C0108862E01087B11002012
:1047C00071110020751100207611002024000020B6
:1047D000B22C0108C12C0108D32C0108F12C0108CE
:1047E0008B290108FC2C0108092D0108202D010846
:1047F000412D0108A7280108522D0108652D010847
:10480000742D01087E2D01088F2D0108A82D0108A7
:10481000C72D0108DE2D01080B2E0108182E0108F6
:10482000252E0108352E010878110020552E01088B
:104830006A2E01089F2E010870B5994B88B01A782E
:10484000FAB901224FF4167196481A70FEF764F80F
:104850004FF416719448FEF75FF81E219348FEF757
:104860005BF864219248FEF757F8C8219148FEF79B
:1048700053F832219048FEF74FF80A218F48FEF78F
:104880004BF88F4C2378142B00F2E281DFE813F011
:104890001500450054007F009400BF00D600ED00D5
:1048A000E001E001E0017501E001E0018F01D901C3
:1048B000E0019801A101B501BE018249824B0A784D
:1048C0001B78012A14D1012B04D100220A707F49E0
:1048D0000A7023707E4B1E78012E07D100257D487B
:1048E0001D7007F05DFF7C4B25701E7008B070BD19
:1048F000012BEFD16C48FEF71DF820B16A48FEF796
:1049000013F81323E5E76748FEF714F80028E1D011
:104910006448FEF709F81123DBE7704B70491A88E9
:10492000684607F0B1FD1021684600F03DFA5F4887
:10493000FDF7FAFF0223CCE76A4B93F8FF350A2B09
:1049400004D1694807F02CFF0323C2E70C2B0CD1DC
:10495000664807F025FF0122654B1A70654B1978F0
:10496000654807F01DFF0F23B3E70D2B01D1634806
:10497000EFE74E48FDF7DEFF0028ABD0604807F0B8
:104980000FFF5C4B19780131C9B21970E8E70022BA
:104990005C4B524D1A705C492A885C4809F0CCFB8C
:1049A00029885A48FFF756F9594807F0F9FE404858
:1049B000FDF7BAFF04238CE74A4B93F8FF350B2B26
:1049C00007D1544807F0ECFE3C48FDF7ADFF052346
:1049D0007FE70C2B0ED1504B5048196807F0E0FED2
:1049E0004F4807F0DDFE4F4B4F4819780131C9B2EF
:1049F0001970B6E72E48FDF79DFF00283FF46AAF17
:104A0000454B4648196807F0CBFE4848E9E73D4B5F
:104A10001B78012B07D100223A4B45481A7007F04A
:104A2000BFFE0E2355E72548FDF784FF00283FF41D
:104A300051AF00223F4B1A7006234AE73E4807F069
:104A4000AFFE3C4B1B78062B01D93C48C9E700233D
:104A50003B4A112113803B4A3B48138000F0A4F9E4
:104A60001548FDF761FF072333E71E4B93F85F26D8
:104A7000012A6FD1FF22334D314E83F85F263188F2
:104A80002A88324807F08CFE32882B889A4261D1FE
:104A90002F4807F085FE0748FDF746FF0B2318E770
:104AA00004110020FC100020F4100020EC10002065
:104AB000E4100020DC100020D4100020CC100020D6
:104AC000CA100020851100207B11002084110020D5
:104AD0006F110020D73001088311002080110020C1
:104AE000BC2E010824000020CB2E0108D92E01087D
:104AF0007411002076110020E92E0108002F010812
:104B00001B2F0108A9100020583400205830002025
:104B1000332F01084A2F0108C40F00205D2F010820
:104B20006E2F0108751100207F2F0108952F0108B5
:104B3000B42F0108C9100020C92F0108E62F010871
:104B4000AC100020AA100020073001081530010821
:104B5000323001083F4B1B78012B3FF45CAF3E48DD
:104B6000FDF7E8FE00283FF4B5AE3C4807F018FE1C
:104B70003B4A1378013313705EE7364B1B78012BE9
:104B80003FF449AF3748FDF7D5FE00283FF4A2AE09
:104B90000122354B35481A7007F002FE344B354878
:104BA00019780131C9B2197007F0FAFD23E001222A
:104BB000314B1A700023314A13702D4A137088E666
:104BC00006212F4800F0F0F82E48FDF7ADFE122325
:104BD0007FE62D4B93F83F32012B06D12B4B1978F2
:104BE00019B1632901D02A48DEE72648FDF7A2FE65
:104BF00000283FF46FAE00236BE61421254800F037
:104C0000D3F82048FDF790FE142362E61E4B93F87C
:104C10007F37012B07D1204A20481370FBF7CAFCCD
:104C20001F492048C0E7642B03D11F4807F0B8FD97
:104C3000E1E71448FDF77EFE00283FF44BAE1B4829
:104C4000F4E71B4807F0ACFD01221A4B1A70D2E7BB
:104C50001948EBE7A9100020D41000204D300108BE
:104C6000C9100020DC1000208211002064300108EF
:104C7000751100207F2F010884110020761100207B
:104C80003B280108EC100020240000209B38002065
:104C90008730010848290108000F0020541C00201B
:104CA000681C0020512901085D29010870290108AC
:104CB0009930010883110020B030010808B5204B5D
:104CC0001A786AB901221E211E481A70FDF724FEC7
:104CD00064211D48FDF720FE0A211C48FDF71CFE3B
:104CE0001B4B1A78012A06D100221A481A7007F0C5
:104CF00057FDFFF71FF8184B1A78022A06D9002231
:104D000016481A7007F04CFDFFF714F8144B1A7888
:104D1000022A06D9002213481A7007F041FDFFF756
:104D200009F8114B1A78012A08D100220F481A708D
:104D300007F036FDBDE80840FEF7FCBF08BD00BF28
:104D4000C8100020C0100020B8100020B0100020B3
:104D500074110020EE30010875110020083101089F
:104D6000761100202C3101087A11002055310108FC
:104D700008B5FFF767F9FFF7C1FBFFF75DFDBDE879
:104D80000840FFF79BBF002330B5DCB2A24201D838
:104D9000002030BDC55C2DB1CC5C1CB1A54203F137
:104DA0000103F2D00120F4E76022064B1970064B94
:104DB000013902FB0133FF220146044883F85F20DA
:104DC000FEF74CBF7E11002024000020972401082C
:104DD0002DE9F843002580460E272E4639460A2045
:104DE00018F8014BFBF7D6FB303C61434FEAE479FE
:104DF00000FB0911A4FB0040013F64190144FFB20C
:104E000041EB0606FF2F2546E8D1084B320E5A74B7
:104E1000320C9A74320ADA74220E5A75220C9A7580
:104E2000220A1E75DA751C76BDE8F8835838002012
:104E300002292DE9F84F05468B464FD0964E37781C
:104E40001D2F4BD8431813F8022C0D2A03D113F849
:104E5000013C0A2B07D0102F40D1904B5B4413F834
:104E6000013C3E2B3AD160230022013F5F438C4C32
:104E700007F14108A044D3B218F80330924601323A
:104E8000002BF8D150372744DAB2BA5C9946013387
:104E9000002AF9D12846834907F012FD00283FD0A7
:104EA0002846814907F00CFDD0B1804809F052F93D
:104EB0007E49C2B22846FFF766FF78B97C4928468A
:104EC00007F0FEFC7A49013007F0FAFC013006F0E9
:104ED00070FE784B1880784B01221A70BDE8F88F6D
:104EE0002846764907F0ECFC08B1754BF4E72846F4
:104EF000744907F0E5FC20B17348BDE8F84F07F0AE
:104F00004FBC2846714907F0DBFC08B17048F4E754
:104F10002846704907F0D4FC0028DFD06E48ECE743
:104F200033785FFA8AFA013B5FFA89F9132BD5D8F7
:104F3000DFE813F014003B0047005B0066008100CF
:104F40009200A200E80021014B01360160017501C9
:104F500018028801C101F1012D0266025F4809F0C3
:104F6000F9F85E49C2B22846FFF70DFF40B960224A
:104F70003378013B02FB0343012283F85F201EE0EC
:104F8000574809F0E7F85649C2B22846FFF7FBFE3A
:104F90000028ECD0534809F0DDF85349C2B2284646
:104FA000FFF7F1FE002899D1CCE052462946404651
:104FB000FFF7E9FE0028EDD1012384F8BF303070FF
:104FC0008CE7BBF1110F89D1012384F81F31002434
:104FD00029460F224548347009F0AEF8444804745D
:104FE000BDE8F84F0130FFF7F3BE52462946404670
:104FF000FFF7C9FE0028CDD1012384F87F31DEE719
:10500000524629464046FFF7BEFE07460028C1D15A
:105010001422384805F1080109F08EF86022344B5B
:1050200083F83E7033783770013B02FB0343012263
:1050300083F85F2052E7524629464046FFF7A3FE19
:105040000028A7D101233070A81D84F83F3206F054
:10505000B0FD294B187041E7524629464046FFF7FC
:1050600092FE18B9012384F89F32A8E72348FFF77E
:105070008AFE0028F6D08DE7524629464046FFF7C3
:1050800082FE18B9012384F8FF3298E71C48FFF725
:105090007AFE0028F6D07DE77E11002050280020FF
:1050A00024000020663101086D31010872310108C9
:1050B00081310108A4100020A810002083310108CC
:1050C0007A1100208A31010898310108AA310108BB
:1050D000B2310108C6310108CF310108FE290108AB
:1050E0002A320108E2310108E8310108593800206C
:1050F00058380020823800209B380020F431010805
:10510000FF3101082846AC4907F0DAFB18B3012249
:10511000AA4BA94883F8292009F01CF80246A649A1
:10512000A74809F009F8524629464046FFF72BFEEA
:1051300000283FF41CAF4A463846FFF724FE0028FB
:105140007FF428AF60223378013B02FB03436422E3
:1051500083F85F20C2E628469A4907F0B1FB002891
:10516000E1D00222954B974883F8292008F0F2FFFE
:1051700094490246D4E7524629464046FFF703FECB
:1051800018B9012384F8BF3319E74A463846FFF7B8
:10519000FAFD00287FF4FEAE642384F8BF339DE659
:1051A000524629464046FFF7EEFD18B9012384F820
:1051B0007F3404E74A463846FFF7E5FD00287FF4D0
:1051C000E9AE642384F87F3488E652462946404697
:1051D000FFF7D9FD18B9012384F81F34EFE64A46DA
:1051E0003846FFF7D0FD00287FF4D4AE642384F85E
:1051F0001F3473E6524629464046FFF7C4FD18B9EE
:10520000012384F8DF34DAE64A463846FFF7BBFD6F
:1052100000287FF4BFAE642384F8DF345EE6524694
:1052200029464046FFF7AFFD18B9012384F83F3502
:10523000C5E64A463846FFF7A6FD00287FF4AAAE29
:105240006423F3E7012229465F48FFF79CFD18B964
:105250000A2384F8FF3541E607225C48FFF793FDF7
:1052600018B90B2384F8FF35A9E609225848FFF73F
:105270008AFD08B90C23F5E705225648FFF783FDA0
:105280000028F7D006225448FFF77DFD08B90D230A
:10529000E8E7504808F05EFF2946C2B24F48FFF7E2
:1052A00072FD00287FF41AAE60223378013B02FBC6
:1052B00003430C2261E6524629464046FFF763FD50
:1052C000F0B92846464907F0FBFA20B1023006F053
:1052D00070FC444B18802846434907F0F1FA20B18E
:1052E000013006F066FC414B188060223378013BA8
:1052F00002FB0343012283F85F2000233370EDE5B6
:105300004A463846FFF73FFD00287FF443AE64234A
:1053100084F85F36E2E5524629464046FFF733FD02
:1053200050B93349284607F0CBFA013006F041FC6A
:10533000304B1870304BCFE502223048FFF723FD89
:1053400028B9012384F8BF362B4B187037E64A463C
:105350003846FFF718FD00287FF41CAE642384F85C
:10536000BF36BBE5524629464046FFF70CFD18B94B
:10537000012384F89F3522E64A463846FFF703FDAD
:1053800000287FF407AE642384F89F35A6E55246D3
:1053900029464046FFF7F7FC18B9012384F81F3768
:1053A0000DE64A463846FFF7EEFC00287FF4F2ADE2
:1053B000642384F81F3791E50B3201085838002028
:1053C0007138002018320108233201082532010803
:1053D0002D320108E231010837320108E8310108B5
:1053E000F2310108AC10002081310108AA10002020
:1053F000882401087C1100207D1100202A32010838
:10540000524629464046FFF7BEFC002840D1012302
:1054100029493070284684F87F3707F051FA4278DE
:105420008178303A254B01F5F46102EB820201EB01
:1054300042021A8002794179303A303902EB820215
:1054400001EB42029A70C279017A303A303902EBAC
:10545000820201EB4202DA70827AC17A303A303944
:1054600002EB820201EB42021A71427B817B303AED
:10547000303902EB820201EB42025A71027C417C1C
:10548000303A02EB8202303901EB42029A7125E593
:105490000B4808F05FFE0B49C2B22846FFF773FCC9
:1054A00000287FF41BAD60223378013B02FB0344EC
:1054B000642384F85F3011E57F310108541C00201B
:1054C000E2310108E8310108F8B54B780A788E78A6
:1054D0001B0204460F4643EA024305210A201E43ED
:1054E000FBF758F802460B46304600210CF0D8FB7B
:1054F000042120700A20FBF74DF802460B46304687
:1055000000210CF0CDFB0A2200230CF0C9FB032183
:1055100062700A20FBF73EF802460B463046002137
:105520000CF0BEFB0A2200230CF0BAFB0221A27091
:105530000A20FBF72FF802460B46304600210CF0FC
:10554000AFFB0A2200230CF0ABFB0121E2700A2022
:10555000FBF720F80A2502460B46304600210CF0E6
:105560009FFB0A2200230CF09BFBB6FBF5F305FB27
:1055700013662271667107212846D7F80360FBF78E
:1055800009F836BA02460B46304600210CF088FB7B
:105590000621A0712846FAF7FDFF02460B46304669
:1055A00000210CF07DFB0A2200230CF079FB052181
:1055B000E2712846FAF7EEFF02460B46304600211C
:1055C0000CF06EFB0A2200230CF06AFB042122720D
:1055D0002846FAF7DFFF02460B46304600210CF062
:1055E0005FFB0A2200230CF05BFB0321627228465A
:1055F000FAF7D0FF02460B46304600210CF050FB74
:105600000A2200230CF04CFB0221A2722846FAF772
:10561000C1FF02460B46304600210CF041FB0A2236
:1056200000230CF03DFB0121E2722846FAF7B2FF9D
:1056300002460B46304600210CF032FB0A220023C2
:105640000CF02EFBB6FBF5F305FB136622736673B5
:10565000FB79B3FBF5F3A373FB79B3FBF5F205FB21
:105660001233E3733B7AB3FBF5F205FB1233237479
:10567000F8BD000010B5044686B00A4601A80749E7
:1056800006F002FF621E01AB0F3413F8011B303924
:1056900002F8011FA242F8D106B010BDB53B0108C7
:1056A000002330B5421E01390F3012F8015F11F8A6
:1056B000014F904205FB04339BB2F6D10B22B3FBA2
:1056C000F2F102FB113080B20A2802D018B1C0B248
:1056D00030BD0020FCE70520FAE70000F8B51F4CBC
:1056E0001F492046FFF7F0FE1E491F48FFF7C2FF83
:1056F00020461D49FFF7D4FF237C83422CD11B4851
:1057000007F04EF827461125194E17F8011B1948C6
:1057100001F1300306F8013B013D07F041F815F0B7
:10572000FF05F2D1144807F03BF8A27B134B42B9B6
:10573000E27B012A0ED112481A7007F031F80120DD
:10574000F8BD052A06D1E27B052A03D102220D48C5
:105750001A70F2E700221A700020F1E7A911002068
:10576000C91100203E3201089D3800205E32010838
:10577000881100206D240108E9200108861100200D
:10578000693201088432010838B5044608480D1909
:1057900007F006F8AC4204D1BDE83840044806F0F2
:1057A000FFBF14F8011B034806F0FAFFF2E700BF41
:1057B000E9200108D32101082DE9F0438BB002AFA5
:1057C00020220021384606F0FDFFDFF81891212243
:1057D0000021444806F0F6FF20220021424806F04E
:1057E000F1FF4D464FF00008404E3F4C32782846BE
:1057F0003F49120906F048FE16F8012B681C1309F0
:1058000023703B4902F00F0206F03EFE16F8013C01
:1058100008F1020803F00F03B8F1200F637005F1DF
:10582000020504F10204E1D1002399F80020462A80
:1058300038D1304A13702F4C2F48217806F0B0FF32
:1058400021782948FFF7A0FF26492C4806F0A8FF39
:105850002278A2F10A030A2B42D8002438462149B3
:1058600008F06AFC3846ADF8044008F073FC431EAB
:1058700003F0010348BF5B421D464FF00A08C6B261
:105880003744AEB90A2394FBF3F203FB124424BB62
:1058900003221B4B1B481A7006F082FF01200BB03D
:1058A000BDE8F0830133202B09F10109BDD1C2E726
:1058B00017F8013D01A88DF8043006F07AF906F0DA
:1058C00001039D4208BF400090FBF8F208FB120064
:1058D00014440444701EC6B2D3E70B4806F060FFC0
:1058E0000020DCE788110020A9110020C911002048
:1058F0009F32010887110020A4320108B13201084B
:1059000086110020BD320108CE3201082DE9F04198
:10591000254C23787A2B45D163786C2B42D12122F8
:1059200000212248224D06F04DFF20220021204870
:1059300006F048FF0027A8461C4E227830461D4935
:10594000120906F0A1FD14F8012B701C13092B702D
:10595000184902F00F0206F097FD14F8013C0237D7
:1059600003F00F03202F6B7006F1020605F102050C
:10597000E3D10A2198F8043098F805200E4801FB7D
:10598000032203320D4B5200D2B208491A7006F0BE
:1059900007FF03220A4B0B481A7006F001FF012093
:1059A000BDE8F0810020FBE7C9110020881100202C
:1059B000A91100209F320108DD3201088711002063
:1059C00086110020F332010807B50121052005F0FA
:1059D000E5FD064B01A90648019305F008FD4FF4CB
:1059E0000041034805F058FD03B000BD00800310DE
:1059F0000008014008B5FFF771FE20B10848BDE876
:105A0000084006F0CDBEFFF7D7FE08B10548F6E71F
:105A1000FFF77CFF08B10448F1E70448EFE700BF57
:105A20000A33010819330108263301083533010808
:105A300008B5C82005F07AFC08210748FDF722F9CF
:105A4000C82005F073FC05481521FDF71BF9BDE8DA
:105A50000840C82005F06ABC790B0020640B0020C8
:105A600038B506F02DFF08B9002038BD0F4906F003
:105A700027FF0028F8D0441C204608F06BFB431E8B
:105A80001B06F1D40A4D802200212870094806F037
:105A900099FE21462A78074808F04EFB054A2978E6
:105AA000054806F07DFE0120DFE700BF4233010814
:105AB000D9110020AE38002044330108F8B504465F
:105AC00008F048FB234685B2002061198B4219D1AA
:105AD000204608F03FFB294682B22B4806F060FEC4
:105AE0002A49204606F0ECFE0646204608F032FB26
:105AF0007F280FD9264806F053FEBDE8F840254818
:105B000006F04EBE1A780D2A01D00A2A00D118706C
:105B10000133DBE7DEB1304608F01CFB01221E4BEF
:105B20001E4FC5B231461A7038702A461C4808F01C
:105B300003FB00231A4A1B48535506F031FE18494F
:105B4000194806F02DFE3978184806F029FE20463F
:105B50001749FFF785FF174D074628B1164806F08D
:105B60001FFE01232B70F8BD204608F0F3FA0B4E00
:105B70003946307080220A4806F024FE21463278E9
:105B8000074808F0D9FAECE75833010869330108EF
:105B90007133010880330108DA110020D911002087
:105BA000AE38002095330108A6330108B43301084C
:105BB000C5330108DE110020E733010810B51B4B87
:105BC0001A7852B90122642119481A70FCF7A4FE10
:105BD0004FF496711748FCF79FFE1548FCF7AAFE94
:105BE00010B11348FCF7A0FE134B144C1A78144B59
:105BF00010481B789A4238BF1A46124B1B789342C2
:105C000038BF13462370FCF795FE70B10948FCF7C6
:105C10008BFE20780BF04CFE0BF064FABDE81040D0
:105C200002460B46084806F0BBBD10BDF01100202F
:105C3000E8110020E0110020F3110020F4110020F1
:105C4000F2110020F1110020FC33010808B50021F9
:105C500001200C4A00F02AFD00210220094A00F030
:105C600025FD00210320074A00F020FD0021064AFF
:105C7000084600F01BFDBDE8084000210220034A51
:105C800000F014BD13340108243401083534010830
:105C90001E2903460A4614D8B9B101391D2914D862
:105CA000DFE801F01513191B1D131F211323131314
:105CB0002527292B192D1313131313131313131340
:105CC000132F3F291FD0402921D0124901E0124A49
:105CD0001249184619E0124AFAE7124AF8E7124A3E
:105CE000F6E7124AF4E7124AF2E7124AF0E7124ADC
:105CF000EEE7124AECE7124AEAE7124AE8E7124AEC
:105D0000E6E7124AE4E7124A044906F0BDBB114A2D
:105D1000FAE700BF6D340108A0340108B53B010863
:105D200046340108493401084C3401084F34010855
:105D30005234010855340108583401085B34010815
:105D40005E3401086134010864340108AA34010892
:105D5000673401086A3401081E29034614D8B9B112
:105D600001391D2914D8DFE801F01513191B1D1383
:105D70001F21232323132527292B192D1313131335
:105D8000131313131313132F3F291FD0402921D0AE
:105D9000114A00E0114A1846114919E0114AFAE780
:105DA000114AF8E7114AF6E7114AF4E7114AF2E717
:105DB000114AF0E7114AEEE7114AECE7114AEAE727
:105DC000114AE8E7114AE6E7114AE4E7114A0449B3
:105DD00006F05ABB104AFAE71F3401087134010873
:105DE000B53B0108763401087B3401088034010892
:105DF000853401088A340108EC4001088F34010819
:105E000094340108993401089E340108A334010830
:105E1000A8340108673401086A34010870B50E46D9
:105E200014461D469CB000210120214A00F03EFC92
:105E3000002102201E4A00F039FC1D4A00210320E7
:105E400000F034FC314608A8FFF722FF21460DA8D8
:105E500012ACFFF71DFF2946204617ADFFF718FFCC
:105E600028469DF88010FFF713FF124B1B78042B78
:105E70000DD0052B13D0022100200F4A00F016FC94
:105E8000002102200D4A00F011FC1CB070BD0C492D
:105E900000940DAB08AA03A806F0F6FAEBE7CDE9EB
:105EA000004508490DAB08AA03A806F0EDFAE2E7A1
:105EB000133401081D000020C93401081019002006
:105EC000AD340108BA34010838B52B4B1C78F4B94D
:105ED00001250A2129481D70FCF71EFD2146284690
:105EE000274A00F0E3FB21460220254A00F0DEFBB2
:105EF00021460320224A00F0D9FB02212046214AF4
:105F000000F0D4FB214602201F4A00F0CFFB1F4BBC
:105F10001A7822BB1E4A19481278012A08BF1A7043
:105F2000FCF708FDD8B11B4C1448FCF7FDFC2378A6
:105F3000032B0DD8DFE803F002141618104A0021D5
:105F4000022000F0B3FB144A0021022000F0AEFB57
:105F500023780133DBB2032B88BF0023237038BDC5
:105F60000E4AF1E70E4AEFE7054A0021022000F051
:105F70009DFB054AE8E700BF201200201812002010
:105F800013340108D2340108DB3401081612002052
:105F90005838002015120020EC340108FD340108A7
:105FA0000E35010808B500F07DFB0021164A0846B1
:105FB00000F07CFB00210120134A00F077FB002158
:105FC0000220114A00F072FB002103200E4A00F06B
:105FD0006DFB012100200D4A00F068FB002102202A
:105FE0000B4A00F063FB032000210A4A00F05EFB2D
:105FF000094B1878431E1F2B05D8BDE80840033015
:10600000C00800F055BB08BD133401082634010850
:106010001F350108303501089B38002008B50021E4
:1060200001200F4A00F042FB002102200C4A00F040
:106030003DFB002103200A4A00F038FB022100202A
:10604000084A00F033FB00210220074A00F02EFB33
:10605000BDE8084000210320044A00F027BB00BF30
:1060600013340108413501084A3501085B35010840
:1060700008B5002101200A4A00F018FB0021022087
:10608000074A00F013FB00210320054A00F00EFB35
:10609000BDE8084000210220024A00F007BB00BF13
:1060A000133401086C3501082DE9F043002406463D
:1060B0008DB00120894615462146364A98460094FF
:1060C000149FCDF8034000F0F1FA21460220314A36
:1060D00000F0ECFA032021462E4A00F0E7FA701E89
:1060E000042840D8DFE800F0033742474C00B9F1FC
:1060F000000F2DD0694605F10A03103513F8012F62
:106100003032AB4201F8012BF8D16A46224902A88D
:1061100006F0BAF938460BF0CBFB20490BF0D4FC63
:106120000AF0E0FF0B4602461D4907A806F0ACF94D
:106130001C4B197819B901201B4A00F0B7FA02AAC2
:106140000021022000F0B2FA07AA0021032008E093
:1061500042461649DBE7164806F022FB154A0021A5
:10616000022000F0A3FA0DB0BDE8F083124806F05B
:1061700017FB124AF3E7124806F012FB114AEEE74A
:10618000114806F00DFB114A0021022000F08EFAA2
:106190000F4ADAE7133401087D3501080000C842D0
:1061A0008A350108220000209E3501089535010836
:1061B000AF350108BC350108CD350108DC350108D3
:1061C000ED350108FA3501080B36010818360108CB
:1061D0002936010810B5044686B0002103200A4A7A
:1061E00000F064FA5CB12246084901A806F04CF9B7
:1061F0000021032001AA00F059FA06B010BD04499D
:1062000001A806F041F9F3E7133401083A36010812
:106210004B360108F0B507469DB000201C460E46DF
:10622000154600F041FA0021454A084600F03EFAC2
:1062300000210120424A00F039FA00210220404AA0
:1062400000F034FA3E4A0021032000F02FFA3D4BC3
:1062500003A81978FFF780FD38460BF029FB3A496F
:106260000BF032FC0AF03EFF03AACDE900013749EA
:1062700008A806F009F9364B03A81978FFF76CFD5A
:1062800030460BF015FB30490BF01EFC0AF02AFFDC
:1062900003AACDE900012D490DA806F0F5F82D4B14
:1062A00003A81978FFF758FD28460BF001FB264993
:1062B0000BF00AFC0AF016FF03AACDE900012349FE
:1062C00012A806F0E1F8244B03A81978FFF744FD63
:1062D00020460BF0EDFA1C490BF0F6FB0AF002FF2A
:1062E00003AACDE90001194917A806F0CDF81B4B08
:1062F0001B78042B03D0052B11D01DB0F0BD00215D
:10630000012008AA00F0D2F90DAA0021022000F015
:10631000CDF912AA0021032000F0C8F9EDE7002111
:1063200008AA084600F0C2F9002101200DAA00F0D9
:10633000BDF912AA0021022000F0B8F917AAE9E776
:10634000133401081B0000200000C8425C3601081D
:106350001A00002019000020180000201D00002055
:1063600010B588428AB094BF081A00200C460BF082
:106370009FFA20490BF0A8FB0AF0B4FE02460B4638
:1063800068461D4906F080F820460BF091FA19493D
:106390000BF09AFB0AF0A6FE0B460246174905A829
:1063A00006F072F80021164A084600F07FF9002135
:1063B0000120134A00F07AF900210220104A00F06F
:1063C00075F9002103200E4A00F070F90221002027
:1063D0000C4A00F06BF96A460021022000F066F9D1
:1063E000002105AA032000F061F9012000F05CF90A
:1063F0000AB010BD0000C842693601088A3501089C
:106400001334010841350108002108B50846134A34
:1064100000F04CF900210120104A00F047F900215A
:1064200002200E4A00F042F9002103200B4A00F03E
:106430003DF9022100200A4A00F038F9002102202B
:10644000084A00F033F903200021074A00F02EF932
:10645000BDE80840012000F027B900BF133401084F
:106460004135010874360108853601087FB51346A9
:106470000A46F0B1114901A806F006F800210120F2
:106480000F4A00F013F9002102200D4A00F00EF926
:10649000002103200A4A00F009F900210220094ADC
:1064A00000F004F90021032001AA00F0FFF807B072
:1064B00000BD054901A805F0E7FFDFE796360108B2
:1064C00013340108B2360108A63601087FB502462A
:1064D0000F4901A805F0D8FF002101200D4A00F066
:1064E000E5F8002102200B4A00F0E0F8002103202B
:1064F000084A00F0DBF801AA0021022000F0D6F8DB
:1065000000210320044A00F0D1F807B000BD00BF0D
:10651000C336010813340108D03601087FB502469E
:106520000F4901A805F0B0FF002101200D4A00F03D
:10653000BDF8002102200B4A00F0B8F8002103202A
:10654000084A00F0B3F801AA0021022000F0AEF8DA
:1065500000210320044A00F0A9F807B000BD00BFE5
:10656000C336010813340108DF3601087FB502463F
:106570000F4901A805F088FF002101200D4A00F015
:1065800095F8002102200B4A00F090F8002103202A
:10659000084A00F08BF801AA0021022000F086F8DA
:1065A00000210320044A00F081F807B000BD00BFBD
:1065B000C336010813340108F036010870B52F4BBB
:1065C0001A7872B9012232212D481A70FCF7A4F909
:1065D00032212C48FCF7A0F94FF416712A48FCF739
:1065E0009BF92A4C2A4E2378012B1DD9022B23D04C
:1065F000284A96F842301178994205D0022B137040
:1066000033D1052000F054F8234B1878234B1A7827
:10661000824232D01870431E1F2B2ED8BDE8704026
:106620000330C00800F044B81548FCF783F900288F
:10663000DED002232370DBE7194D2B78002BD7D156
:10664000FFF742FC3378012B04D12B70FFF7AAFC33
:10665000032323700C48FCF76DF90028C8D00123F0
:106660002B70FFF79FFC0323E4E7032B01D10620E7
:10667000C8E7042BC8D10720C4E770BD141200205E
:106680000C12002004120020FC110020F811002040
:1066900058380020F61100209B380020F51100200A
:1066A000F711002000F08EB800F0D2B800F0DCB88E
:1066B00000F0F4B838B50546002405FA04F31B06CB
:1066C0004FF0400109480DD504F0E6FE20210748AF
:1066D00004F0E2FE01342021044804F0DFFE082C1F
:1066E000EBD138BD04F0DAFEF0E700BF000C01404A
:1066F00008B5FC20FFF7DEFF08BD000010B504461A
:1067000080210D4804F0C8FEFFF7F2FFF820FFF7E4
:10671000D1FF04F0F000FFF7CDFF200100F0F00002
:10672000FFF7C8FF642004F0E7FDBDE810408021BA
:10673000014804F0B3BE00BF000C014010B5044690
:1067400080210D4804F0A8FEFFF7D2FFFA20FFF7E2
:10675000B1FF04F0F000FFF7ADFF200100F0F00002
:10676000FFF7A8FF642004F0C7FDBDE810408021BA
:10677000014804F093BE00BF000C014038B534203E
:10678000FFF7BCFF3620FFF7B9FF002565F07F005B
:10679000C0B2FFF7B3FF8020FFF7B0FF2024002036
:1067A000013CFFF7CBFF14F0FF04F8D10135202D99
:1067B000ECD13620FFF7A2FFBDE838403020FFF7CC
:1067C0009DBF000007B50121082004F0E7FE01216C
:1067D000082004F0E3FE0121082004F0DFFE184B3E
:1067E00001A91848019304F002FE174B01A91548AE
:1067F000019304F0FCFD154B01A91248019304F02C
:10680000F6FD022004F092FD3020FFF777FF05200F
:1068100004F08CFD0C20FFF771FF052004F086FDCD
:106820000120FFF76BFF052004F080FD0620FFF735
:1068300065FF052004F07AFDFFF7A0FF03B000BD5F
:1068400020000310000C01404000031080000310E2
:1068500008B501280CBF36203420FFF74FFFBDE8F4
:1068600008403020FFF74ABF0023032898BF0A4B97
:1068700010B598BF1B5C14465818C0B2FFF73EFF16
:10688000013C14F8010F00B910BDFFF757FF32208B
:1068900004F032FDF5E700BF4951010838B5044660
:1068A000114D3420FFF72AFF362005EB4415FFF782
:1068B00025FF83242046FFF721FF8020FFF71EFFDE
:1068C00001342878FFF73AFFE4B26878FFF736FF23
:1068D000932C05F10205EDD13620FFF70FFFBDE83F
:1068E00038403020FFF70ABF4D51010807B501219C
:1068F000102004F053FE0121102004F04FFE01216E
:10690000042004F04BFE0121042004F047FE012185
:10691000082004F043FE0121082004F03FFE204B34
:1069200001A92048019304F062FD04211D4804F0F0
:10693000B5FD1D4B01A91B48019304F058FD08212A
:10694000184804F0ABFD194B01A91948019304F054
:106950004EFD0121164804F0A1FD164B01A9144873
:10696000019304F044FD0221114804F097FD124BFD
:1069700001A91248019304F03AFD4FF400510F4869
:1069800004F08CFD0E4B01A90C48019304F02FFD7F
:106990004FF48041094804F081FD03B000BD00BF01
:1069A0000400031000100140080003100100031050
:1069B000000801400200031000200310000C0140F9
:1069C0000040031008B5431E0146052B2CD8DFE814
:1069D00003F0030B11171D240421164804F05CFD7D
:1069E000154B01221A7008BD0821124804F054FD0D
:1069F000124BF6E70121124804F04EFD114BF0E76F
:106A000002210F4804F048FD0F4BEAE74FF4005114
:106A10000E4804F041FD0E4BE3E74FF480410B4874
:106A200004F03AFD0B4BDCE70B48BDE8084005F0ED
:106A3000B7BE00BF00100140261200202512002022
:106A4000000801402412002023120020000C014005
:106A50002212002021120020FD36010808B5431E35
:106A60000146052B2CD8DFE803F0030B11171D247A
:106A70000421164804F012FD154B00221A7008BDBF
:106A80000821124804F00AFD124BF6E701211248D2
:106A900004F004FD114BF0E702210F4804F0FEFC66
:106AA0000F4BEAE74FF400510E4804F0F7FC0E4B91
:106AB000E3E74FF480410B4804F0F0FC0B4BDCE7BC
:106AC0000B48BDE8084005F06BBE00BF0010014058
:106AD0002612002025120020000801402412002068
:106AE00023120020000C014022120020211200205D
:106AF000FD36010813B50121082004F04FFD0121E6
:106B0000102004F04BFD0121102004F047FD01216D
:106B1000102004F043FD0121102004F03FFD01216D
:106B2000042004F03BFD0121042004F037FD012185
:106B3000042004F033FD2B4B01A92B48019304F0F2
:106B400056FC4FF40041284804F0A8FC274B01A94B
:106B50002748019304F04BFC4021254804F09EFC9B
:106B6000244B01A922480193234C04F040FC8021CE
:106B70001F4804F093FC01A91D48019404F037FC60
:106B80004FF480711A4804F089FC1C4B01A9184885
:106B9000019304F02CFC4FF40071154804F07EFCC6
:106BA00001A91748019404F022FC4FF480711448A5
:106BB00004F074FC134B01A91148019304F017FC75
:106BC0004FF400610E4804F069FC0F4B01A90C481A
:106BD000019304F00CFC4FF48051094804F05EFC72
:106BE00002B010BD00800310000C014040000310F3
:106BF0000010014080000310000103100002031088
:106C0000000801400008031000100310014610B5F1
:106C1000441E1C4805F0C4FD032C0FD8DFE804F027
:106C2000020F1A264FF40041174804F037FC4021A8
:106C3000164804F031FC164B01221A7010BD802159
:106C4000124804F02BFC4FF48071104804F024FC2F
:106C5000104BF1E74FF400710C4804F01FFC4FF4A7
:106C600080710D4804F018FC0C4BE5E74FF400610F
:106C7000094804F013FC4FF48051074804F00CFC61
:106C8000074BD9E719370108000C014000100140FB
:106C90002A1200202912002000080140281200209A
:106CA00027120020014610B5441E1C4805F078FD4F
:106CB000032C0FD8DFE804F0020F1A264FF400412E
:106CC000174804F0E9FB4021164804F0E7FB164B97
:106CD00002221A7010BD8021124804F0DDFB4FF42F
:106CE0008071104804F0DAFB104BF1E74FF40071AB
:106CF0000C4804F0D1FB4FF480710D4804F0CEFB3A
:106D00000C4BE5E74FF40061094804F0C5FB4FF474
:106D10008051074804F0C2FB074BD9E72E37010822
:106D2000000C0140001001402A120020291200200E
:106D3000000801402812002027120020013810B559
:106D4000032815D8DFE800F0021524344FF4004181
:106D50001F48204C04F0A2FB40211F4804F09EFB7A
:106D600023781BB101211D4805F01AFD0023237073
:106D700010BD802118481A4C04F090FB4FF480712C
:106D8000154804F08BFB2378002BEFD00221EAE7B3
:106D90004FF400711048134C04F080FB4FF48071E5
:106DA000114804F07BFB2378002BDFD00321DAE7C6
:106DB0004FF400610C480D4C04F070FB4FF480510F
:106DC000094804F06BFB2378002BCFD00421CAE7DD
:106DD000000C01402A120020001001404337010836
:106DE000291200202812002000080140271200204C
:106DF00010B5244B1A782AB90122142122481A709E
:106E0000FBF78AFD214C2378032B38D8DFE803F009
:106E1000020D172D4FF480711D4804F037FB08B99F
:106E2000032300E00123237007E00120FFF73AFF6E
:106E3000022315482370FBF777FD002010BD124890
:106E4000FBF778FD18B10120FFF778FFE8E74FF472
:106E500080710F4804F01AFB10B90120FFF76EFF94
:106E60000C4B1B78002BDBD0E7E70B4805F098FCB8
:106E70000120FFF763FF002301202370DEE70748AE
:106E8000F4E700BF5C1200205412002051120020D1
:106E9000000C01402A120020583701087037010801
:106EA00070B5964B1A782ABB012195481970FBF7EB
:106EB00033FD03219348FBF72FFD05219248FBF793
:106EC0002BFD0A219148FBF727FD02219048FBF793
:106ED00023FD19218F48FBF71FFD10218E48FBF77A
:106EE0001BFD14218D48FBF717FD40F6B8318C4887
:106EF000FBF712FD8B4C2378092B0FD9A3F130023D
:106F0000042A01D900232CE0313B032B00F2B1808D
:106F1000DFE813F0B700C600D800DF00013B082B04
:106F200006D8DFE803F01720263650616C839A00FC
:106F30007D4E3578012D45D17C4805F031FC00238C
:106F40007B4A337013707B4A137014227A4B1A7089
:106F5000257037E06E48FBF7E7FC6E48FBF7E4FC72
:106F6000022323702EE06A48FBF7E4FC50B30323AE
:106F7000F7E7724805F014FC0120FFF747FE0423F1
:106F80006F48237005F00CFC6348BDE87040FBF7C8
:106F9000CBBC6048FBF7CEFC5F48FBF7CBFC68B18D
:106FA0000120FFF7CBFE674805F0FAFB664805F0C5
:106FB000F7FB5B48FBF7B8FC0523D2E7634B1B7874
:106FC000002BF3D070BD5A4B1A78012A03D100224E
:106FD0001A700623C5E75248FBF7ACFC0028F1D035
:106FE0005B4805F0DDFBF4E75A4805F0D9FB0120CA
:106FF000FFF758FE4948FBF797FC0723B1E74748DE
:10700000FBF798FC20B10120FFF798FE0823A8E7C2
:107010004FF48071504804F039FA10B90120FFF79D
:107020008DFE4A4B1B78002BCCD1ECE74FF48071DE
:10703000494804F02BFA404B60B132221A702022EA
:10704000464B47481A700122464B1A7005F0A8FBC0
:10705000092386E714221A70FAE700250122324B31
:1070600041481D70324B1D70324B1A7005F098FB71
:107070006EE73E4805F094FB2548FBF755FC3123AD
:107080006FE72348FBF756FC00289BD0384805F0F3
:1070900087FB0120FFF7BAFD32231948237074E7FC
:1070A0001748FBF747FC00288CD0324805F078FBE6
:1070B0000120FFF743FE332323702F48BDE87040C3
:1070C00005F06EBBFFF794FE01287FF47BAF3423FD
:1070D00047E74FF48071204804F0D8F9164B38B1D7
:1070E00032221A7020221D4B1A7001221D4BB2E76A
:1070F000142203481A70FBF717FCA9E78C13002031
:10710000841300207C130020741300206C130020D3
:10711000641300205C130020541300204C13002043
:107120004413002041130020820E00208D370108F7
:107130007E0E00207A0E0020680E0020A037010885
:10714000AC370108BE370108D03701082A120020E9
:10715000DE370108F5370108000C0140640E0020FD
:10716000033801086E0E00201D3801082B38010875
:1071700038380108453801085A38010810B5244B41
:107180001A782AB90122142122481A70FBF7C4FB8D
:10719000214C2378032B38D8DFE803F0020D172D9C
:1071A0004FF400711D4804F071F908B9032300E0A1
:1071B0000123237007E00220FFF774FD0223154826
:1071C0002370FBF7B1FB002010BD1248FBF7B2FBA8
:1071D00018B10220FFF7B2FDE8E74FF400710F4845
:1071E00004F054F910B90220FFF7A8FD0C4B1B78EE
:1071F000002BDBD0E7E70B4805F0D2FA0220FFF7BF
:107200009DFD002301202370DEE70748F4E700BF5F
:10721000501200204812002045120020000C0140AE
:1072200029120020693801088138010870B5964B91
:107230001A782ABB012195481970FBF76DFB0321D1
:107240009348FBF769FB05219248FBF765FB0A2190
:107250009148FBF761FB02219048FBF75DFB192188
:107260008F48FBF759FB10218E48FBF755FB142183
:107270008D48FBF751FB40F6B8318C48FBF74CFBCF
:107280008B4C2378092B0FD9A3F13002042A01D9A2
:1072900000232CE0313B032B00F2B180DFE813F038
:1072A000B700C600D800DF00013B082B06D8DFE896
:1072B00003F01720263650616C839A007D4E357896
:1072C000012D45D17C4805F06BFA00237B4A3370D1
:1072D00013707B4A137014227A4B1A70257037E0B2
:1072E0006E48FBF721FB6E48FBF71EFB0223237061
:1072F0002EE06A48FBF71EFB50B30323F7E7724802
:1073000005F04EFA0220FFF781FC04236F4823703A
:1073100005F046FA6348BDE87040FBF705BB6048DE
:10732000FBF708FB5F48FBF705FB68B10220FFF79E
:1073300005FD674805F034FA664805F031FA5B4808
:10734000FBF7F2FA0523D2E7634B1B78002BF3D04F
:1073500070BD5A4B1A78012A03D100221A700623F5
:10736000C5E75248FBF7E6FA0028F1D05B4805F084
:1073700017FAF4E75A4805F013FA0220FFF792FCD7
:107380004948FBF7D1FA0723B1E74748FBF7D2FAA0
:1073900020B10220FFF7D2FC0823A8E74FF40071C8
:1073A000504804F073F810B90220FFF7C7FC4A4BAD
:1073B0001B78002BCCD1ECE74FF40071494804F066
:1073C00065F8404B60B132221A702022464B474884
:1073D0001A700122464B1A7005F0E2F9092386E77C
:1073E00014221A70FAE700250122324B41481D7021
:1073F000324B1D70324B1A7005F0D2F96EE73E48E1
:1074000005F0CEF92548FBF78FFA31236FE72348C3
:10741000FBF790FA00289BD0384805F0C1F902200C
:10742000FFF7F4FB32231948237074E71748FBF782
:1074300081FA00288CD0324805F0B2F90220FFF71B
:107440007DFC332323702F48BDE8704005F0A8B9B8
:10745000FFF794FE01287FF47BAF342347E74FF416
:107460000071204804F012F8164B38B132221A701D
:1074700020221D4B1A7001221D4BB2E71422034833
:107480001A70FBF751FAA9E74013002038130020C7
:107490003013002028130020201300201813002090
:1074A000101300200813002000130020F812002001
:1074B000F5120020810E00209E3801087D0E00206C
:1074C000790E0020670E0020B1380108BD38010890
:1074D000CF380108E138010829120020EF380108EF
:1074E00006390108000C0140640E0020143901081F
:1074F0006D0E00202E3901083C3901084939010878
:10750000563901086B39010810B5234B1A782AB98E
:107510000122142121481A70FBF7FEF9204C237830
:10752000032B36D8DFE803F0020C162B01211D488F
:1075300003F0ACFF08B9032300E00123237007E048
:107540000320FFF7AFFB022314482370FBF7ECF98D
:10755000002010BD1148FBF7EDF918B10320FFF72B
:10756000EDFBE8E701210F4803F090FF10B903207D
:10757000FFF7E4FB0C4B1B78002BDCD0E8E70B4853
:1075800005F00EF90320FFF7D9FB0023012023703B
:10759000DFE70748F4E700BF441200203C12002058
:1075A0003912002000100140281200207A39010809
:1075B0009239010870B5984B1A782ABB0121974877
:1075C0001970FBF7A9F903219548FBF7A5F90521E7
:1075D0009448FBF7A1F90A219348FBF79DF90F2185
:1075E0009248FBF799F919219148FBF795F90F217A
:1075F0009048FBF791F914218F48FBF78DF940F67D
:10760000B8318E48FBF788F98D4C2378092B0FD9B8
:10761000A3F13002042A01D9002330E0313B032BCF
:1076200000F2AF80DFE813F0B800C700DC00E20032
:10763000013B082B06D8DFE803F018242B3B5F6FD3
:107640007A9098007F4E3578012D40F085807E48F5
:1076500005F0A6F800237D4A337013707C4A13703E
:1076600014227C4B1A70257076E00320FFF7AAF9EC
:107670006E48FBF759F96E48FBF756F90223237061
:107680006AE06A48FBF756F9002865D00323F6E75D
:10769000714805F085F80320FFF7B8FA04236F4816
:1076A000237005F07DF86348BDE87040FBF73CB9F6
:1076B0005F48FBF73FF910B10320FFF7CFF95D48B2
:1076C000FBF738F980B10320FFF738FB0320FFF701
:1076D000C5F9634805F064F8624805F061F8574859
:1076E000FBF722F90523CAE75F4B1B78002B33D148
:1076F0000320FFF7B3F9EFE7544B1A78012A03D1BF
:1077000000221A700623BAE74C48FBF713F918B3A6
:10771000564805F045F8F5E7554805F041F80320CF
:10772000FFF7C0FA4448FBF7FFF80723A7E74248F2
:10773000FBF700F920B10320FFF700FB08239EE7C9
:1077400001214C4803F0A2FE10B90320FFF7F6FA1E
:10775000454B1B78002BEED070BD0121454803F04E
:1077600095FE002850D0302389E700250122354BB3
:1077700041481D70354B1D70354B1A7005F010F8DF
:1077800071E73E4805F00CF80320FFF71BF9274886
:10779000FBF7CAF8312372E72448FBF7CBF800283F
:1077A000DAD0374804F0FCFF0320FFF72FFA32232A
:1077B0001A48237078E71948FBF7BCF80028CBD0AB
:1077C000304804F0EDFF0320FFF748F90320FFF7EE
:1077D000B5FA332323702C48BDE8704004F0E0BFB5
:1077E000FFF792FE0128B7D1342348E70121214851
:1077F00003F04CFE174B48B132221A702022234B63
:107800001A700122224B1A70092338E71422034808
:107810001A70FBF789F8F7E7F4120020EC12002049
:10782000E4120020DC120020D4120020CC12002030
:10783000C4120020BC120020B4120020AC120020A0
:10784000A9120020800E0020AF3901087C0E002014
:10785000780E0020660E0020C2390108CE390108DA
:10786000E0390108F239010828120020003A010825
:10787000173A010800100140253A0108333A01087F
:10788000403A01084D3A0108623A0108640E0020AE
:107890006C0E002010B5234B1A782AB9012214214E
:1078A00021481A70FBF738F8204C2378032B36D880
:1078B000DFE803F0020C162B02211D4803F0E6FD61
:1078C00008B9032300E00123237007E00420FFF739
:1078D000E9F9022314482370FBF726F8002010BDB5
:1078E0001148FBF727F818B10420FFF727FAE8E75B
:1078F00002210F4803F0CAFD10B90420FFF71EFA59
:107900000C4B1B78002BDCD0E8E70B4804F048FF59
:107910000420FFF713FA002301202370DFE7074854
:10792000F4E700BF38120020301200202F12002090
:107930000010014027120020713A0108893A01081D
:1079400070B5984B1A782ABB012197481970FAF73D
:10795000E3FF03219548FAF7DFFF05219448FAF782
:10796000DBFF0A219348FAF7D7FF0F219248FAF775
:10797000D3FF19219148FAF7CFFF0F219048FAF76A
:10798000CBFF14218F48FAF7C7FF40F6B8318E4875
:10799000FAF7C2FF8D4C2378092B0FD9A3F13002DF
:1079A000042A01D9002330E0313B032B00F2AF80E1
:1079B000DFE813F0B800C700DC00E200013B082B51
:1079C00006D8DFE803F018242B3B5F6F7A9098000D
:1079D0007F4E3578012D40F085807E4804F0E0FE32
:1079E00000237D4A337013707C4A137014227C4B41
:1079F0001A70257076E00420FEF7E4FF6E48FAF76F
:107A000093FF6E48FAF790FF022323706AE06A48FA
:107A1000FAF790FF002865D00323F6E7714804F0D9
:107A2000BFFE0420FFF7F2F804236F48237004F030
:107A3000B7FE6348BDE87040FAF776BF5F48FAF7D3
:107A400079FF10B10420FFF709F85D48FAF772FFDB
:107A500080B10420FFF772F90420FEF7FFFF6348AE
:107A600004F09EFE624804F09BFE5748FAF75CFF64
:107A70000523CAE75F4B1B78002B33D10420FEF7A8
:107A8000EDFFEFE7544B1A78012A03D100221A7058
:107A90000623BAE74C48FAF74DFF18B3564804F0EE
:107AA0007FFEF5E7554804F07BFE0420FFF7FAF867
:107AB0004448FAF739FF0723A7E74248FAF73AFFA5
:107AC00020B10420FFF73AF908239EE702214C4831
:107AD00003F0DCFC10B90420FFF730F9454B1B78AC
:107AE000002BEED070BD0221454803F0CFFC0028EA
:107AF00050D0302389E700250122354B41481D70C5
:107B0000354B1D70354B1A7004F04AFE71E73E4844
:107B100004F046FE0420FEF755FF2748FAF704FF5D
:107B2000312372E72448FAF705FF0028DAD03748F6
:107B300004F036FE0420FFF769F832231A48237058
:107B400078E71948FAF7F6FE0028CBD0304804F061
:107B500027FE0420FEF782FF0420FFF7EFF833230F
:107B600023702C48BDE8704004F01ABEFFF792FE67
:107B70000128B7D1342348E70221214803F086FCCD
:107B8000174B48B132221A702022234B1A7001225F
:107B9000224B1A70092338E7142203481A70FAF7A7
:107BA000C3FEF7E7A8120020A012002098120020C0
:107BB00090120020881200208012002078120020ED
:107BC0007012002068120020601200205D12002058
:107BD0007F0E0020A63A01087B0E0020770E0020C1
:107BE000650E0020B93A0108C53A0108D73A0108E4
:107BF000E93A010827120020F73A01080E3B010874
:107C0000001001401C3B01082A3B0108373B0108DA
:107C1000443B0108593B0108640E00206B0E002014
:107C200008B5FFF73DF9FFF701FBFFF7C3FCBDE81F
:107C30000840FFF785BE0000F8B5134F3B7813B935
:107C4000FFF7D6F83870114E337813B9FFF796FA6C
:107C500030700F4D2B7813B9FFF756FC28700D4C80
:107C6000237813B9FFF716FE20703B78012B0AD159
:107C70003378012B07D12B78012B04D12378012BEA
:107C800004BF054A1370F8BD2E1200202D120020EB
:107C90002C1200202B1200208D13002038B5044632
:107CA00008480D1904F07CFDAC4204D1BDE8384011
:107CB000044804F075BD14F8011B034804F070FD7E
:107CC000F2E700BFE9200108D121010808B503F05F
:107CD00007F860B101F0BAF90522084B08491A709B
:107CE00004230B7007490A70074A137008BD074840
:107CF00004F056FD01F0C8FAEEE700BF1D000020B9
:107D00001C000020550E0020540E0020683B010886
:107D1000084B09481978094B1B7859436FF06303E6
:107D200091FBF3F1064B1B781944064BC9B219704D
:107D300004F036BD11000020853B01081200002030
:107D400010000020580E002010B51B4804F028FD3C
:107D50001A4A1B491B4804F097FB4FF47A7003F052
:107D6000E5FAFBF765FAFBF7CFFCFBF7CDFAFEF778
:107D700099FCFDF76BFFFEF7B9FDFDF725FEFCF75B
:107D800009F802F009FEFEF7B5FEFFF79FFFFFF7C7
:107D9000BFFF0D4C237863B101F0D0F80020FEF74F
:107DA00087FC0122094B0A481A70BDE8104004F014
:107DB000F7BCFFF741FFEDE79B3B010850210108AD
:107DC000B03B0108101900208D130020E80E0020A0
:107DD000B83B010808B5254804F0E2FC244804F04B
:107DE000DFFC03F04BFA4FF47A7003F09FFA03F0D4
:107DF00055FA4FF47A7003F099FA1E4804F0D0FC5B
:107E00000420FEF74FFF4FF47A7003F08FFA04203E
:107E1000FEF794FF4FF47A7003F088FA164804F0E6
:107E2000BFFC03F00BFA4FF47A7003F07FFA03F013
:107E300015FA4FF47A7003F079FA104804F0B0FCA8
:107E40000320FEF7BFFD0420FEF7BCFD4FF47A705F
:107E500003F06CFA0320FEF701FE0420FEF7FEFD9E
:107E6000BDE80840064804F09BBC00BFD13B0108B8
:107E7000E03B0108F33B0108063C0108173C010800
:107E8000283C01080346F0B490B008469E181946F5
:107E90006C466B46B14209D1034600EB5202934255
:107EA00049D1102110B0F0BCFFF7F8BE11F8015B0A
:107EB000303D362D1FD8DFE805F01C20222426286F
:107EC0002A2C2E301E1E1E1E1E1E1E323436383A1E
:107ED0003C1E1E1E1E1E1E1E1E1E1E1E1E1E1E1EA4
:107EE0001E1E1E1E1E1E1E1E1E1E1E323436383A3A
:107EF0003C0000251D700133CCE70125FAE702257F
:107F0000F8E70325F6E70425F4E70525F2E706255B
:107F1000F0E70725EEE70825ECE70925EAE70A255B
:107F2000E8E70B25E6E70C25E4E70D25E2E70E255B
:107F3000E0E70F25DEE714F8025B14F8011C41EAC4
:107F4000051103F8011BAAE71FB51A4CB4F900206C
:107F50002388002A24DAC3F30E03222B22D1164BE6
:107F60009A7F302A01D0462A1CD1DB7F302B01D0EA
:107F7000462B17D1114804F013FC202269460E4805
:107F8000FFF780FF102269460D4806F0D5F8FDF78F
:107F900031FD80220021084804F014FC00232380D6
:107FA00004B010BD074804F0FBFB0348FDF786FD55
:107FB000EFE700BFC80F0020CC2400203B3C0108A5
:107FC000C9110020463C0108F8B55E4B1A7872B919
:107FD000012264215C481A70FAF79EFC4FF4FA61A2
:107FE0005A48FAF799FC0A215948FAF795FC594D75
:107FF0002C78012C1FD0032C00F09580D4B9564F5B
:108000003E78012E16D1554804F0CAFB544B554812
:108010001C70554B3C701C70544B1C70544B1C70A6
:10802000544B1C70544B1C7004F0BAFB4748FAF7D1
:108030007BFC2E70F8BD4548FAF77CFC38B14F4BFD
:108040004F481C7004F0ACFB03232B70F2E74D4B40
:108050001A78012A06D118703C48FAF765FC4A489C
:1080600004F09EFB494C2378FF2B1BD10023237087
:108070000123474A1370474A12780AB93A4A1370E3
:10808000454B1B7813B90122384B1A70434B1B78B0
:1080900013B90122364B1A70414B1B7813B90122D8
:1080A000344B1A702378A3B10121394A013B117076
:1080B000032B0CD8DFE803F00219232D354B1B7876
:1080C0008BB90122284B37481A7004F069FB002352
:1080D0002370294A1378012BACD100211170274A53
:1080E00031481370AEE73148EFE72B4B1B7823B9CB
:1080F00001221E4B2E481A70E7E72E48E5E7274B72
:108100001B7823B901221A4B2B481A70DDE72B4844
:10811000DBE7234B1B7823B90122164B28481A7042
:10812000D3E72848D1E700230B4A1370264A13707F
:108130000D4A13700D4A13700D4A13700D4A1370D7
:1081400083E700BF5814002050140020481400207A
:10815000401400203D140020880E0020533C0108EC
:10816000620E0020783C0108860E0020850E00205B
:10817000840E0020830E0020760E0020720E002058
:10818000893C0108740E00209C3C0108A40E0020CC
:1081900092100020CB0E0020CA0E0020C90E002035
:1081A000C80E0020B93C0108313D0108C93C010856
:1081B000D73C0108E73C0108F53C0108053D0108F2
:1081C000133D0108233D01084C2800200023064AE6
:1081D0001370064A1370064A1370064A1370064A53
:1081E0001370064A137070474C280020880E002038
:1081F000860E0020850E0020840E0020830E0020B5
:108200002DE9F04FA04B89B01A7852BB01219F484D
:108210001970FAF781FB0F219D48FAF77DFB0521C4
:108220009C48FAF779FB0A219B48FAF775FB102165
:108230009A48FAF771FB3C219948FAF76DFB4FF425
:10824000E1619848FAF768FB40F6B8319648FAF7CA
:1082500063FB14219548FAF75FFB0A219448FAF76B
:108260005BFB944C2378212B25D8212B29D8DFE8E0
:1082700013F02A00C600F9007901420256021503E4
:108280003E03280028002800280028002800280095
:1082900028002800F503FA03FC0304040A0428005C
:1082A000280028002800280028002800280028008E
:1082B00028001104C300402B00F09E80502B00F0DA
:1082C0000E830023CCE07C4B1B78012B0CD07B4B26
:1082D0001B78012B08D07A4B1B78012B04D0794BEB
:1082E0001B78012B40F088800125774804F058FA6C
:1082F000764B774A1D7000231370764ADFF8D8E179
:108300001370764ADFF8D8811370764A764E137070
:10831000764A774F1370774ADFF8DCA11370774AFB
:108320001370774A1370774A1370774A1370774A3D
:108330001370774A1370774A1370774A1370774A2D
:108340001370774A1370774A1370774A1380774A0D
:108350001380774A1380774AB2F800C0764AAEF8A5
:1083600000C01088A8F800C0744ADFF8D4C1118892
:10837000ACF800003080734A73481288018039805D
:108380007249AAF800200A80714A7248137004F0FA
:1083900007FAB8F8000009F08BFA6F4909F094FB6E
:1083A00008F0A0FE8046BAF80000894609F080FA7D
:1083B000694909F089FB08F095FECDE90401388888
:1083C00009F076FA644909F07FFB08F08BFECDE9ED
:1083D0000201308809F06CFA5F4909F075FB08F07A
:1083E00081FE4246CDE900014B465C4804F0D8F9D5
:1083F0002648FAF799FA257009B0BDE8F08F2348AE
:10840000FAF798FA0028F7D02B4A1378012B05D1F8
:10841000002111702F4A1370364A1370274A1378BF
:10842000012B05D1002111702C4A1370334A1370AF
:10843000234A1378012B05D100211170294A1370AA
:108440002F4A13701F4A1378012B05D10021117098
:10845000264A13702B4A13701348FAF765FA022361
:108460002370C9E71048FAF765FA20B13C4804F0D8
:1084700097F90423F4E70B48FAF756FA0A48FAF793
:1084800053FA0323ECE700BF3C140020341400200F
:108490002C140020241400201C140020141400208C
:1084A0000C14002004140020FC130020F4130020FE
:1084B000EC130020E8130020860E0020850E00201B
:1084C000840E0020830E0020463D0108CC0E0020C3
:1084D0009F0E0020820E0020DE130020810E00205F
:1084E000BE0E0020800E0020BA0E00207F0E00205D
:1084F000B60E0020E7130020B20E0020E613002085
:10850000E5130020E4130020E3130020E213002011
:10851000E1130020E01300207E0E00207D0E0020DD
:108520007C0E00207B0E0020AE0E0020AC0E002042
:10853000AA0E0020A01000209E1000209C100020F9
:10854000DC1300209A100020DA130020D81300203A
:10855000700E00205B3D01080000C842703D01081C
:10856000AD3D01089848FAF7E5F938B1042397487A
:10857000237009B0BDE8F04F04F012B9944B1D7898
:10858000012D0BD11870934B93481D70934B1D70A8
:10859000FAF7CAF9924B1D70924B1D70924B1D78E1
:1085A000012D0CD100221A70904B8B481D70904BFE
:1085B0001D70FAF7B9F98A4B1D708A4B1D708D4BEF
:1085C0001D78012D0CD100221A708B4B82481D7032
:1085D0008A4B1D70FAF7A8F9814B1D70814B1D70F5
:1085E000874B1D78012D0CD100221A70854B7A48DB
:1085F0001D70854B1D70FAF797F9794B1D70794BFB
:108600001D70824B82491A880B889A420ED9D31A60
:10861000042B0BDD70480A80FAF786F90123704AB3
:108620007C4813706F4A137004F0BAF87A4B7B4998
:108630001A880B889A420ED9D31A042B0BDD664890
:108640000A80FAF771F90123654A75481370654A83
:10865000137004F0A5F8734B73491A880B889A427B
:108660000ED9D31A042B0BDD5B480A80FAF75CF9AC
:1086700001235B4A6D4813705A4A137004F090F856
:108680006B4B6C491A880B889A420ED9D31A042B6B
:108690000BDD51480A80FAF747F90123504A664832
:1086A0001370504A137004F07BF84B48FAF74EF9F8
:1086B0000A23B0FBF3F0614BC0B21870604B1A682C
:1086C000824207D0186001235E4A0328137004BF5A
:1086D0005D4A13704048FAF72DF920B15B4804F069
:1086E0005FF85B48C3E65B4B1A78012A7FF484AEDF
:1086F00018705948F3E7594804F052F80123584AD2
:1087000058481370584A1370584A1370584A1370D7
:108710000523237009B0BDE8F04FFAF705B95148B9
:10872000FAF708F930B106235248237004F038F8FC
:108730005148EFE7294B514A1B78012B03D1504B8D
:108740001B78012B01D101231370294B1B78012BBE
:1087500003D14C4B1B78012B02D101214A4B1970DC
:10876000264B1B78012B03D1484B1B78012B02D1E0
:108770000121474B1970244B1B78012B03D1454B2A
:108780001B78012B02D10121434B19701378012B67
:108790007FF432AE3C4D2B78012B7FF42DAE3C485C
:1087A0000378012B7FF428AE3B490B78012B7FF433
:1087B00023AE00230370304813702B700B70FAF750
:1087C000B3F806234CE600BFFC130020AD3D0108C2
:1087D000860E0020820E002004140020E7130020E3
:1087E000750E0020740E0020850E0020810E0020E2
:1087F000E6130020840E0020800E0020E5130020E8
:10880000830E00207F0E0020E4130020A010002023
:10881000DE130020C33D01089E100020DC13002061
:10882000D13D01089C100020DA130020DF3D010833
:108830009A100020D8130020ED3D0108700E002092
:10884000D4130020710E002090100020FB3D010881
:108850000A3E01089F0E0020133E01082A3E01082F
:108860007E0E00200C1400207D0E00207C0E0020C7
:108870007B0E0020413E0108F4130020E31300208A
:108880007A0E0020790E0020E2130020780E0020DE
:10889000E1130020770E0020E01300208848FAF74B
:1088A00049F800283FF4A8AD864B87481A88874BC3
:1088B0001A80874B1A88874B1A80874B1A88874BF8
:1088C0001A80874B1A88874B1A800022864B1A70B1
:1088D0000122864B1A70FAF727F85023C0E57A4830
:1088E000FAF728F800283FF487AD0723B8E5804E53
:1088F000804803F055FF308808F0DAFF7E4909F020
:10890000E3F808F0EFFB714F80463888894608F09D
:10891000CFFF794909F0D8F808F0E4FBDFF8DCA1D3
:1089200042464B46CDE90001754803F039FFBAF8DD
:10893000000008F0BDFF704909F0C6F808F0D2FB4E
:10894000644D80462888894608F0B2FF6A4909F0DC
:10895000BBF808F0C7FB4246CDE900014B46694829
:1089600003F01EFF684BDFF874B1188808F0A0FF11
:10897000614909F0A9F808F0B5FB8046BBF8000092
:10898000894608F095FF5C4909F09EF808F0AAFBBB
:108990004B46DFF878914246CDE900015C4803F090
:1089A000FFFEB9F8000008F083FF534909F08CF886
:1089B00008F098FB02460B46DFF82881CDE9062334
:1089C000B8F8000008F074FF4B4909F07DF808F092
:1089D00089FBDDE90623CDE900014E4803F0E0FE06
:1089E0003B883288934231D39B1A9BB2092B98BFA4
:1089F0000023494A13802B88BAF80020934227D3DA
:108A00009B1A9BB2092B98BF0023444A13803E4A0D
:108A1000BBF80030128893421CD39B1A9BB2092BDF
:108A200098BF00233E4A1380B8F80030B9F8002000
:108A3000934211D39B1A9BB2092B98BF0023394A4A
:108A40003948138003F0ACFE112309E50023D0E779
:108A50000023DAE70023E5E70023F0E7334803F0DB
:108A60009FFE1223FCE41323FAE4314803F098FE3E
:108A70000122304B1A701423F2E4FFF7A7FB2E48B3
:108A800003F08EFE1DE42D4803F08AFEF8F7F6FD94
:108A90002B48F5E72B4803F083FEF8F7EFFD0120A4
:108AA000FAF712FE0220FAF70FFE0123264A2748A2
:108AB0001370274A137003F073FE2123D0E400BF24
:108AC000F4130020A0100020EC130020BC0E0020A6
:108AD0009E100020B80E00209C100020B40E002034
:108AE0009A100020B00E0020CC0E00209914002017
:108AF000BE0E0020543E01080000C842BA0E0020FD
:108B0000693E01088B3E0108B60E0020B20E00201F
:108B1000AD3E0108CF3E0108C60E0020C40E002065
:108B2000C20E0020C00E0020F13E0108063F0108E1
:108B3000193F0108760E0020323F01084A3F010824
:108B40006B3F0108893F0108690E0020A43F01081E
:108B50006A0E002010B5174B1A7832B901224FF473
:108B6000E16115481A70F9F7D7FE144C237813B158
:108B7000012B11D010BD124B1B78022B03D0114BCF
:108B80001B78022BF6D1104803F00AFE0A48F9F7C9
:108B9000CBFE01232370EDE70748F9F7CBFE002851
:108BA000E8D00A4803F0FCFD0023054A1370054A8B
:108BB0001370EFE7D0130020C8130020C513002066
:108BC000AA140020A8140020C63F0108ED3F0108A8
:108BD00010B5234B1A784AB90122022121481A7094
:108BE000F9F79AFE02212048F9F796FE1F4C2378E8
:108BF000032B0FD8DFE803F002121D2A1C4A13785A
:108C0000012B07D10021117002221A490A701A495A
:108C10000A702370BDE81040FFF79CBF174803F0AF
:108C2000BFFD0620FDF7CEFE0E48F9F77DFE0223BC
:108C3000EFE70C48F9F77EFE0028EBD00620FDF7A1
:108C40000DFF0948F9F770FE0323E2E70648F9F73C
:108C500071FE0028DED00023054A1370D9E700BF5B
:108C6000C4130020BC130020B4130020B113002053
:108C7000610E0020AA140020A81400200240010860
:108C800038B51A4B1A782AB90122962118481A7059
:108C9000F9F742FE174C25781DB1012D13D00023A2
:108CA00022E0154B1D78012D0CD12846FDF78AFED8
:108CB0000220FDF787FE114803F072FD0C48F9F71A
:108CC00033FE257038BD0A48F9F734FE0028F9D084
:108CD0002846FDF7C3FE0220FDF7C0FE084803F05A
:108CE0005FFD0023044A13702370EBE7B0130020EC
:108CF000A8130020A5130020E90F0020134001084D
:108D00002440010810B5174B1A782AB901226421B2
:108D100015481A70F9F700FE144C237813B1012B93
:108D200010D010BD124B1B78272BFAD9114803F035
:108D300037FD0320FDF746FE0420FDF743FE012327
:108D40002370EEE70A4B1B78262BEAD80A4803F07B
:108D500027FD0320FDF782FE0420FDF77FFE0023A0
:108D6000EEE700BFA41300209C13002099130020FD
:108D7000F4110020354001085240010838B5284B55
:108D80001A782AB90122642126481A70F9F7C4FD1D
:108D9000254C2378012B23D0022B2AD0A3B9012103
:108DA000224802F073FB80B9214803F0F9FC04204B
:108DB000FDF778FF01231F4A652013701E4A1370C8
:108DC000F8F7DCF90223237038BD1C4B1B784F2BBE
:108DD000FAD91B4803F0E4FC0123164A1370F2E7AA
:108DE000164B1B784B2B17D8164803F0D9FC0023E1
:108DF000E9E701210D4802F049FB01280CD10025CB
:108E0000114803F0CDFC0420FDF798FF0A4B6520C4
:108E10001D70F8F7B3F925700122064B1A70D3E7DD
:108E200098130020901300208E13002000100140A2
:108E3000654001088F100020E10E0020F411002091
:108E40008A400108AA400108C44001081E280146C2
:108E500014D8D0B1431E1D2B17D8DFE803F01D1620
:108E60002022241626282C2A2E16303234363A3C5C
:108E700016161616161616161616163E512826D053
:108E800006D83F282BD040282BD0174803F088BCA9
:108E90005228FAD1154800E0154803F081BC154866
:108EA000FBE71548F9E71548F7E71548F5E71548D2
:108EB000F3E71548F1E71548EFE71548EDE71548E2
:108EC000EBE71548E9E71548E7E71548E5E71548F2
:108ED000E3E71548E1E71548DFE71548DDE7154802
:108EE000DBE71548D9E700BF234101080941010824
:108EF00071340108763401087B340108803401089C
:108F0000DD4001088A340108E6400108F14001080B
:108F1000FC4001088F340108943401089934010899
:108F20009E340108034101080F410108A3340108E0
:108F3000A8340108154101081C410108F7B5324861
:108F400003F02EFC314803F02BFC3149314803F08B
:108F500027FC314B314C1B78314D013B314E324FA8
:108F6000042B0DD8DFE803F0031A252738002F481B
:108F700003F016FC2078FFF769FF2D4803F010FC82
:108F80003B782348009333782A782178FCF746FF12
:108F9000284803B0BDE8F04003F002BC264803F0C7
:108FA000FFFB2078FFF752FF244803F0F9FB2878F5
:108FB000E1E72348F3E7234803F0F2FB2078FFF7CB
:108FC00045FF1E4803F0ECFB2878FFF73FFF1B48E6
:108FD00003F0E6FB3078CEE71B4803F0E1FB207896
:108FE000FFF734FF154803F0DBFB2878FFF72EFF6F
:108FF000124803F0D5FB3078FFF728FF0F4803F045
:10900000CFFB3878B7E700BF2C410108E4410108E5
:10901000101900203B4101081D0000201B0000200A
:109020001A00002019000020180000204441010807
:1090300082270108D54101085F4101087A410108F2
:109040007D4101089F410108BA4101082DE9F74F10
:10905000594A5A4B12785A491A705A4A5A4B12783E
:109060005A480A705A4A5B4C12785B4D1A705B4A38
:10907000DFF86CB112785B4E02705B4A5B48127885
:10908000006822705A4ADFF86CA112785A4F2A7091
:109090005A4ADFF86CE11268DFF86881CBF80020EB
:1090A000594ADFF86891106059485A4A00785A4C7A
:1090B00010705A485A4D007830705A485A4E00780D
:1090C0008AF800005948007838705948594F00789C
:1090D0008EF800005848007888F800005748DFF8FC
:1090E0006081007889F800005648DFF85C910078CC
:1090F00020705648564C007889F800005548007892
:1091000030705548007838705448007888F800006E
:10911000534800782070534800782870524803F074
:109120003FFB524803F03CFB2549244B0978364A63
:109130000091DBF800101B7812684D4803F030FBFB
:109140009AF80030DFF89CC0324A1F4900939CF81F
:10915000003012780978474803F022FB294BDFF8EA
:10916000A0E01B781948244A00939EF8003001784B
:109170001278414803F014FB99F800301549009328
:10918000DFF88890244B99F800201B7809783B4839
:1091900003F006FB98F800300F49009332783B78D3
:1091A0000978374803F0FCFA2A782178354803B06B
:1091B000BDE8F04F03F0F4BA1D000020550E00206A
:1091C000540E00201C000020530E0020520E0020E0
:1091D0001B000020510E0020500E00201A0000201D
:1091E0004C0E0020450E0020190000205C0E0020CF
:1091F00018000020440E0020430E00201400002020
:10920000420E0020410E0020480E0020400E00209B
:1092100011000020460E00203F0E0020100000200C
:10922000390E00200F0000203D0E00200E0000200F
:109230000D0000203C0E00200C0000200B00002040
:109240003B0E00200A0000203E0E002009000020F6
:109250003A0E002008000020070000200600002031
:10926000570E0020560E0020F34101081442010859
:109270002242010844420108614201087E4201087D
:109280009B420108B84201082DE9F74F594BDFF81E
:1092900068B11B68594ACBF80030594B59481B68D4
:1092A000594C1360594B5A4A1B785A4D13705A4BFC
:1092B0005A4E1B78DFF868A103705A4B5A481B7846
:1092C0005A4F23705A4B04241B78DFF868812B70A7
:1092D000052505705848594B047059481D70007891
:1092E000584BDFF8649118705848594900780C7051
:1092F00030705848584C0078584D8AF8000058484B
:10930000584E007838705848584F007888F8000058
:109310005748DFF86081007889F800005648DFF888
:109320005C91007820705648564C0078287056485A
:10933000564D007889F8000055480078307055483F
:10934000007838705448007888F800005348007856
:109350002070534800782870524803F021FA524890
:1093600003F01EFA3A49354B0978244A0091DBF89C
:1093700000101B7812684D4803F012FA9AF800307A
:10938000DFF898E0DFF8BCC0214900939EF8003078
:109390009CF800200978464803F002FADFF8A8C0DC
:1093A00018489CF80030214A0093224B01781B7822
:1093B0001278404803F0F4F999F80030264A0093F7
:1093C0001149264B12781B7809783B4803F0E8F9DD
:1093D00098F800300F49009332783B780978374885
:1093E00003F0DEF92A782178354803B0BDE8F04F64
:1093F00003F0D6B94C0E0020140000205C0E0020B3
:10940000480E00201A00002019000020530E0020F2
:109410001B00002018000020520E00201000002029
:109420000F000020510E0020550E00200E000020DD
:10943000500E00200D000020540E00201D000020C2
:10944000460E0020110000200C000020450E0020D8
:109450001C000020440E00200B0000200A00002009
:10946000430E002008000020420E002007000020CC
:10947000410E002006000020400E002009000020C0
:109480003F0E0020570E00203E0E0020560E0020FA
:109490003D0E00203C0E00203B0E00203A0E002026
:1094A000390E0020CA420108E9420108224201089F
:1094B00044420108614201087E4201089B420108C2
:1094C000B842010838B5044604F044FE092811D812
:1094D0000A49204603F07EF90546204604F03AFE8C
:1094E000854204D12046BDE8384002F062BB044802
:1094F00003F056F94FF0FF3038BD00BFF7420108C6
:109500000243010870B504460D1F00EB0216B44279
:1095100001D101200CE02046FFF7D4FF431C03D00B
:10952000103445F8040FF2E7024803F039F900203F
:1095300070BD00BF1343010870B54FF4807204463C
:1095400000212D4803F03EF92C4803F029F90023AF
:109550002B4D20462B492B7003F04CF90446264E28
:109560003CBB2978284803F01BF9234E2B78E1B245
:109570008B4237D8254803F013F91F48FFF7A2FFA5
:10958000431C36D0224C234D2070C1B2224803F038
:1095900007F923782A789A4209D0012B07D00122B3
:1095A0001E4B1F481A7003F0FBF823782B70012024
:1095B00070BD204604F0CEFD0F280ED82878214635
:1095C00006EB001004F0A2FD00200E4903F012F992
:1095D0002B78044601332B70C2E7124803F0E0F801
:1095E0000020E5E7104806EB011103F0D9F801343B
:1095F000BCE70E48F2E700BF2E39002026430108E1
:10960000AD38002081310108504301086D43010845
:109610003F3A002088140020714301080D0E0020FD
:109620007E43010835430108684301088F43010860
:109630002DE9F04F9B49BBB003F042F9044680226C
:1096400000211AA803F0BEF8611C1AA804F05EFD00
:109650001AA8FFF771FF0128044624D1924D9348C0
:10966000297803F09DF82B780D2B12D8DBB1013B44
:109670000C2B18D8DFE813F022003C005000D30078
:109680001700EB0003011700170017001700170061
:109690007A01382B00F0768208D81E2B00F0448225
:1096A0001F2B00F059823BB0BDE8F08F642BFAD13C
:1096B0007F4803F075F87F4B1C70F4E77E4803F099
:1096C0006FF87E497E4803F06BF87C48FFF7FAFE9E
:1096D0000146481C7B4B05D07B4A116001221A7061
:1096E0007A4867E000227A481A7003F059F8DAE7FE
:1096F000784803F055F87149714803F051F86F4804
:10970000FFF7E0FE421C0146734B01D0734AE4E7C9
:10971000002273481A70E8E7724803F041F867497D
:10972000674803F03DF86548FFF7CCFE431C13D0B3
:109730006D4BC1B218706D4803F032F86C496D483A
:1097400003F02EF86A48FFF7BDFE471C09D100223E
:10975000694B6A481A70C8E70022674B68481A705C
:10976000C3E7684CC1B22070674803F019F80023C2
:10977000227866480AA9CDE90A33CDE90C33FFF710
:10978000C1FE012804D000225B4B61481A70ACE78F
:1097900020780C9B0138DDE90A12032883D8DFE822
:1097A00000F0020C192901225A4B5B481970524BE8
:1097B000C9B21A7002F0F4FF75E70120554B197019
:1097C000564BC9B21A704C4BD2B21870544802F0C2
:1097D000E7FF68E701244F4801705048C9B20270A2
:1097E0005048D2B203704448DBB204704E4802F0D5
:1097F000D7FF58E70125474C0D982170474CC9B257
:109800002270484CD2B22370484CDBB220703A4CE4
:10981000C0B225700090464802F0C2FF43E74548B9
:1098200002F0BEFF2549264802F0BAFF2348FFF7A1
:1098300049FE461C0146404B05D0404A10600122BB
:109840003F481A70B6E700223E481A704DE73E487E
:1098500002F0A6FF19491A4802F0A2FF1748FFF7C5
:1098600031FE451C394B06D0394A10700122C1B275
:109870001A7038489EE7002237481A7035E7374893
:1098800002F08EFF0D490E4802F08AFF0B48FFF7E9
:1098900019FE441C324B01D0324AE6E7002232481E
:1098A0001A7022E7F23101083F3A00209C43010878
:1098B000F8470108020E0020AC4301083E390020A1
:1098C000C74301080C0E0020280E0020D7430108D2
:1098D000E6430108FF4301080B0E0020240E002080
:1098E000164401082F440108310E00204A440108A3
:1098F0004E3900205D440108090E0020A1440108F2
:109900006D440108300E0020864401085E390020B5
:10991000224501082F0E0020C24401082E0E00200F
:10992000D44401082D0E0020EA4401082C0E00202A
:10993000044501083F450108080E0020200E0020C4
:109940005C4501086D45010888450108070E0020A7
:10995000110E0020B4450108C3450108EE45010879
:10996000060E0020100E002016460108904802F056
:1099700017FF9049904802F013FF8E48FFF7A2FDB1
:10998000411C3FF4E4AE8D4FC1B238708C4802F0F8
:1099900007FF00233A788B4802EB4202D2B20AA9B1
:1099A000CDE90A33CDE90C33CDE90E33CDE91033DF
:1099B0001293FFF7A7FD012840F0B180DDE90A12FC
:1099C000DDE90C30DDE90E45DDE9106C3F78DDF8AE
:1099D00048E0013F032F3FF666AEDFE807F00210D4
:1099E0002C5A0124784801707848C9B2027078482E
:1099F000D2B203707748DBB204707748F7E60127EC
:109A0000714E3170714EC9B23270714ED2B2337034
:109A1000724EDBB23070724EC0B23470714EE4B22E
:109A200035706C4EEDB237700090029501946E481F
:109A300002F0B6FE37E64FF00108634F3970634F0E
:109A4000C9B23A70624FD2B23B70644FDBB2387029
:109A5000634FC0B23C70634FE4B23D70634FEDB2F0
:109A60003E70634FF6B287F800C0624F87F800E09F
:109A7000584F87F800805FFA8EF705975FFA8CF7EA
:109A8000009004970396029501945B4802F088FECB
:109A900009E64FF0010B4C4FDDF84C8039704B4F0D
:109AA000DDF850903A704A4FDDF854A03B704B4FB0
:109AB000DBB238704A4FC0B23C704A4FE4B23D70DE
:109AC0004A4FEDB23E704A4FF6B287F800C0494F98
:109AD000D2B287F800E0494FC9B287F80080484FFA
:109AE00087F80090474F87F800A03A4F87F800B0FA
:109AF0005FFA8AF708975FFA89F707975FFA88F79E
:109B000006975FFA8EF705975FFA8CF70090049737
:109B10000396029501943C4802F042FEC3E5002200
:109B20003A4B3B481A70E0E53A4802F039FE2149C9
:109B3000214802F035FE1F48FFF7C4FC421C06D046
:109B4000354BC1B21870354B35481C7032E60022D7
:109B5000344B35481A70C8E5344802F021FE1549E7
:109B6000154802F01DFE1348FFF7ACFC0130304BE6
:109B700004D01C70284B2F4819781BE600222E4871
:109B80001A70B2E52D4802F00BFE0A490A4802F0AD
:109B900007FE0848FFF796FC431C0146284B03D0FC
:109BA000284A1C7010609BE5002227481A709CE52B
:109BB0003D4601083E390020C7430108300E002011
:109BC000864401084E3900201D0E00201C0E002086
:109BD0001B0E0020050E00205F4601081A0E002013
:109BE000190E0020180E002073460108170E0020E1
:109BF000160E0020150E002098460108140E0020B5
:109C0000130E0020120E0020CE460108090E00207F
:109C100015470108324701080F0E0020040E0020EE
:109C2000494701080C0E00205C47010879470108EC
:109C3000030E002090470108A3470108C047010810
:109C40000A0E0020240E0020DB47010810B50B4B44
:109C50001C78012C0FD100221A70094B1A68094B8D
:109C60001B689A4204D1084802F09AFD204610BDB4
:109C7000064802F095FD0024F8E700BF0C0E002016
:109C800014000020280E00201B4801082E4801085F
:109C900070B51C4C237813B1012B0BD070BD1A4941
:109CA0000A78012AFAD10B70184922700B701849F2
:109CB0000B70F3E7154B1E78012E1AD100251D708D
:109CC000144B1A68144B1B689A420DD1134802F0CA
:109CD00067FD134B13481A68134B1A6002F060FDBE
:109CE000124B25701E70D9E71148BDE8704002F094
:109CF00057BD074A1378012BD0D100230D481370AC
:109D00002370F2E7871400200B0E00200C0E0020B9
:109D10000D0E002014000020280E00201B48010812
:109D2000240E0020414801084C0E00200E0E002099
:109D30002E4801085448010838B5094D2C7874B9EB
:109D4000084A1378012B0AD11470074A0748116892
:109D5000074A1160074A137002F022FD2C7038BDCB
:109D6000861400200A0E0020240E00206F480108EF
:109D70004C0E00200E0E002070B5264C237813B137
:109D8000012B0ED070BD244A1578012DFAD1137025
:109D9000224A23481370234A137002F001FD2570F4
:109DA000F0E71E4B1E78012E2AD100251D701E4B98
:109DB0001A681E4B1B689A421DD11D4802F0F0FC28
:109DC0001C4B1A781C4B1A701C4B1A781C4B1A70BF
:109DD0001C4B1A781C4B1A701C4B1A781C4B1A70AF
:109DE0001C4B1A781C4B1A701C4B1A781C4B1A709F
:109DF0001C4B1E70D3E71C48BDE8704002F0D0BC7D
:109E0000084A1378012BBDD1002318481370237022
:109E1000F2E700BF85140020090E00200C0E002080
:109E2000864801080D0E002014000020280E002096
:109E30001B480108310E0020550E0020300E002076
:109E4000540E00202F0E0020530E00202E0E002056
:109E5000520E00202D0E0020510E00202C0E00204E
:109E6000500E00200E0E00202E4801085448010814
:109E700070B51C4C237813B1012B0BD070BD1A495F
:109E80000A78012AFAD10B70184922700B70184910
:109E90000B70F3E7154B1E78012E1AD100251D70AB
:109EA000144B1A68144B1B689A420DD1134802F0E8
:109EB00077FC134B13481A68134B1A6002F070FCBE
:109EC000124B25701E70D9E71148BDE8704002F0B2
:109ED00067BC074A1378012BD0D100230D481370BB
:109EE0002370F2E784140020080E00200C0E0020DE
:109EF0000D0E002014000020280E00201B48010831
:109F0000200E0020A5480108480E00200E0E00205B
:109F10002E4801085448010838B5214C237813B164
:109F2000012B0BD038BD1F490A78012AFAD10B70DA
:109F30001D4922700B701D490B70F3E71A4B1A78FC
:109F4000012A23D100221A70194B1A68194B1B6879
:109F50009A4216D1184802F023FC184B184D1B7872
:109F600018482B7002F01CFC2B78012B0CBF1648F4
:109F7000164802F015FC0122154B1A7000232370BD
:109F8000D0E71448BDE8384002F00ABC074A13780D
:109F9000012BC7D10023104813702370F2E700BFD4
:109FA00083140020070E00200C0E00200D0E002050
:109FB00014000020280E00201B480108110E00206C
:109FC0003A0E0020BA480108E3480108EE480108AB
:109FD0000E0E00202E4801085448010838B5214CC7
:109FE000237813B1012B0BD038BD1F490A78012A01
:109FF000FAD10B701D4922700B701D490B70F3E7ED
:10A000001A4B1A78012A23D100221A70194B1A68A8
:10A01000194B1B689A4216D1184802F0C1FB184B25
:10A02000184D1B7818482B7002F0BAFB2B78012BC7
:10A030000CBF1648164802F0B3FB0122154B1A70EC
:10A0400000232370D0E71448BDE8384002F0A8BBD5
:10A05000074A1378012BC7D10023104813702370CF
:10A06000F2E700BF82140020060E00200C0E002034
:10A070000D0E002014000020280E00201B480108AF
:10A08000100E0020390E0020F9480108EE480108A2
:10A09000E34801080E0E00202E480108544801082C
:10A0A00070B5324C237813B1012B0ED070BD304AFD
:10A0B0001578012DFAD113702E4A2F4813702F4AAC
:10A0C000137002F06DFB2570F0E72A4B1E78012E0D
:10A0D00042D100251D702A4B1A682A4B1B689A42F0
:10A0E00035D1294802F05CFB284B1A78284B1A70AE
:10A0F000284B1A78284B1A70284B1A78284B1A705C
:10A10000284B1A78284B1A70284B1A78284B1A704B
:10A11000284B1A78284B1A70284B1A78284B1A703B
:10A12000284B1A78284B1A70284B1A78284B1A702B
:10A13000284B1A78284B1A70284B1A78284B1A701B
:10A14000284B1A78284B1A70284B1E70BBE72848FA
:10A15000BDE8704002F024BB084A1378012BA5D15A
:10A160000023244813702370F2E700BF81140020FD
:10A17000050E00200C0E0020864801080D0E002060
:10A1800014000020280E00201B4801081D0E00208E
:10A19000460E00201C0E0020450E00201B0E002045
:10A1A000440E00201A0E0020430E0020190E00203D
:10A1B000420E0020180E0020410E0020170E002035
:10A1C000400E0020160E00203F0E0020150E00202D
:10A1D0003E0E0020140E00203D0E0020130E002025
:10A1E0003C0E0020120E00203B0E00200E0E002020
:10A1F0002E48010854480108F8B57C4B1A786AB912
:10A2000001221E217A481A70F8F786FB0A21794844
:10A21000F8F782FBC8217848F8F77EFB774C237863
:10A22000112B1ED8DFE813F012001E00410064005D
:10A230009900C7001D001D001D001D001D001D0010
:10A240001D001D001D001D00D300DB006C490A78B5
:10A25000012A06D100230B706A4922700B706A49EB
:10A260000B70F8BD674B1A78012A15D100221A70BD
:10A27000664B1A68664B1B689A4208D1654802F023
:10A280008FFA654802F08CFA02232370E9E76348ED
:10A29000BDE8F84002F084BA5B4A1378012BE0D1A4
:10A2A00000235F4813702370F2E75E4D2878FCF7B7
:10A2B0000DF92B7853B95C4B1B78012B03D1FBF7BD
:10A2C00071FE0023E1E7FBF7A9FEFAE7574AA12058
:10A2D00013700023564A1370564A13700122564BCE
:10A2E0001A7000F075FE4448F8F71EFB0323CCE714
:10A2F0004148F8F71FFB38B1504802F051FA0022EC
:10A300004D4B1A7010232370464D2B78012B0ED025
:10A31000022BD6D1474B1E78012EA2D1484802F01D
:10A320003FFA2878FCF7FAF80023464A0BE0404B46
:10A330001E78012E95D1444802F032FA2878FCF7B5
:10A34000EDF80023414A13703B4A2B481370404BF1
:10A350001E70F8F7E9FA042397E72748F8F7EAFAB6
:10A36000054638B1354802F01BFA0022384B1A7006
:10A3700010238AE72B4E3378012B08D0022BA0D173
:10A38000304B1F78012F7FF46CAF324805E02F4B24
:10A390001F78012F7FF465AF2F4802F001FA307863
:10A3A000FCF7E4F82A4B12481D702C4B1F70F8F78D
:10A3B000BBFA052369E70E48F8F7BCFA00283FF41A
:10A3C00050AF00231C4A1370214A137073E7A52075
:10A3D00000F0FEFD0748F8F7A7FA112355E70548F6
:10A3E000F8F7A8FA00283FF43CAFE2E78014002019
:10A3F00078140020701400206814002067140020D6
:10A40000040E00200C0E00200D0E00201400002071
:10A41000280E00201B4801081E4901082E4801088B
:10A42000544801080F0E002005000020991000205C
:10A4300097100020951000208E100020314901084F
:10A4400062490108941000204C4901089610002030
:10A450008D1000208E4901087849010891100020D4
:10A4600038B5074D2C7854B9064A1378012B06D11C
:10A470001470054A0548137002F092F92C7038BD2B
:10A4800066140020030E0020610E0020A44901087C
:10A4900038B5194C2378012B0DD0102B2BD04BB98C
:10A4A00016490A78012A05D10B70154922700B70E4
:10A4B00014490B7038BDFFF7C9FB012805460CD1C4
:10A4C000114802F06DF900F01DFD00220F4B1D70C8
:10A4D0000A4B1A7010232370ECE70A4A1378012BF9
:10A4E000E8D100231370054A237013700848BDE8B3
:10A4F000384002F055B9FEE765140020020E002036
:10A500000C0E00200D0E0020B94901089210002009
:10A510005448010838B5194B1A782AB90122142178
:10A5200017481A70F8F7F8F9164C237813B1012B75
:10A5300013D038BD144A1578012DFAD1137000F0EC
:10A54000A1FAFEF7A1FEFDF7E3FBFEF7F7FC25708D
:10A550000B48BDE83840F8F7E7B90948F8F7EAF9D9
:10A560000028E6D0094B1B78012B04D1FBF71AFD1C
:10A5700000232370DDE7FBF751FDF9E764140020A9
:10A580005C140020591400200E0E0020050000204D
:10A5900010B5124C2378012B07D1114802F000F9B5
:10A5A000002310482370FFF743F8FFF771FBFFF714
:10A5B000C3FBFFF7E1FBFFF75BFCFFF7ADFCFFF729
:10A5C0000DFDFFF76DFDFFF717FEFFF749FFFFF7E2
:10A5D0005FFFBDE81040FFF79DBF00BFDA1100200C
:10A5E000D0490108AE3800202DE9F74FA64B1A7864
:10A5F0002AB901226421A5481A70F8F78DF9A44BF5
:10A6000093F800A0BAF1000F00F00581A14BA24A17
:10A610001B781278934200F201816426D21AD2B2DA
:10A620005643B6FBFAF69D4BF6B21B789246B34200
:10A630008CBF002301239A4A13709A4A92F8009023
:10A64000B9F1000F00F0EE80974A98491278097826
:10A650008A4200F2EA806425891AC9B24D43B5FBEB
:10A66000F9F5934AEDB212788946AA428CBF0022CE
:10A670000122DFF840B28BF800208F4A92F8008068
:10A68000B8F1000F00F0D5808C4A8D491278097816
:10A690008A4200F2D1806424891AC9B24C43B4FBC7
:10A6A000F8F4884AE4B212788846A2428CBF0022AD
:10A6B000012285490A70854A1778002F00F0C08072
:10A6C000834A8449127809788A4200F2BC80891A48
:10A6D0006422C9B24A43B2FBF7F2D2B201927E4A77
:10A6E000019812780F4682428CBF002201227B49DA
:10A6F00001200A707A4A1288022A04D0794A128804
:10A70000022A40F0A480F8F7DFFF0220F8F7C2FF2A
:10A710000320F8F7D9FF0420F8F7BCFF604B724A1A
:10A720001B7812789A4211D1704A11789BF8002058
:10A7300091420BD16E4A1178634A1278914205D149
:10A740006C4A1178654A127891423CD0012B0CBFBB
:10A7500069486A4802F024F8514B4E491A78624B16
:10A7600009781A7066485246334602F019F89BF889
:10A770000030012B0CBF6348634802F011F89BF8CE
:10A7800000205A4B48491A7009782B464A465F48C0
:10A7900002F006F84C4B49491A78554B09781A7063
:10A7A0004E4B5B481A78534B1A702346424601F0D1
:10A7B000F7FF47493A46019B0978564801F0F0FFF8
:10A7C0006220F6F7DBFC3148F8F7B4F8002800F017
:10A7D000B1802E48F8F7A8F82E493346524609783A
:10A7E0004D4801F0DDFF30492B464A4609784B4879
:10A7F00001F0D6FF3149234642460978484801F026
:10A80000CFFF3A463249019B0978464803B0BDE87C
:10A81000F04F01F0C5BF534656460CE700231E46D5
:10A820009A4608E74A464D4623E7002215469146D8
:10A830001FE7424644463CE700221446904638E76C
:10A840003A46019753E70022174601924FE7C3B1FA
:10A85000F8F720FF9BF800300220002B64D0F8F7B7
:10A8600019FF194B03201B78002B60D0F8F712FF5B
:10A870001A4B04201B78002B7FF44EAFF8F724FF0F
:10A880004CE7F8F721FFE5E798140020901400202A
:10A8900011000020840B0020100000200F00002079
:10A8A000CB0E00200E000020830B00200D000020A6
:10A8B0000C000020CA0E00200B000020820B00209C
:10A8C0000A00002009000020C90E00200800002016
:10A8D000810B00200700002006000020C80E002089
:10A8E000FE0D0020FC0D00208C1400208B14002095
:10A8F0008A14002089140020EA490108F649010859
:10A90000044A0108244A0108304A01083E4A010865
:10A910005E4A01087E4A01089E4A0108C54A0108AC
:10A92000EC4A0108134B0108F8F7CEFE99E7F8F757
:10A93000CBFE9DE703B0BDE8F08F00BF00B589B046
:10A9400002460649684601F09FFD684603F002FC96
:10A9500081B26846F8F796F909B000BD3A4B010894
:10A9600007B50121092000F019FE0121074800F078
:10A9700097FD074B01A90748019300F038FD082116
:10A98000044800F08BFD03B000BD00BF00023000A2
:10A9900008000310000C014008B5FFF7E1FFBDE817
:10A9A00008401420FFF7CABF00B589B002460A4923
:10A9B000684601F069FD0821084800F06DFD01229C
:10A9C000074B68461A7003F0C5FB81B26846F8F77A
:10A9D00059F909B000BD00BF404B0108000C01400F
:10A9E000A51400200122024B1A70024B1870704708
:10A9F000A7140020A614002038B51A4B1A782AB9DB
:10AA00000122322118481A70F7F786FF174C237875
:10AA1000012B10D0022B0DD08BB9154A1578012DC2
:10AA200008D11370134B1878FFF7BEFF0E48F7F7E5
:10AA30007BFF257038BD0E4B1B78012B01D1002305
:10AA40000EE00948F7F776FF0028F3D00A4801F036
:10AA5000A7FE0821094800F021FD0023084A1370D1
:10AA60002370E7E7A41400209C1400209A1400200F
:10AA7000A7140020A6140020484B0108000C014038
:10AA8000A5140020F8B55F4D5F48296801F088FEE5
:10AA90005E4C00F0DBFF5E4801F012F84FF6FF71EC
:10AAA0005B4801F02DF861885A4801F029F82188A7
:10AAB000594C5A4801F024F86188594801F020F8AF
:10AAC0002188584801F01CF8574B58481978584BC2
:10AAD000584E1B78584C43EA012101F011F8574BAE
:10AAE00057481978574B584F1B7843EA012101F01A
:10AAF00007F8564B56481978564B1B7843EA012104
:10AB000000F0FEFF544B55481978554B1B7843EA2B
:10AB1000012100F0F5FF534B53481978534B1B7834
:10AB200043EA012100F0ECFF514B52481978524B97
:10AB30001B7843EA012100F0E3FF504B504819789D
:10AB4000504B1B7843EA012100F0DAFF4E4B4F488F
:10AB500019784F4B1B7843EA012100F0D1FF4D4B90
:10AB60004D4819784D4B1B7843EA012100F0C8FF8E
:10AB70004B4B4C4819784C4B1B7843EA012100F0B1
:10AB8000BFFF4A4B4A48197800F0BAFF2968494884
:10AB900001F006FE31787378204643EA0121023441
:10ABA00000F0AEFFBC4206F10206F3D1296842482C
:10ABB00001F0F6FD414B20461978414B1B7843EAE2
:10ABC000012100F09DFF3F4B3F4819783F4B1B7818
:10ABD00043EA012100F094FF3D4B3E48198800F004
:10ABE0008FFF40F60B210A4800F08AFF00F03AFF81
:10ABF0002968394801F0D4FDBDE8F840374801F034
:10AC0000CFBD00BFC40F0020574B01084C0E0020E1
:10AC100000F8070802F80708480E002004F80708A3
:10AC200006F8070808F80708550E00200AF8070874
:10AC3000540E0020CB17002038F80708530E0020D0
:10AC40000CF80708460E002058F80708450E0020AB
:10AC50000EF80708440E0020520E002010F80708D6
:10AC6000430E0020420E002012F80708410E00207B
:10AC7000510E002014F80708400E00203F0E00205F
:10AC800016F807083E0E0020500E002018F807089E
:10AC90003D0E00203C0E00201AF807083B0E002055
:10ACA0003A0E002034F80708390E0020380E002034
:10ACB00036F80708664B0108754B0108370E00206F
:10ACC000360E0020350E00205AF80708340E0020FA
:10ACD000320E00205CF80708844B0108934B0108F2
:10ACE00040F60B212DE9F04F634B93B01A8892B2D6
:10ACF0008A4240F0BB805988604C89B221609A88B2
:10AD00005F4D92B242EA01422260D9885D4E89B21B
:10AD100029601A895C4F92B242EA01422A605A893C
:10AD2000DFF86881110A31703A709A89DFF8609112
:10AD3000110A88F8001089F80020DA895549100AAC
:10AD4000087055490A701A8A5449100A0870544903
:10AD50000A705A8A5349100A087053490A709A8A2D
:10AD60005249100A087052490A70DA8A5149100A89
:10AD7000087051490A701A8B5049100A08705049DE
:10AD80000A705A8B4F49100A08704F490A709A8E00
:10AD90004E49100A08704E494E480A70DA8E4E4BE2
:10ADA0001A704E4B4E4A32F8021B02334FEA112CF6
:10ADB000824203F802CC03F8011CF4D12E4BDFF8D9
:10ADC00024A1B3F85820DFF820B1110A8AF8001046
:10ADD0008BF80020B3F85A00444A010A1170444924
:10ADE0000870B3F85C00434B1880434801F0D8FC6E
:10ADF000404B3F491B883D4A11930B783F481093C5
:10AE000013780F939BF800300E939AF800300D934F
:10AE1000324B0C93304B1B780B932D4B1B780A93C2
:10AE20002A4B1B780993204B1B7808931D4B1B78EA
:10AE300007931B4B1B780693184B1B780593164BF7
:10AE40001B780493134B1B78039399F800300293FB
:10AE500098F8003001933B78009333782A68216892
:10AE600001F09EFC002013B0BDE8F08F244801F0F3
:10AE700097FC0120F7E700BF00F807084C0E002000
:10AE8000480E0020550E0020540E0020530E0020C6
:10AE9000460E0020450E0020440E0020520E0020D9
:10AEA000430E0020420E0020410E0020510E0020D3
:10AEB000400E00203F0E00203E0E0020500E0020CD
:10AEC0003D0E00203C0E00203B0E00203A0E0020DC
:10AED000390E002058F80708380E0020CB17002044
:10AEE00038F80708370E0020360E0020350E0020F7
:10AEF000340E0020320E0020A64B0108B94B010889
:10AF00004F4C010808B500F0A1FD054800F0D8FD40
:10AF100000F0A8FDBDE80840024801F041BC00BFB8
:10AF200000F807086A4C0108FF2810B514D00B4C34
:10AF30000F3024785C436FF0630394FBF3F440F22A
:10AF4000A3631444A4B2A04288BF1046994202D819
:10AF50004A2898BF1046C0B210BD00BF12000020A2
:10AF6000682270B5194BA0B000938DF805200378C6
:10AF700042788DF804308DF806201344082210F82A
:10AF8000021F303B01F109058DF807100B44EDB2AB
:10AF900014460132D2B28034AA426C440FD104F874
:10AFA000803C02F180030DEB030216230A31684650
:10AFB000C9B202F8803CF7F7C7FE20B070BD10F8A8
:10AFC000016F04F8806C3344E2E700BFFEFEFE68C8
:10AFD00038B5002305460B4C014660700A482370C3
:10AFE00001F0DEFBA12D0ABF04210321074B054818
:10AFF00004BF1B78E370CB1EA370BDE83840FFF799
:10B00000AFBF00BF5A3A00208D4C010899100020B4
:10B010002DE9F7435E4D2B78FD2B11D15D4C637804
:10B02000032B00F08D800ED8012B1BD0022B00F0DB
:10B03000838080220021574801F0C4FB00232B703D
:10B0400003B0BDE8F083A22B00F09280A32BF0D1D7
:10B05000E378514A012B137000F09780022BE8D15E
:10B060004E4B67E0B4F803304D4A5BBA138099B297
:10B07000B4F805304B4A5BBA13809EB2B4F807307F
:10B08000494A5BBA13801FFA83F8B4F80930474A7B
:10B090005BBA1FFA83F91380454B1B78002B39D11B
:10B0A000444B454A1B781278E07AFFF73DFF434B4B
:10B0B000434A1870434B07461B7831461278207B71
:10B0C000FFF732FF404B414A1870414B06461B7850
:10B0D00041461278607BFFF727FF3E4B3E4A1870CF
:10B0E0003E4B80461B7812784946A07BFFF71CFF39
:10B0F0003B4B324618703B4B39461F703A4B1E7023
:10B100003A4B83F800803A4B187000904346394818
:10B1100001F046FBE27B384B1A70227C374B1A70E9
:10B12000627C374B1A70A27C364B1A70364BE27C2D
:10B130001A70364B012201E0E278354B1A7078E73D
:10B14000E278344B1A702279334B1A706279334BA0
:10B150001A70D4F80630324A1BBA1360A27A314B07
:10B160001A70D4F80B30304A1BBA13602F4BE1E74A
:10B17000E378094A012B137004D0022B7FF459AFF6
:10B180002B4BD7E72B4A137053E72B4AFBE700BF43
:10B19000CE0F00204C250020981000209410002095
:10B1A000A01000209E1000209C1000209A1000206B
:10B1B000CC0E0020110000201000002021000020F3
:10B1C0000D0000200E000020200000200A000020BA
:10B1D0000B0000201F0000200700002008000020B6
:10B1E0001E000020840B0020830B0020820B002017
:10B1F000810B0020A14C0108F1110020E30E00207A
:10B20000F3110020E70E0020E60E0020000E0020C3
:10B2100006100020DE0E0020DD0E0020DC0E0020D7
:10B22000D80E0020D40E0020D00E0020CD0E00201D
:10B2300095100020971000209610002008B50520DA
:10B24000FBF7C0FB034801F0ABFA0122024B1A7076
:10B2500008BD00BFC44C0108AB14002008B5052090
:10B26000FBF7FCFB034801F09BFA0022024B1A702B
:10B2700008BD00BFD74C0108AB14002008B503205F
:10B28000FBF710FD034801F08BFA0122024B1A7004
:10B2900008BD00BFEA4C0108A914002008B503202E
:10B2A000FBF74CFD034801F07BFA0022024B1A70B9
:10B2B00008BD00BF014D0108A914002008B56FF0BA
:10B2C000040000F089F8084B084A1B68B3FBF2F34E
:10B2D000074ADBB21370C3EB431203EB8203054A48
:10B2E000DB00138008BD00BF0000002000127A00C0
:10B2F000AE140020AC1400200B4B00221B785843E6
:10B300004FF0E02358619A611A6942F001021A6114
:10B310001A69D10701D5D203FAD51A6922F00102C0
:10B320001A6100229A617047AE1400200B4B002274
:10B330001B8858434FF0E02358619A611A6942F024
:10B3400001021A611A69D10701D5D203FAD51A6927
:10B3500022F001021A6100229A617047AC140020A9
:10B36000034B40F0BF6040F40030D860704700BF2E
:10B3700000ED00E030B5C2780378EAB1144A0F2539
:10B38000D1684478C943C1F30221C1F10402944059
:10B39000827825FA01F10A400E49224312010B443A
:10B3A00083F8002301220378580903F01F0302FAEF
:10B3B00003F341F8203030BD01215A0903F01F0387
:10B3C000994002F12003034A42F82310F3E700BF3B
:10B3D00000ED00E000E100E04FF0E0231A690428EE
:10B3E0000CBF42F0040222F004021A617047CB78CD
:10B3F000F0B503F00F04DB0644BF8B781C430B78D9
:10B40000D3B1002201274FF00F0C03680D8807FA13
:10B4100002F636EA05050BD195000CFA05FE23EA83
:10B420000E0304FA05F52B43CD78282D2AD1466169
:10B430000132082AEAD103600B88FF2B21D90023AF
:10B440004FF0010C4FF00F0E46680D8803F1080213
:10B450000CFA02F232EA05050FD19D000EFA05F74B
:10B4600026EA070604FA05F52E43CD78282D08BFF5
:10B470004261CD78482D08BF02610133082BE4D129
:10B480004660F0BD482D08BF0661D1E783681942C8
:10B4900014BF01200020704701617047416170476F
:10B4A00030B50028164C00F44015B4BFE36963685A
:10B4B000B5F5401F82B212D1656823F0706325F0A4
:10B4C00070656560440D2401A2401A43002918BF2D
:10B4D00013460B4A0028B4BFD361536030BDC40289
:10B4E0004DBF0324440D2401C0F303454CBFAC40C1
:10B4F00002FA04F423EA040343F07063E2E700BFB6
:10B500000000014010B51A4A536803F00C03082BE1
:10B510002CD153685168C3F38343CC0303F1020376
:10B5200002D5516889031FD512494B430360516806
:10B53000114CC1F30311615CCB4043605168C1F30E
:10B540000221615C23FA01F181605168C1F3C221DB
:10B55000615CCB40C36052680849C2F381328A5CA7
:10B56000B3FBF2F3036110BD0549DEE7044BDDE7F1
:10B570000010024000093D00515201084D520108DF
:10B5800000127A00044B5A6911B102435A617047A4
:10B5900022EA0002FAE700BF00100240044B9A6959
:10B5A00011B102439A61704722EA0002FAE700BF34
:10B5B00000100240044BDA6911B10243DA617047AE
:10B5C00022EA0002FAE700BF00100240044BDA68EA
:10B5D00011B10243DA60704722EA0002FAE700BFC5
:10B5E00000100240044B1A6911B102431A617047FE
:10B5F00022EA0002FAE700BF0010024008B5214B22
:10B6000098420BD101214FF48040FFF7DFFFBDE8E6
:10B61000084000214FF48040FFF7D8BF1A4B9842F2
:10B620000BD101214FF40030FFF7DCFF00214FF474
:10B630000030BDE80840FFF7D5BF144B984208D151
:10B6400001214FF48020FFF7CDFF00214FF480202F
:10B65000EFE70F4B984208D101214FF40020FFF78C
:10B66000C1FF00214FF40020E3E70A4B984208D1C4
:10B6700001214FF48010FFF7B5FF00214FF4801037
:10B68000D7E708BD003801400044004000480040B2
:10B69000004C00400050004030B50446038ACA8880
:10B6A00023F44053134387B0038283898A8823F4A9
:10B6B000B05323F00C0313430A890D4613434A8900
:10B6C00013438381838A8A8923F4407313438382DB
:10B6D00001A8FFF717FFDDE9033214498C4208BFC8
:10B6E00013461922A18953432A680D044CBF520006
:10B6F00092006421B3FBF2F3B3FBF1F201FB1233CE
:10B70000A08900044BBFDB001B01323332334BBF37
:10B71000B3FBF1F3B3FBF1F303F0070303F00F0303
:10B7200043EA0212228107B030BD00BF0038014059
:10B73000838919B143F400538381704723F4005384
:10B74000FAE7012310B5C1F34214012C01F01F01E7
:10B7500003FA01F305D10C3042B1026813430360D0
:10B7600010BD022C0CBF10301430F5E7026822EA3D
:10B770000303F4E7838A12B119438182704723EAF5
:10B78000010383827047C1F308018180704780887C
:10B79000C0F3080070470388194214BF012000203D
:10B7A0007047C943018070470123C1F3421210B5AD
:10B7B000012A01F01F0403FA04F30FD1828992B227
:10B7C000134001220088090A8A4080B21040002BF1
:10B7D00018BF002814BF0120002010BD022A0CBF92
:10B7E000028A828AEBE70000214A0388904212D045
:10B7F00002F5006290420ED0B0F1804F0BD0A2F55E
:10B800009832904207D002F58062904203D002F550
:10B810008062904203D14A8823F070031343154A93
:10B82000904207D002F5806290421EBFCA8823F47E
:10B830004073134303808B8883850B8803850C4BEF
:10B8400098420FD003F5006398420BD003F5406394
:10B85000984207D003F58063984203D003F58063D4
:10B86000984201D10B7A038601238382704700BF7F
:10B87000002C014000100040038819B143F001037F
:10B880000380704723F00103FAE7838912B119435B
:10B890008181704723EA0103838170478184704767
:10B8A000038A8289114214BF01200020194200F04E
:10B8B000010008BF00207047C943018270470000A3
:10B8C000036823F001031B041B0C036000230360C7
:10B8D00043608360C360294B984204D1284A53686F
:10B8E00043F00F0326E0274B984204D1244A5368C3
:10B8F00043F0F0031EE0244B984204D1204A5368E1
:10B9000043F4706316E0214B984204D11C4A5368FB
:10B9100043F470430EE01E4B984204D1184A53681A
:10B9200043F4702306E01B4B984205D1144A536838
:10B9300043F4700353607047174B984204D1104A88
:10B94000536843F07063F5E7144B984201D1144AF1
:10B95000C5E7144B984201D1114AC8E7124B9842EF
:10B9600001D10F4ACBE7114B984201D10C4ACEE7E7
:10B970000F4B9842DFD10A4AD1E700BF08000240CE
:10B98000000002401C00024030000240440002401F
:10B99000580002406C00024080000240080402404F
:10B9A000000402401C0402403004024044040240EF
:10B9B0005804024010B58B680C6A026823430C6976
:10B9C0006FF30E1223434C6923438C692343CC69E4
:10B9D00023434C6A23438C6A234313430360CB689D
:10B9E00043600B6883604B68C36010BD036819B186
:10B9F00043F001030360704723F001031B041B0C99
:10BA0000F8E7416070470000014B1860704700BFC5
:10BA100000300040014B5860704700BF00300040CC
:10BA2000014B9860704700BF003000404AF6AA22E0
:10BA3000014B1A60704700BF003000404CF6CC420A
:10BA4000014B1A60704700BF00300040034B044AAE
:10BA50005A6002F188325A60704700BF00200240ED
:10BA600023016745024A136943F08003136170475D
:10BA700000200240084BDA68D10709D4DA6852077F
:10BA800008D4DB6813F0100F0CBF042003207047AC
:10BA900001207047022070470020024010B5044684
:10BAA000FFF7E8FF012806D10CB9052010BDFFF70C
:10BAB000E1FF013CF6E7002C08BF0520F6E7000097
:10BAC00038B505464FF43020FFF7E8FF042813D1BE
:10BAD0000A4C4FF43020236943F00203236165616F
:10BAE000236943F040032361FFF7D8FF236923F064
:10BAF0000203DB04DB0C236138BD00BF00200240E1
:10BB000070B505464FF400500E46FFF7C7FF0428F6
:10BB10000FD1084C4FF40050236943F00103236117
:10BB20002E80FFF7BBFF236923F00103DB04DB0C4E
:10BB3000236170BD0020024070B50E4615460024FA
:10BB4000AC4201DB284670BD40210548FFF723FECB
:10BB50000028F9D0315D0248FFF715FE0134EFE708
:10BB6000005000400D480E490E4A914200D304E0B7
:10BB700050F8043B41F8043BF7E70B490B4A00231C
:10BB8000914200D302E041F8043BF9E7F4F74AFCA4
:10BB900001F044FAF4F786FBFEE700005456010872
:10BBA00000000020B80D0020B80D00205C3B0020F4
:10BBB000FEE70A22002100F0CBBD002B2DE9F04763
:10BBC0001D46BBBF03F100431D4600232D2388B053
:10BBD000149F144627F02007B8BF1446129A462F28
:10BBE000109EDDF84CA0137004D0452F00D1013613
:10BBF000022300E0032307AA049206AACDE902A2C9
:10BC0000CDE9003622462B4602F05EFB472F8046E8
:10BC10001AD1119BDB070ED500EB06090022002389
:10BC20002046294605F01EFD08B1CDF81C903022B3
:10BC3000079B4B451ED34046079B159AA3EB080371
:10BC4000136008B0BDE8F087462F00EB0609E5D188
:10BC50000378302B0AD1002200232046294605F024
:10BC600001FD18B9C6F10106CAF80060DAF8003023
:10BC70009944D3E7591C07911A70D9E7F7B5002901
:10BC8000B6BF2D232B2349420929027043702BDDB7
:10BC90000DF10704A6460A26871CB1FBF6F5A4465B
:10BCA00006FB1512632902F13002294604F1FF3424
:10BCB0000CF8012CF1DC3031ACF1020204F8011C6B
:10BCC0001446411C72450AD30DF10903A3EB0C0382
:10BCD000A64538BF00233B44181A03B0F0BD12F844
:10BCE000013B01F8013FEDE7302330318370C17033
:10BCF000031DF1E72DE9F04F93B00C46DDF870809D
:10BD000016461F46054602F0F3F9036818460B93E2
:10BD100002F020FA00231093D8F8003094F818A00D
:10BD2000073323F00703F3E80212D4F800B0CDE99B
:10BD30000812C8F8003013460A46C4E91223DDE9A8
:10BD4000088323F000490C904FF0FF3240464946EB
:10BD50009A4B05F0B9FC70BB4FF0FF3240464946A4
:10BD6000964B05F093FC30BBDDE90801002200236F
:10BD700005F082FC10B12D2384F84330904A914B9A
:10BD8000BAF1470F8CBF9046984603234FF0000945
:10BD900023612BF004032360334621462846009795
:10BDA00011AA00F0D1F9013040F08F804FF0FF3040
:10BDB00013B0BDE8F08FDDE908231046194605F001
:10BDC00083FC40B1099B804A002BBCBF2D2384F823
:10BDD00043307E4BD4E763680AF0DF095A1C3ED13A
:10BDE0000623636000224BF480632360069210AA4E
:10BDF000CDE904A20FAA03920DF13B02CDE9013275
:10BE0000636828460093DDE90823FFF7D6FEB9F101
:10BE1000470F80460F9929D1C81C02DB63688B420B
:10BE200041DAAAF1020A5FFA8AFA5246013904F1AC
:10BE300050000F91FFF722FF109A81461318012A34
:10BE4000236102DC2268D20701D5013323619DF80A
:10BE50003B30002BA0D02D2384F843309CE7B9F170
:10BE6000470FBFD1002BBDD10123BAE7BAF1650F4F
:10BE7000DBD9BAF1660F18D1002963680BDD2161A7
:10BE800013B92268D00702D501330B4423614FF068
:10BE90000009A165DBE713B92268D20701D5023397
:10BEA000F4E70123F2E74FF0670A109B8B4205DCB1
:10BEB00023682161D807EAD54B1CE7E70029CCBFEE
:10BEC0000122C1F102021344E0E723685A0507D4B6
:10BED0002369424631462846B847013028D165E7F4
:10BEE000BAF1650F40F2DC80D4E912010022002390
:10BEF00005F0B8FB90B3012331462846344AB847D1
:10BF000001303FF453AFDDE90F38434502DB2368CE
:10BF1000D8070DD5DDE90B2331462846B847013057
:10BF20003FF444AF4FF0000908F1FF38C84509DC81
:10BF300023689B0700F10581E068119B9842B8BF18
:10BF4000184635E701233146284604F11A02B8475E
:10BF500001303FF42BAF09F10109E7E70F9B834262
:10BF600038DC012331462846194AB84701303FF4EE
:10BF70001DAFDDE90F3959EA030302D12368D90760
:10BF8000D6D5DDE90B2331462846B84701303FF4CA
:10BF90000DAF4FF0000A0F9B5B42534501DC4B464F
:10BFA00097E701233146284604F11A02B8470130C9
:10BFB0003FF4FCAE0AF1010AEDE700BFFFFFEF7F9F
:10BFC0001C4D0108184D0108244D0108204D0108A1
:10BFD00013300108A36DDDF840B05B45A8BF5B4698
:10BFE000002B089337DC4FF0000904F11A02089B7C
:10BFF000D4F858A0002BB4BF5346AAEB03034B451B
:10C0000031DC0F9B9B453ADC2368DA0737D40F9B62
:10C01000ABEB0309ABEB0A039945A8BF9946B9F10D
:10C02000000F34DC4FF000080F9BB9F1000FABEBB1
:10C030000303A8BFA3EB090343457FF779AF0123AF
:10C040003146284604F11A02B84701303FF4AEAE3B
:10C0500008F10108E8E7424631462846089BB84700
:10C060000130C0D1A2E60123314628460D92B847DF
:10C0700001303FF49BAE0D9A09F10109B7E7314653
:10C08000DDE90B232846B8470130C0D18EE64B4688
:10C090003146284608EB0A02B8470130C2D185E68E
:10C0A000DDF840A0BAF1010F01DCDB0735D5012333
:10C0B000424631462846B84701303FF477AEDDE9C5
:10C0C0000B2331462846B84701303FF46FAED4E920
:10C0D0001201002200230AF1FF3A05F0C3FAC8B9A1
:10C0E000534608F1010231462846B84701300DD1C8
:10C0F0005CE601233146284604F11A02B8470130B4
:10C100003FF454AE08F10108D045F2DB4B4604F190
:10C110005002DFE64FF00008F6E701234246E2E76F
:10C1200001233146284604F11902B84701303FF493
:10C130003DAE08F10108E36811995B1A4345EFDC55
:10C14000FAE64FF00008F6E72DE9F04791469846E9
:10C150008A680B6907469342B8BF1346C9F8003096
:10C1600091F843200C46089E12B10133C9F8003003
:10C170002368990642BFD9F800300233C9F800306D
:10C18000256815F0060507D104F1190AE368D9F806
:10C1900000209B1AAB4229DC94F843302268003B14
:10C1A00018BF012392062ED44146384604F14302BB
:10C1B000B047013021D02368A16803F00603042BA7
:10C1C00012BF0025E568D9F80030226904BFED1AD6
:10C1D00025EAE5758B1A2B449142C8BF1D464FF0E6
:10C1E00000091A344D451AD1002008E001235246B7
:10C1F00041463846B047013003D14FF0FF30BDE82B
:10C20000F0870135C2E73020E11881F843005A1C5D
:10C2100094F845102244023382F84310C4E7012306
:10C22000224641463846B0470130E6D009F10109BF
:10C23000D8E700002DE9F04398460B7E85B0782BB7
:10C24000174606460C460C9A09D8622B01F14301A9
:10C2500008D8002B00F0DC80582B00F0BD8004F1E2
:10C26000420539E0A3F163001528F8D801A555F877
:10C2700020F000BFCDC20008E1C200085FC2000884
:10C280005FC200085FC200085FC20008E1C2000888
:10C290005FC200085FC200085FC200085FC20008FA
:10C2A000F1C300080DC300089FC300085FC2000867
:10C2B0005FC2000819C400085FC200080DC300086F
:10C2C0005FC200085FC20008A7C30008136804F13A
:10C2D0004205191D1B68116084F842300123A8E053
:10C2E00013682568181D1060280601D51B6803E037
:10C2F0006A06FBD5B3F90030002B03DA2D225B422E
:10C3000084F843200A22DFF878C113E0256810681A
:10C3100015F0800F50F8043B02D16D0648BF9BB268
:10C320001060227EDFF858C16F2A5DD108220020FC
:10C3300084F843006568002DA56005DB20681D4377
:10C3400020F00400206051D00D46B3FBF2F002FB58
:10C35000103E1CF80EE09A4205F801ED0346F4D9B0
:10C36000082A0BD12368DA0708D5236962689A4244
:10C37000DEBF302305F8013C05F1FF35491B216183
:10C380003B4621463046CDF8008003AAFFF7DCFE8D
:10C39000013053D14FF0FF3005B0BDE8F083236882
:10C3A00043F0200323607823DFF8D8C084F84530B9
:10C3B0002068156810F0800F55F8043B03D110F089
:10C3C000400F18BF9BB21560C50744BF40F0200066
:10C3D000206023B11022AAE7DFF8A4C0E6E72268B4
:10C3E00022F020022260F5E70A22A0E70D46B7E717
:10C3F0001368D4F800C01D1D60691CF0800F156023
:10C400001B6801D0186003E01CF0400FFAD01880C0
:10C4100000230D462361B3E71368191D11601D68E1
:10C4200000212846626801F079FE08B1401B606077
:10C4300063682361002384F84330A1E72A46394624
:10C4400030462369C0470130A4D023689B0714D429
:10C45000E068039B9842B8BF18469DE70123394620
:10C46000304604F11902C047013093D00135E3682A
:10C4700003995B1AAB42F1DCEAE70025F7E700BF5E
:10C48000284D0108394D01080EB46FF0004110B578
:10C4900000249DB01FAB02900690079104910948BB
:10C4A000094953F8042B0591006802A901931B94D4
:10C4B00002F08EFD029B1C701DB0BDE8104003B061
:10C4C000704700BF9C0B00200802FFFF002310B53F
:10C4D0000446C0E90033C0E90433836081814366C8
:10C4E000C2818361194608225C3000F06BF90D4B64
:10C4F000246263620C4BA3620C4BE3620C4B23631C
:10C500000C4B9C4206D003F16802944202D0D03317
:10C510009C4205D104F15800BDE8104001F0BCBBBD
:10C5200010BD00BF99FD0008BFFD0008F7FD000821
:10C530001DFE0008B0140020024A0349034800F021
:10C5400011B900BF880B00201DFF0008A00B0020C0
:10C5500041680C4B10B59942044601D003F0DEFC53
:10C56000A168094B994202D0204603F0D7FCE1684C
:10C57000064B994204D02046BDE8104003F0CEBCE3
:10C5800010BD00BFB0140020181500208015002039
:10C5900010B50A4B0A4A04211A600A480022FFF724
:10C5A00095FF012209210848FFF790FFBDE81040E0
:10C5B000022212210548FFF789BF00BFE8150020BD
:10C5C00039C50008B014002018150020801500207F
:10C5D000014801F063BB00BFEF150020014801F0E6
:10C5E0005FBB00BFEF15002010B50446FFF7F0FF5A
:10C5F000236A1BB1BDE81040FFF7F0BF044B236274
:10C60000044B1B68002BF5D1FFF7C2FFF2E700BF18
:10C6100051C50008E815002010B59AB000910491AA
:10C620006FF000410024059102910549199403918E
:10C63000694602F0CDFC009B1C701AB010BD00BF13
:10C640000802FFFF13460A46014602480068FFF74A
:10C65000E3BF00BF9C0B0020242B2DE9F047884648
:10C6600001D8012B06D100F0D3FC16230360002073
:10C67000BDE8F0870D46344E294615F8014B375D6D
:10C6800017F00807F8D12D2C10D101272C788D1C1C
:10C6900033F0100115D1302C0DD1297801F0DF01D4
:10C6A000582908D16C78023510230AE02B2C04BFDE
:10C6B0002C788D1CECE7002BF6D1302C14BF0A230C
:10C6C0000823002107F1004E0EF1FF3EBEFBF3F9F7
:10C6D0000E4603FB19EAA4F1300CBCF1090F10D887
:10C6E0006446A3421EDDB1F1FF3F07D0B14516D32A
:10C6F00001D1A24513DB012106FB034615F8014BCE
:10C70000E9E7A4F1410CBCF1190F01D8373CE8E787
:10C71000A4F1610CBCF1190F04D8573CE1E74FF0CC
:10C72000FF31EBE74B1C05D122237646036032B97B
:10C7300030469DE707B17642002AF9D009B105F1EC
:10C74000FF38C2F80080F3E721540108FFF784BFE7
:10C7500013460A46014602480068FFF77DBF00BF46
:10C760009C0B00202DE9F84380468946144600269C
:10C77000D4E90175013F05D52468002CF8D1304675
:10C78000BDE8F883AB89012B07D9B5F90E30013329
:10C7900003D029464046C84706436835EAE700000B
:10C7A0000FB407B5064904AB086853F8042B816839
:10C7B000019302F0DBFD03B05DF804EB04B07047B9
:10C7C0009C0B002003460244934200D1704703F8BB
:10C7D000011BF9E7034670B51C781E4644B10133CE
:10C7E0004A1E01E0A542F7D012F8015F002DF9D1F1
:10C7F000301A70BD1B4B2DE9F0411C680646656C74
:10C800000F463DBB502002F0DBFC606428B90246B5
:10C810005B21154B154801F0A9FC8560626CC0E9ED
:10C820000055C2E90355626C2B46C2E90555626C9E
:10C83000C2E90A55626CC2E90C55626CC2E90E5538
:10C84000626CC2E91055626CC2E91255626C1577D0
:10C85000656C6B622A4639463046BDE8F0410123DB
:10C8600000F006B89C0B00204A4D0108614D0108FC
:10C87000F0B5044608B9146844B1204614F8015BC9
:10C880004F1E17F8016F1EB965B91560002005E04D
:10C89000B542F6D1002BF0D114600370F0BD1C46F8
:10C8A0000CE01DB9274614F8013B4E1E16F8015F37
:10C8B000AB42F6D1002BF2D000233B701460EDE7C1
:10C8C0000A7870B56AB970BD9A4209D10C4605461E
:10C8D00014F8013F002BF6D015F8016F9E42F7D0F7
:10C8E00001300378002BEFD11846ECE738B50B4B3D
:10C8F00005461C68626B52B9242002F061FC0246B6
:10C90000606320B93221064B064801F02FFC28460F
:10C91000BDE83840114600F007B800BF9C0B00206E
:10C920004A4D0108C44D01082DE9F0410C46064668
:10C9300003F034FD21460746304603F033FD4369DA
:10C940000446990703F26C7806D1642298FBF2F34F
:10C9500002FB1383002B6FD14FF4C87398FBF3F5E0
:10C9600003FB1585B5FA85F56D09644B6D4205F03D
:10C9700030051D4401F07EF901F088F9604B1B6819
:10C98000002B68D07B68434558D1D6E90023D7E90E
:10C9900008013E68002E59D1824273EB01015CDB35
:10C9A000012323623B6D4FF4616293FBF2F002FBC3
:10C9B00010333C2293FBF2F602FB163321686268C7
:10C9C000C91AA368921B1B1A3B2921606260A360ED
:10C9D0004FDD013262603C3921603B2A4FDD01337B
:10C9E000A3603C3A6260172B4FDDE269183B0132CD
:10C9F000E261A269A3600132072AA8BF0022A261F6
:10CA0000E26823690132E26055F823108A420EDDA4
:10CA10000B2BA2EB0102E26003F1010205BF002231
:10CA200063692261013302BF22616361E26101F047
:10CA300027F92046BDE8F081012596E7404601F040
:10CA400067F80028A1D14FF0FF3304E0824273EB76
:10CA5000010102DA0023236209E0D7E912018242D0
:10CA60008B41B4BF012300232362002B9AD1BB6A00
:10CA700099E70029B1DA013A62603C31ACE7002A5B
:10CA8000B1DA013BA3603C32ACE7002BCFDAE269BC
:10CA90001833013AE261A269A360013A48BF062255
:10CAA000A261E268013AE260002AC0D12369013B39
:10CAB00004D4236155F82330E360B8E70B232361E6
:10CAC00063695A1E6261920703F26B7305D1642198
:10CAD00093FBF1F201FB12326AB94FF4C87293FB77
:10CAE000F2F102FB1133B3FA83F35B0903F5B6737A
:10CAF000E3610B23DEE70123F8E700BFC45201081E
:10CB000010160020F7B5016804463B2911D93C22D4
:10CB1000684601F049FB019A63680099002A0B44BA
:10CB20006360BBBF3C3203F1FF3322602260B8BFB9
:10CB3000636061683B2911D93C22684601F034FBEF
:10CB4000019AA3680099002A0B44A360BBBF3C3242
:10CB500003F1FF3362606260B8BFA360A168172968
:10CB600011D91822684601F01FFB019AE368009969
:10CB7000002A0B44E360BBBF183203F1FF33A2600D
:10CB8000A260B8BFE36021690B2911D90C22684665
:10CB900001F00AFB019A63690099002A0B44636162
:10CBA000BBBF0C3203F1FF3322612261B8BF636166
:10CBB00063699A073FD1642193FBF1F201FB1232C2
:10CBC000002A3AD14FF4C87203F26C7393FBF2F16E
:10CBD00002FB1133002B0CBF1D231C23E268002A2B
:10CBE0002DDD304D216901290CBF184655F8210073
:10CBF00082424DDD0131121A0C29E2602161F1D12E
:10CC0000002063692061591C8807616146D1642056
:10CC100091FBF0F600FB1611002941D14FF4C871C9
:10CC200003F26D7393FBF1F001FB1033002B0CBF8B
:10CC30001D231C23D6E71C23D0E71D23CEE70B259D
:10CC40006420184E216901392161013116D16369CF
:10CC5000591E8F07C4E904511CD191FBF0F700FB6A
:10CC60001711C9B94FF4C87103F26B7393FBF1F755
:10CC700001FB1733002B0CBF1D231C232169012945
:10CC80000CBF194656F821100A44002AE260D9DD8B
:10CC900003B0F0BD1C23F1E71D23EFE71C23A1E740
:10CCA0001D239FE7945201082DE9F74F074603F033
:10CCB00075FB81463846FFF725FFD7E90363D7E9BF
:10CCC0000041B448013E50F82300012BBA687D6949
:10CCD000064411DDA8070FD1642095FBF0F300FB9B
:10CCE000135343B94FF4C87005F26C7393FBF0FC17
:10CCF00000FB1C3303B9013644F6206005F51C53D4
:10CD000010338342FE6100F26D813C2303FB01443A
:10CD10004FF46163462D03FB024440F3B180462388
:10CD200040F26D1C64214FF4C8709A0740F0A28055
:10CD300093FBF1F201FB1232002A40F09E8003F2D5
:10CD40006C7292FBF0FE00FB1E22002A0CBF4FF417
:10CD5000B77262460133AB421644E6D18E4B4FEABE
:10CD6000E478C6FB034800F085FF00F08FFF8B4B93
:10CD70001B68002B00F04381D7F820A07869534648
:10CD8000012BA8BF01230193D9F8043000F26C7085
:10CD9000834240F0B880D9E91221D9F828C0D9F8E7
:10CDA0005030B2EB0C0B61EBEC7E5C4578EB0E0087
:10CDB00080F2CC80D9E90812D9F80000C91A62EBD8
:10CDC000E372002800F0CB808C4278EB0202C0F2C4
:10CDD00013815C4578EB0E0EB4BF4FF0010B4FF0A2
:10CDE000000BBAF1000FC0F29580019A82EA0B0A9B
:10CDF000BAF1010F40F08E80BBF1000F00F0BE8051
:10CE0000ACEB03033A681C191A443A60FA683846D6
:10CE100048EBE3780192FFF775FEFB68019A9B1AD5
:10CE200078D0012B00F3AD80B3F1FF3FA8BF9A4645
:10CE3000FB6956441AEB030340F1B2806B1E99075D
:10CE400040F0A280642293FBF2F102FB1133002B2D
:10CE500040F09D804FF4C87305F26B7595FBF3F2BB
:10CE600003FB1255002D40F26D1318BF4FF4B6733B
:10CE7000FB614FE040F26D126CE74FF4B77269E767
:10CE80003FF46CAF452340F26D1C64214FF4C87031
:10CE900012E062BB93FBF1F201FB123252BB03F2D0
:10CEA0006C7292FBF0FE00FB1E22002A0CBF4FF4B6
:10CEB000B7726246B61A013BAB4203F00302E8DCEC
:10CEC000DAB9642295FBF2F302FB1353C3B94FF4B2
:10CED000C87205F26C7393FBF2F102FB1133002B65
:10CEE00040F26D1308BF4FF4B773F61A36E740F2FD
:10CEF0006D12DFE74FF4B772DCE740F26D13F4E731
:10CF00004FF4B773F1E700F003FE00287FF443AF5E
:10CF1000DDF804B0BBF1010F73D14FF0010BD9F86C
:10CF200050301C1948EBE37800F0AAFE07230436C2
:10CF300096FBF3F3C3EBC303F61A51D4C7F820B042
:10CF4000BE612046414603B0BDE8F08FD21A61EBC6
:10CF5000E371944278EB0101BFF62CAFD8E78C4225
:10CF600078EB020242DA5C4578EB0E0EB4BF4FF06C
:10CF7000010B834635E74FF0000B36E7A3EB0C03BC
:10CF800040E74FF0FF3A53E74FF4B67370E740F2D3
:10CF90006D136DE7645201088051010010160020E6
:10CFA000AA0717D1642195FBF1F201FB1252A2B935
:10CFB0004FF4C87205F26C7595FBF2F102FB115546
:10CFC000002D40F26D1208BF4FF4B7729342A8BF14
:10CFD0009B1A4DE740F26D12F8E74FF4B772F5E790
:10CFE0000736ABE74FF0FF34A046AAE7BAF1000FCF
:10CFF00093DB4FF0010BF8E6BAF1000FBBDA4FF00C
:10D00000000BD9F828301C1948EBE3788CE700BFF7
:10D01000014B1868704700BF9C0B002070B50026BC
:10D020000C4C0D4B1D1BB6EBA50F09D1002608F0CB
:10D03000FDFA0A4C0A4B1D1BB6EBA50F05D170BDBE
:10D0400054F8043B98470136EDE754F8043B984701
:10D050000136F1E74C5601084C5601084C560108C0
:10D0600050560108426940F26C73002AA8BF6FF065
:10D0700063031344920705D1642193FBF1F201FB92
:10D080001232CAB94FF4C87293FBF2F102FB1133AA
:10D09000B3FA83F35B09D0E90602400000EB02100B
:10D0A000184441F2A263984227D011DC01280ADC1F
:10D0B000C043C00F404270470123ECE7104BC34010
:10D0C00043F3000070470A381728F7D9002070474B
:10D0D00041F2B463984206DC41F2B1639842D4BF96
:10D0E000002001207047A0F5B65002381528EDD871
:10D0F000044BC34003F0010070470120704700BF9C
:10D10000CF00CC001F002A002DE9F04F1E4600235F
:10D1100007460D461C468FB002931378002B00F093
:10D12000D984252B40F081805378302B00F0878004
:10D130002B2B00F08480002302F1010898F80020D6
:10D14000313AD2B2082A7DD840460A2206A9039372
:10D1500002F0FAFF8146DDF81880039B98F8001072
:10D16000452901D04F2901D108F1010898F80000A4
:10D17000A0F12501552900F25081DFE811F0A30448
:10D180004E014E014E014E014E014E014E014E0127
:10D190004E014E014E014E014E014E014E014E0117
:10D1A0004E014E014E014E014E014E014E014E0107
:10D1B0004E014E014E018500B300EC002F014E01DF
:10D1C0006001D90173027A024E014E014E019202B2
:10D1D0004E014E019D024E01CD02540375038A0398
:10D1E00092030004E800160479044E014E014E013A
:10D1F0004E014E014E0166009D00CA00240124012B
:10D200004E0183019D004E018B0273027A028F0250
:10D2100094024E019D02C602E000D6026D037C031B
:10D22000C903F703E40008043F04691EA14240F269
:10D23000F480013204F1010A3B5554466DE702F1D6
:10D2400002087BE74FF0000988E7B369AB4A18335F
:10D2500052F823B0584600F07DFF0BF1FF3B04EB82
:10D26000000A6B1E544507D198F80030002B00F0DF
:10D27000328408F10102E0E7A34240F2CE801BF8BD
:10D28000012F3A550134EDE7B2699C4B03EB820361
:10D29000D3F87CB0584600F05DFF0BF1FF3B04EB88
:10D2A000000A6B1EA245DFD0A34240F2B6801BF8F5
:10D2B000012F3A550134F5E7904B326953F822B00B
:10D2C000584600F047FF0BF1FF3B04EB000A6B1ED2
:10D2D0005445C9D0A34240F2A0801BF8012F3A5513
:10D2E0000134F5E73369854A0C3352F823B05846C8
:10D2F00000F030FF0BF1FF3B04EB000A6B1EA24570
:10D30000B2D0A34240F289801BF8012F3A55013474
:10D31000F5E77A4BD3F8A0A0504600F01BFF9AF82F
:10D320000030002B00F06D8333465246291B38191C
:10D33000FFF7EAFE002870DD04EB000A94E76F4B6C
:10D34000D3F8E4A0E8E76D4BD3F89CA0E4E76B4B7F
:10D35000D3F898A0E0E7D6F814A069498A45ACBF95
:10D360004FF0000B4FF0010BBAF1000F0BDB642004
:10D370009AFBF0F0133083B1632801DD2B2B20D012
:10D38000604B61490BE00AF26C70039300F0EAFE17
:10D390006421039B90FBF1F0EDE75A4B5B49019050
:10D3A000B9F1020F2CBFCBEB0900CBF10200584AB8
:10D3B000009053488245B8BF13460A46291B3819C6
:10D3C00022E0544BDDE7544A5449F368642818BFFF
:10D3D0000A46291B381902F0E9F817E07069336929
:10D3E000002803F1010A07EB040BF368A5EB04091D
:10D3F00019DB642290FBF2FC02FB1C00CDE900303B
:10D40000494653465846464A02F0D0F8002804DB05
:10D4100000EB040A55453FF627AF4FF0000A50468F
:10D420000FB0BDE8F08F00F26C70039300F09AFE2D
:10D43000642290FBF2FC039B0CFB1200DEE725212B
:10D440000DF11A0A8DF818105BB1B9F1050F8DF8BE
:10D45000193013D85046334900F058FE334606AA17
:10D4600064E72B238DF8193004231E2150462E4AE1
:10D4700002F09CF80028EDDD5044ECE7B9F106031A
:10D48000E8D0F2E73046FFF7EDFD73698246002BE6
:10D4900016DB642293FBF2F1B0F1FF3F02FB113384
:10D4A00040F020830AEB0300642390FBF3F203FBBC
:10D4B00012021A44B2FBF3F103FB1123164A88E768
:10D4C00003F26C7000F04EFE642390FBF3F2BAF1AD
:10D4D000FF3F02FB130306D17169144A9142E1DA5E
:10D4E0004FF0010ADEE7BAF1010F40F0FE827169E8
:10D4F000034A9142F4DA4FF0FF3AD3E7245301088C
:10D5000094F8FFFFEB2001082D4E0108264E01087C
:10D5100041510108354E0108414E01086D340108A2
:10D52000374E01084A4E0108464E010895F8FFFFA4
:10D53000BE490593736930468B42ACBF002101217F
:10D5400003930491FFF78EFD039B8246002BDDE9D8
:10D55000041347DB4FF0640B039A92FBFBFB0BF1C8
:10D56000130B706900284BDB4FF0640C90FBFCFE42
:10D570000CFB1E00BAF1FF3F51D1AD4AD6F814C0E2
:10D58000944502DA4FF0010A51468244BAF1FF3F56
:10D5900055D14FF0630A0BF1FF3B642000FB0BAA4F
:10D5A000002954D12B2B54D142F20F70824550D90F
:10D5B00019468DF8181001210DF1190CB9F1000F61
:10D5C00001D0A9EB010925218CF80010002B43D1D3
:10D5D0000CF10100974900F099FD4B46CDF800A0F1
:10D5E00006AA9DE0CDE90431039B03F26C7000F0C4
:10D5F000B9FDDDE904314FF0640C90FBFCFBB0E7B2
:10D6000000F26C70CDE9043100F0ACFDDDE90431CD
:10D610004FF0640C90FBFCFE0EFB1C00AAE7BAF175
:10D62000010F05D18149039A8A4204DB0021ACE74E
:10D630004FF0000AA9E751464FF0FF3AA5E7BAF1CB
:10D64000640F04BF4FF0000A0BF1010BA5E72D2179
:10D65000AFE70DF1180CB1E730230CF102008CF8A4
:10D660000130B7E7744A7549B3686B2818BF0A469A
:10D67000AFE6B36863B10C2B04D00C2193FBF1F23D
:10D6800001FB12336D4A6C49492818BF0A46A0E6CF
:10D690000C23F7E7F3696A4A01339AE633690133E9
:10D6A0000CE773680AE76B1E9C42BFF4B6AE0A2310
:10D6B00004F1010A3B55D7E5B3680B2BD4BF002218
:10D6C0000122604B03EB8203D3F8A4B0584600F06C
:10D6D00041FD04EB000A5C480BF1FF3B691EA245CB
:10D6E0003FF4C2ADA1427FF698AE98F800201BF837
:10D6F000013F502A06D1C25C02F00302012A08BF92
:10D700002033DBB23B550134E9E70322336993FB55
:10D71000F2F34E4A01335CE673684D4A0093B368F6
:10D72000291B381901F042FF70E6336A002B77DBC2
:10D7300000F0A0FA029B0BB900F0A8FA02F02EFE4E
:10D74000336A002BD4BF00220122282302FB0333BB
:10D75000C358C3F1000A00F093FA012302937269DF
:10D76000291BB2F145034FEAE27C6CF1000CBCF1DD
:10D77000000F07EB040002DA03334CF1000C4FF00A
:10D78000640B02F1FF3E9EFBFBFE4FF4C87B9B083F
:10D7900043EA8C73B3EB0E034FEAAC0C6CEBEE7CFC
:10D7A00002F22B1E9EFBFBFE13EB0E034CEBEE7CFA
:10D7B00040F26D1E463A0EFB02F24FF0180E9B1817
:10D7C0004CEBE27CF2699B184CEBE27CA3FB0E2352
:10D7D0000EFB0C33D6F808C012EB0C0243EBEC73D3
:10D7E0004FF03C0CA2FB0C2E0CFB03E3D6F804E03C
:10D7F00012EB0E0243EBEE73A2FB0CE20CFB0322D6
:10D80000D6F800C01EEB0C0342EBEC72B3EB0A033C
:10D8100062EBEA72CDE900320E4A01F0C7FEF5E58F
:10D820004FF0000A9BE7336848E600BF94F8FFFF1B
:10D8300095F8FFFF524E01086D340108414E010872
:10D84000564E010824530108215401085B4E01087B
:10D850006A4E0108604E01086B1E9C42BFF4DDADAC
:10D86000092304F1010A25E73368A14A019373688B
:10D870000093B368A2E56B1E9C42BFF4CEADB369C2
:10D8800004F1010A3C4413B937232370ECE430332C
:10D89000FBE7F369B26907339B1A072293FBF2F3A4
:10D8A0000CE63046FFF7DEFBB269034662B1013A8F
:10D8B000012B3FF403AE0133F16907D007230A318E
:10D8C000891A91FBF3F3F9E50622F1E7531A72691D
:10D8D00040F26B71002AA8BF6FF064010A449107FF
:10D8E00005D1642092FBF0F100FB112171B94FF4D6
:10D8F000C87192FBF1F001FB1022B2FA82F25209D8
:10D900009A1A042ACCBF34233523D7E50122F7E73E
:10D910000DF1180B77495846039300F0F7FB584672
:10D9200000F018FC039B0BEB000A0AF1010A73B12B
:10D93000B9F1050F0BF8003002D9B9F106030AD18D
:10D9400050466D4900F0E2FB33465A46EEE42B2385
:10D950000BF8003004230EA95046A1EB0A01674AD8
:10D9600001F024FE0028C8BF8244E9E76B1E9C42F8
:10D97000BFF453AD337E04F1010A30339AE6B26945
:10D980001AB1013AF369073386E70622FAE77069AC
:10D99000002805DB642390FBF3F202FB13038DE503
:10D9A00000F26C7000F0DEFBF4E7716954488142CC
:10D9B00012DA4FF02D0CA0EB010A8DF818C00120EF
:10D9C0000DF11901B9F1000F01D0A9EB00092520D3
:10D9D00008707BB9481CFDE52B2B01F26C7A06D14F
:10D9E00042F20F718A4502D98DF81830E7E700201E
:10D9F00006A9E7E73023881C4B70EBE5336A002B60
:10DA000001DAA24630E400F035F9029B0BB900F0D0
:10DA10003DF902F0C3FC336A002BD4BF002201227F
:10DA2000282302FB0333C358C3F1000900F028F98F
:10DA30003C2399FBF3F001F067FA3C2390FBF3F2EF
:10DA400002FB13004FF46163009099FBF3F32D4A3E
:10DA5000291B381901F0AAFD0028FFF6DEAC00EB07
:10DA6000040A55457FF6D9AC01230293FFF7FCBBAE
:10DA7000336A002BC5DB00F0FDF8029B0BB900F008
:10DA800005F9336A204A002BD4BF0023012352F842
:10DA90002390A246484600F05DFB09F1FF3920447F
:10DAA0006B1E824502D100F0EBF8DDE79A4506D205
:10DAB00019F8012F07F80A200AF1010AF1E700F02E
:10DAC000DFF8AAE46B1E9C42BFF4A7AC252304F147
:10DAD000010AEFE5A246002D3FF4A1AC002307F8B0
:10DAE0000A309CE401283FF4FBAC4FF0000AD9E473
:10DAF000654E0108744E0108C94F0108464E0108E1
:10DB000094F8FFFF7C4E0108940B0020FFF7FCBA4D
:10DB10002DE9F041044602F041FC40F2B1739C4211
:10DB200040F3A1806FF4F662A61840F26D12A4F2E1
:10DB3000B273B61002FB03666FF06302A4F26D735A
:10DB400093FBF2F36FF4C8614FF4C8721E4463187C
:10DB5000B3FBF2F30546454A44601E4400F150070A
:10DB60002B7A4A2B3AD1696914F0030F01EB0603B3
:10DB700008D14FF0640E94FBFEFC0EFB1C4CBCF174
:10DB8000000F08D14FF4C87E94FBFEFC0EFB1C4C2A
:10DB9000BCF1000F20D13B29D4BF002101210B444F
:10DBA000013BA9694FEAE17CC3FB021CAB6AC918BF
:10DBB0004CEBE373C5E908132835AF42D0D1D0E967
:10DBC0000843D0E912128C429341B4BF01230023D1
:10DBD00003600120BDE8F0810021E0E7442B02D181
:10DBE0006B693344DDE7A30705D1642194FBF1F3AE
:10DBF00001FB13438BBB4FF4C87194FBF1F301FBA2
:10DC00001343B3FA83F35B0959424FF0000E3346D6
:10DC1000DFF85CC001F03001D5F80C8061440EF1F2
:10DC2000010EF04551F82EC019DC072103F1040E56
:10DC30009EFBF1F1C1EBC101AEEB010E6969B1EBE5
:10DC40000E0E296948BF0EF1070E0139C1EBC10163
:10DC50007144614505DA0B44A3E70123D4E763442B
:10DC6000DDE70739F5E70020B4E700BF8051010088
:10DC7000C0520108014800F010B800BFEC150020A8
:10DC8000014800F00CB800BFEC150020014B1868EB
:10DC900000F008B89C0B0020704770477047704731
:10DCA000704700002DE9F04F8DB0074602F076FB7B
:10DCB000BC490446384601F021F9BB4D06462968A7
:10DCC00010BBBA4BBA4A1860BA4BC4E90366186075
:10DCD000B94B4A20C3E9002200220023207284F8B5
:10DCE0003000C4E905660846C4E90823C4E90D66A6
:10DCF000C4E90F66C4E91223A662266501F068FA3A
:10DD00002E600DB0BDE8F08F002940F08F802868AC
:10DD100001F05EFA304600F01DFA411C384601F071
:10DD200081FA2860002840F087800023A14A002063
:10DD300013600021A14AA04FC4E90333C7E90022C0
:10DD40004A22C4E90533C4E90801C4E90D33C4E932
:10DD50000F33C4E91201DFF854A22272CAF800306E
:10DD6000A36284F83020236533780DF1280B3A2B19
:10DD700008BF013633783C2B62D1751C5B462846C0
:10DD80008F4A904901F0DCFF0028BADD0A9BDA1EB9
:10DD9000072AB6D8EA5C3E2AB3D10236F518F35CFE
:10DDA0002D2B5BD14FF0FF38013500230DF12009F9
:10DDB000ADF81E30ADF820300DF11E03009328465B
:10DDC0005B46CDE901B98049CDF80CB007AA01F056
:10DDD000B7FF002895DD3C22BDF81E30BDF820605D
:10DDE00002FB03664FF46162BDF81C3002FB036660
:10DDF0000A9B08FB06F605EB0308EB5C3C2B40F0A6
:10DE0000ED8008F101055B462846704A6D4901F036
:10DE100097FF002828DC98F801303E2B24D1684B6E
:10DE2000A662C7E90033CAF800606AE700F064F947
:10DE300000287FF46CAF64E7314600F067F974E7BF
:10DE40005B4630465E4A624901F07AFF00287FF760
:10DE500058AF0A9BDA1E072AA0D952E72B2B4FF0A6
:10DE6000010808BF0135A0E70A9BDA1E072A3FF622
:10DE700048AFEA5C3E2A7FF444AF08F1020808EBA1
:10DE8000030518F803302D2B40F0B7804FF0FF3812
:10DE900001350023ADF81C30ADF81E30ADF8203050
:10DEA0000A930DF11E03009328465B46CDE9029BC1
:10DEB0004549CDF804B007AA01F042FF002800F35D
:10DEC000A280A6F56163A0464FF0000B04930A9B65
:10DED0001D442B782C2B08BF013595F80090B9F123
:10DEE0004D0F40F0A0800AAB0DF12602CDE90132C2
:10DEF00009AA00922846374903930DF1220201F046
:10DF00001FFF03287FF4FDAEBDF822104B1E0B2B24
:10DF10003FF6F7AEBDF82420531E042B3FF6F1AEBA
:10DF2000BDF82630062B3FF6ECAEC8E9031288F8A0
:10DF30000890C8F814300A9B05EB030900254FF040
:10DF40000203ADF81E50ADF81C30ADF820500A9514
:10DF500099F800302F2B40F094800AAB08AACDE945
:10DF600001320DF11E02009248461B49039307AA95
:10DF700001F0E6FEA84200F384804A21002200233B
:10DF8000C4E90355C4E90555C4E90823C4E90D559E
:10DF9000C4E90F55C4E912232172A56284F8301038
:10DFA0002565AEE6884E0108F01500200C1600200D
:10DFB0008B4E010810160020940B0020EB20010866
:10DFC000001600208F4E0108C44E0108F4150020F1
:10DFD000A24E0108B04E0108C34E01085B46404600
:10DFE0003F4A404901F0ACFE00287FF718AF0A9B7A
:10DFF000DA1E072A7FF643AF83E62B2B4FF001088A
:10E0000008BF013545E73C21BDF81E20BDF8203092
:10E0100001FB02334FF46161BDF81C2001FB0233A8
:10E0200008FB03F34FE7B9F14A0F0ABF4B464423FD
:10E0300001350A2228460BA9059302F085F8DDF880
:10E040002C90059BA945ADF8260014D14D23BBF1BA
:10E05000000F07D1032123720223C4F814B0C4E9CE
:10E0600003136BE70B2284F830300123C4E90D233E
:10E070000023E36362E780B288F80830C8F8140030
:10E080005CE73C21BDF81E20BDF8203008F12808CF
:10E0900001FB02334FF46161BDF81C2001FB023328
:10E0A00048F8103C0A9D0BF10103022B4FF0010BC5
:10E0B0004D447FF40EAF049B606823650A4BA66253
:10E0C0003B60074B7B60FFF723FDA26A236DCAF814
:10E0D00000209B1A18BF0123044A136011E600BFF9
:10E0E000F4150020A24E0108001600201016002092
:10E0F00000487047380D002010F8012B11F8013B43
:10E10000012A28BF9A42F7D0D01A7047034611F867
:10E11000012B03F8012B002AF9D17047034610B5F3
:10E12000C9B20244934201D1002004E018460478A9
:10E1300001338C42F6D110BD0A44914200F1FF3305
:10E1400000D1704710B511F8014B914203F8014F0F
:10E15000F9D110BD034613F8012B002AFBD1181A80
:10E16000013870470028B8BF404270471FB51D46B0
:10E17000094B06461B68D86852B1084C3346CDE9B6
:10E18000014200912A46064901F0F0FE02F0E4F94E
:10E19000044C2246F2E700BF9C0B0020F84F010818
:10E1A00005500108EB20010891FBF2F302FB13116B
:10E1B0000360416070472DE9F74F03690C698046A1
:10E1C000A3427EDB013CA30000F1140501F114071A
:10E1D000009305EB8403019357F8243055F824206D
:10E1E00001339A42B2FBF3F607EB84092ED34FF0CA
:10E1F000000ABC46AE46D3465CF8043B98B206FB28
:10E2000000A01B0C020C06FB0323DEF8002080B2EA
:10E2100092B2121A5A44DEF800004FEA134A9BB237
:10E22000C3EB224303EB104392B242EA0342E145BF
:10E230004FEA234B4EF8042BDED2009BEB582BB950
:10E24000019B1A1F954230D3C8F81040404601F098
:10E250006BFC002825DB29460020013657F8042BEB
:10E26000D1F800C01FFA82FE1FFA8CF3A3EB0E0355
:10E270000344120CC2EB234202EB1C429BB243EA62
:10E280000243B9454FEA224041F8043BE6D255F833
:10E29000242005EB840322B9043B9D420BD3C8F82C
:10E2A0001040304603B0BDE8F08F1368002BCBD18F
:10E2B000043A013CC6E71A68002AF0D1043B013C4D
:10E2C000EBE70020EEE700002DE9F04F16461F4671
:10E2D000C26999B08146CDE90E67259C82B91020AC
:10E2E00000F06EFF0246C9F81C0020B9EF21A24BD6
:10E2F000A248FFF73BFF0023C0E901330360C3607E
:10E30000116859B101235268484693404A608B60B6
:10E3100001F0BCF90022D9F81C301A60B7F10008EE
:10E32000B5BF0123002323602360954BBCBF28F0B9
:10E330000048CDF83C8033EA08031AD142F20F734B
:10E34000249AC8F3130858EA0608136000F06D8594
:10E35000269B53B98B4B21E08B4B03930833269AB2
:10E360001360039819B0BDE8F08F864B0393033315
:10E37000F5E7DDE90E34CDE90A34DDE90A010022D2
:10E38000002303F06FF9824650B10123249A1360F1
:10E39000269B13B17D4B269A13607D4B0393E0E7D8
:10E3A00016AB019317AB00934846DDE90A2301F051
:10E3B0006FFC5FEA1854169D04907CD0DDE90A01D9
:10E3C0000B9BA4F2FF34C3F3130343F07F5343F4D6
:10E3D0004013CDF850A0194600226E4B02F022FDEA
:10E3E0005FA3D3E9002302F0D5FE5FA3D3E90023A6
:10E3F00002F01AFD064620460F4602F061FE5CA3BD
:10E40000D3E9002302F0C6FE02460B4630463946E9
:10E4100002F00AFD06460F4603F06CF90022804622
:10E4200000233046394603F027F948B1404602F050
:10E4300047FE32463B4603F015F908B908F1FF38AC
:10E44000B8F1160F54D8DDE90A01534B03EBC803AA
:10E45000D3E9002303F010F900284BD0002308F182
:10E46000FF3811932D1B6B1E099349BF0023002712
:10E47000C5F101070993B8F1000F3DDB099BCDF809
:10E4800040804344099300230C93229B092B00F204
:10E490008780052BC4BF043B2293229BC8BF002466
:10E4A000A3F10203D8BF0124032B00F28580DFE82B
:10E4B00003F05153362B179C2C4404F23243202B8B
:10E4C000C1BFC3F1400308FA03F804F2124326FA6D
:10E4D00003F3D6BFC3F1200348EA030006FA03F0B2
:10E4E00002F0DEFD0122A1F1F873013C149272E703
:10E4F0000123B6E71190B5E7C8F100030C930023A0
:10E50000A7EB08071093C0E701230D93239B434417
:10E5100008930133012B0593B8BF012306E00123C3
:10E520000D93239B002B4ADD0893059300210422C1
:10E53000D9F81C0002F114059D4245D941604846B6
:10E5400001F066F80390002841D1024640F2AF1175
:10E55000124BCDE60023E3E70023D6E7AFF30080BC
:10E5600061436F63A787D23FB3C8608B288AC63FD9
:10E57000FB799F501344D33F4A4D01084150010895
:10E580000000F07F3D5001083450010814300108AC
:10E59000133001080000F83F58550108A250010847
:10E5A000012400230D9422934FF0FF33002208939F
:10E5B000059323921223B9E701230D93F4E7012376
:10E5C000089305932393B1E701315200B2E7D9F8DC
:10E5D0001C30039A1A60059B0E2B75D8002C73D043
:10E5E000B8F1000F40F3C4809F4B08F00F0203EB1B
:10E5F000C20318F4807F4FEA2815D3E900AB00F07E
:10E60000A380DDE90A01994B0324D3E9082302F032
:10E61000EBFECDE9060105F00F05944E002D40F00C
:10E620009980DDE9060152465B4602F0DDFE824636
:10E630008B46119B002B00F0C380002250465946A8
:10E640008B4B03F019F8002800F0BA80059B002BD3
:10E6500000F0B680089B002B36DD08F1FF335046F2
:10E66000594606930022834B02F094FD82468B4666
:10E67000089E0134204602F023FD52465B4602F01C
:10E6800089FD00227C4B02F0CFFB0446A1F15075BE
:10E69000CDE91245002E40F09780002250465946A1
:10E6A000764B02F0BFFB22462B4682468B4603F098
:10E6B00001F8002840F0C18222465046594605F133
:10E6C000004302F0D9FF20BB179B002BC0F29181C1
:10E6D000B8F10E0F00F38D81634B03EBC803D3E950
:10E6E00000AB239B002B80F21B81059B002B00F3CA
:10E6F00017810ED10022614B5046594602F04AFD67
:10E7000002460B46DDE90A0102F0C0FF002800F0D6
:10E71000978200252C46239B039EDB4306932746C6
:10E7200000242946484600F0B1FF002F00F0EE809B
:10E730002CB1BC4203D02146484600F0A7FF394621
:10E74000484600F0A3FFE1E0DDE90A34CDE90634F4
:10E75000022462E7E90708D5D6E900235046594666
:10E7600002F018FD82468B4601346D10083655E7DD
:10E7700022D0DDE90A01C8F100053B4B05F00F028C
:10E7800003EBC203D3E9002302F004FD0224824616
:10E790008B46364E2D11002D3FF44BAFEA0708D5BE
:10E7A000D6E900235046594602F0F4FC82468B46D7
:10E7B00001346D100836EEE70224DDE90AAB38E7D4
:10E7C000059ECDF8188055E7274B03EBC60353E9A8
:10E7D00002010D9B002B55D002460B460020284914
:10E7E00002F002FEDDE9122302F01CFB039BCDE9DF
:10E7F00012019D191E465946504602F07BFF00F15A
:10E80000300402F05DFC02460B465046594602F0C9
:10E8100009FBDDE9122306F8014B82468B4602F024
:10E820002BFF002872D152465B460020104902F0AF
:10E83000F9FADDE9122302F01FFF002840F0BA8048
:10E84000AE423FF441AFDDE912010022094B02F074
:10E85000A1FC0022CDE91201064B5046594602F0B8
:10E8600099FC82468B46C6E7585501083055010889
:10E870000000F03F0000244000001C400000144055
:10E880000000E03FDDE9122302F084FC039BCDE9A8
:10E8900012013344039C15935946504602F02AFF57
:10E8A00000F1300502F00CFC0B460246594650467A
:10E8B00002F0B8FA159B04F8015B9C4282468B4635
:10E8C00027D1DDE91201039B00221E44AC4B02F06C
:10E8D000ABFA02460B465046594602F0EBFE0028C2
:10E8E00068D1DDE912230020A54902F09BFA024617
:10E8F0000B465046594602F0BFFE00283FF4E4AEF6
:10E90000334616F8012D302AFAD01E46DDF818805D
:10E910003EE000229B4B02F03DFC82468B46BBE76B
:10E920000024039E974D5246DDE90A015B4602F042
:10E930005BFD02F0DFFE074602F0C2FB52465B467B
:10E9400002F028FC02460B46DDE90A0102F06AFAF1
:10E9500007F1300C06F801CBDDF80CC0DDF814E04F
:10E96000A6EB0C0CE64502460B4633D102F05CFAEE
:10E9700052465B4604460D4602F09CFEC0B9524624
:10E980005B462046294602F06DFE08B1FB070FD416
:10E990004846049900F07AFE0023249A337008F167
:10E9A00001031360269B002B3FF4DBAC1E60D8E410
:10E9B000CDF8188033461E4613F8012D392A06D1AA
:10E9C000039A9A42F7D1069A013206923022013216
:10E9D0001A709BE722462B4602F0DCFB02460B46F0
:10E9E000CDE90A230022002302F03CFE00289AD041
:10E9F000CEE70D9A002A00F0DF80229A012A00F368
:10EA0000C380149A002A00F0B78003F233430C9DB0
:10EA10003E46099A01211A4448461F44099200F0D3
:10EA2000E9FE044656B1099B002B07DDB342A8BF9F
:10EA30003346099AFF1AF61AD31A09930C9B0BB3A3
:10EA40000D9B002B00F0BF80002D00F0B980214607
:10EA50002A46484600F09AFF049A01460446484672
:10EA600000F0DEFE04998246484600F00FFE0C9B43
:10EA70005B1B0C9300F0AA8051460C9A484600F0AC
:10EA800085FF04900121484600F0B4FE109B054626
:10EA9000002B00F0D1811A460146484600F076FF6F
:10EAA000229B0546012B00F399800E9B002B40F022
:10EAB00090800F9BC3F31303002B40F08A800F9BC1
:10EAC00023F000431B0D1B05002B00F085804FF049
:10EAD000010A099B013701330993109B002B00F0B9
:10EAE000B1812B6905EB8303186900F037FEC0F193
:10EAF0002000099B184410F01F0076D01B2870DC02
:10EB0000C0F11C000744064403440993002F05DDAF
:10EB10003A464846049900F095FF0490099B002B63
:10EB200005DD29461A46484600F08CFF0546119B34
:10EB3000002B5FD02946049800F0F6FF002859DA30
:10EB400008F1FF3306930A2200234846049900F097
:10EB5000BFFD0D9B0490002B00F076810023214621
:10EB60000A22484600F0B4FD089B0446002B71DCE5
:10EB7000229B022B47DC6DE0169BC3F1360346E770
:10EB80000000E03F00002440059B5D1E0C9BAB4253
:10EB900008DB5D1B059B002BBFF63AAF059BFE1AF9
:10EBA000002336E70C9B109AEB1A1A440C953E464C
:10EBB0000025059B10922CE73E460C9D0D9C31E7ED
:10EBC000DDF810A058E70C9A049957E7CDF810A08B
:10EBD00058E74FF0000A80E79A467EE74FF0000AB8
:10EBE0007FE71C2892D0C0F120001C30099B07440D
:10EBF000064489E7059BCDF81880002B24DC089398
:10EC0000229B022B22DD089B002B7FF484AD29463A
:10EC10000522089B484600F05BFD01460546049826
:10EC200000F082FF00287FF776AD3123039E06F8BF
:10EC3000013B069B0133069371E535462C46F4E70C
:10EC4000059DCDF81880F9E7059B08930D9B002BD7
:10EC500000F0FE80002E05DD21463246484600F0D9
:10EC6000F1FE0446BAF1000F58D04846616800F042
:10EC7000CFFC064628B9024640F2EF217F4BFFF752
:10EC800037BB226904F10C01023292000C30FFF70D
:10EC900053FA01223146484600F0D4FE0746039B52
:10ECA000039A03F10108089B13440A930E9B03F097
:10ECB0000103099329460498FFF77DFA2146059040
:10ECC00000F1300B049800F02FFF3A4608902946D7
:10ECD000484600F045FFC268064608F1FF3AFAB917
:10ECE0000146049800F020FF0246314648460C9247
:10ECF00000F0CCFC229B0C9A464642EA0301099B99
:10ED000019430FD1BBF1390F28D0089B002B02DD2E
:10ED1000059B03F1310B8AF800B002E52746BEE7F8
:10ED20000122E2E7089B002B04DB22990B4309999F
:10ED30000B4320D1002AEEDD01220499484600F061
:10ED400081FE2946049000F0EFFE002803DCE2D1AA
:10ED50001BF0010FDFD0BBF1390FD9D139238AF86D
:10ED6000003033461E4616F8012C013B392A53D099
:10ED700001321A70D5E4002A07DDBBF1390FEDD05E
:10ED80000BF101038AF80030CBE40A9B08F801BCC0
:10ED900043452BD000230A220499484600F098FCF2
:10EDA000BC4204904FF000034FF00A02214648464F
:10EDB00006D100F08DFC0446074608F1010879E70A
:10EDC00000F086FC3946044600230A22484600F03B
:10EDD0007FFC0746F1E7089B2746002B03F1FF362F
:10EDE000D8BF00260024039B5A1C16440122049914
:10EDF000484600F027FE2946049000F095FE0028C2
:10EE0000AFDC02D11BF0010FABD133461E4613F825
:10EE1000012D302AFAD084E4039A9A42A2D1069BAB
:10EE200001330693312313707BE4269B002B7FF480
:10EE300093AA134BFFF7B2BA229B012B7FF735AE93
:10EE4000DDF840A0012054E6089B002B7FF7D8AEE8
:10EE5000039E29460498FFF7AEF9039B00F1300B9F
:10EE600006F801BBF21A089B9342B4DD00230A2284
:10EE70004846049900F02CFC0490EAE7A2500108EF
:10EE8000345001082DE9F84FDFF86CA0064689469A
:10EE9000174601F07DFBDAF8004034B14A4613789A
:10EEA0004BB13D2B02F10102F9D1304601F076FB66
:10EEB0000020BDE8F88FA2EB09082068A3460028CF
:10EEC000F3D042464946043401F012FA0028F4D146
:10EED00054F8043C03EB080513F808303D2BECD143
:10EEE000DAF800303046ABEB03039B103B6001F0D7
:10EEF00055FB681CDDE700BFB40D002007B501AA73
:10EF0000FFF7C0FF03B000BD0028B8BF4042704704
:10EF10002DE9F0471F468E688246BE420C46904659
:10EF2000334653D8B1F90C0010F4906F2BD06569BB
:10EF30002368096905EB4505A3EB010905EBD575C8
:10EF40007B1C6D104B44AB422A4684BF1D462A46AB
:10EF5000430527D51146504600F064F9064658B3DC
:10EF60004A462169FFF7E8F8A38923F4906343F048
:10EF70008003A38126614E4426603B463E46656180
:10EF8000A5EB0905A5601F463A464146206801F0F9
:10EF900096F90020A3689B1BA36023683B44236071
:10EFA000BDE8F087504600F0F3FF06460028E1D1A7
:10EFB0005046216901F0F8FA0C23CAF80030A38901
:10EFC0004FF0FF3043F04003A381E9E73E46DBE723
:10EFD0002DE9F0471F468B8906461B060D46144651
:10EFE0009CB010D50B6973B9402100F01BF9286063
:10EFF000286130B90C2333604FF0FF301CB0BDE8FE
:10F00000F08740236B610023099320238DF829307A
:10F0100030234FF001080397644F8DF82A302346C0
:10F020001A7899461AB1252A03F10103F8D1B9EBF0
:10F03000040A0BD05346224629463046FFF768FFA4
:10F04000013000F0A380099A5244099299F80030E7
:10F05000002B00F09B8000224FF0FF33CDE90532FA
:10F0600009F10109049207928DF853201A924C4637
:10F07000052214F8011B4D48FFF750F8049AD0B947
:10F08000D00644BF20238DF85330110744BF2B23F3
:10F090008DF8533099F800302A2B13D04B460020BE
:10F0A0004FF00A0C07991A781C46303A092A4AD9B7
:10F0B000A8B1079113E0C01B08FA00F01043A14665
:10F0C0000490D4E7039B191D1B680391002BBBBF61
:10F0D0005B4242F0020207930793B8BF0492237881
:10F0E0002E2B0AD163782A2B32D1039B02341A1DAE
:10F0F0001B68039243EAE3730593DFF8B49003229D
:10F1000048462178FFF70AF838B14022049BA0EB6B
:10F1100009008240134301340493217806222548D4
:10F120008DF82810FEF7FAFF002835D0224818BBCA
:10F13000039B073323F0070308330393099B013430
:10F14000034409936BE701200CFB01210133AAE77B
:10F1500000234FF00A0C18460593611C0A780C46F0
:10F16000303A092A03D9002BC7D00590C5E70123FF
:10F170000CFB00200131F1E703AB00932A46304637
:10F180000E4B04A9FCF7B6FD421CD7D1AB895B0638
:10F190003FF532AF099831E703AB00932A4630467A
:10F1A000064B04A9FDF746F8EEE700BFB35001088F
:10F1B000B9500108BD500108F5BC000811EF000866
:10F1C000024B0146186800F02DB800BF9C0B0020D0
:10F1D000024B0146186801F0E7B900BF9C0B002004
:10F1E00070B50F4C0E462168054611B901F0C6F8FE
:10F1F00020603146284601F0C1F8431C03D14FF08E
:10F20000FF34204670BDC41C24F00304A042F8D093
:10F21000211A284601F0B2F80130F2D1EFE700BF21
:10F22000141600202DE9F843CD1C25F00305083500
:10F230000C2D38BF0C25002D064601DBA94204D950
:10F240000C2333600020BDE8F883334F00F0A2F9AF
:10F250003B681C463CBB29463046FFF7C1FF431CB8
:10F26000044656D13C68A046B8F1000F40D1002CAE
:10F2700049D023684146304604EB030901F07EF88B
:10F28000814540D1216830466D1A2946FFF7A8FF15
:10F29000013038D023682B4423603B685A685ABB3E
:10F2A000C7F800800EE02268521B1ED40B2A16D924
:10F2B0006119A342256018BF5960636808BF3960AF
:10F2C00062514B60304600F06BF904F10B00231DD6
:10F2D00020F00700C21A1CBF1B1AA350B3E76268D4
:10F2E000A3420CBF3A605A60ECE723466468B1E77A
:10F2F0004446D8F80480B7E71A465B68A342FBD1BE
:10F3000000235360DEE70C233046336000F048F9F9
:10F3100098E70560D6E700BF18160020936810B480
:10F32000013B002B936007DA9469A34201DB0A29B1
:10F3300002D110BC00F05ABE1368581C106019703E
:10F34000084610BC7047F8B506460F461446D51857
:10F35000AC4201D1002007E03A46304614F8011BC8
:10F36000FFF7DCFF431CF3D1F8BD00002DE9F047A7
:10F3700006460D4614461F469CB018B1036A0BB9E9
:10F38000FDF732F96B6ED90705D4AB899A0502D423
:10F39000A86DFEF783FCAB891B0701D52B699BB9D0
:10F3A0002946304600F0DAFE70B16B6EDE0704D5F8
:10F3B0004FF0FF301CB0BDE8F087AB899C05F7D457
:10F3C000A86DFEF76DFCF3E70023099320238DF869
:10F3D000293030234FF001080397694F8DF82A3008
:10F3E00023461A7899461AB1252A03F10103F8D168
:10F3F000B9EB040A0BD05346224629463046FFF7A4
:10F40000A2FF013000F0A380099A5244099299F8B2
:10F410000030002B00F09B8000224FF0FF33CDE93D
:10F42000053209F10109049207928DF853201A92CE
:10F430004C46052214F8011B5148FEF76FFE049A52
:10F44000D0B9D00644BF20238DF85330110744BFF4
:10F450002B238DF8533099F800302A2B13D04B46CC
:10F4600000204FF00A0C07991A781C46303A092AF6
:10F470004AD9A8B1079113E0C01B08FA00F0104365
:10F48000A1460490D4E7039B191D1B680391002B30
:10F49000BBBF5B4242F0020207930793B8BF0492DE
:10F4A00023782E2B0AD163782A2B32D1039B023486
:10F4B0001A1D1B68039243EAE3730593DFF8C490B7
:10F4C000032248462178FEF729FE38B14022049BEA
:10F4D000A0EB0900824013430134049321780622F3
:10F4E00029488DF82810FEF719FE00283ED027483D
:10F4F00018BB039B073323F0070308330393099BCF
:10F500000134034409936BE701200CFB0121013313
:10F51000AAE700234FF00A0C18460593611C0A78ED
:10F520000C46303A092A03D9002BC7D00590C5E70D
:10F5300001230CFB00200131F1E703AB00932A46C5
:10F540003046134B04A9FCF7D5FB431CD7D16B6E97
:10F55000D90705D4AB899A0502D4A86DFEF7A0FBA4
:10F56000AB895B063FF524AF099823E703AB009313
:10F570002A463046064B04A9FCF75CFEE5E700BFCF
:10F58000B3500108B9500108BD500108F5BC00088E
:10F5900047F300080148FEF781BB00BFEE150020CD
:10F5A0000148FEF77DBB00BFEE1500200CB430B55E
:10F5B000154B0C1E1D689DB008DA8B234FF0FF30F1
:10F5C0002B601DB0BDE8304002B070474FF0000323
:10F5D0001B9318BF0123E31A049307930B4B02906C
:10F5E00006900593284621AB209A02A90193FFF7C4
:10F5F000EFFC431CBCBF8B232B60002CE1D000220E
:10F60000029B1A70DDE700BF9C0B00200802FFFF81
:10F6100070B5C46905460E4684B91020FFF7D0FDC9
:10F620000446E86128B902466B21164B1648FEF7DE
:10F630009DFD0023C0E901330360C360E36853B953
:10F6400021220421284600F08EFFEB69E060DB6890
:10F650000BB9002070BD53F8260030B1026843F8A2
:10F6600026200023C0E90333F4E7012101FA06F460
:10F67000621D2846920000F076FF0028E9D0C0E91C
:10F680000164EEE74A4D0108C450010870B5C46931
:10F6900006460D4674B91020FFF792FD0246F06150
:10F6A00020B98F21084B0948FEF760FDC0E90144ED
:10F6B0000460C4603DB1F3696A68DB6853F82210E6
:10F6C000296043F8225070BD4A4D0108C45001081A
:10F6D0002DE9F04107460C461E4600200D6901F158
:10F6E000140CDCF80030013099B202FB01611E0CF1
:10F6F0000B0C02FB063389B201EB034185424FEA52
:10F7000013464CF8041BECDC0EB3A368AB4219DCC7
:10F71000616838460131FFF77BFF804628B9024611
:10F72000BA210C4B0C48FEF721FD226904F10C01B3
:10F73000023292000C30FEF7FFFC21463846FFF7FC
:10F74000A5FF444604EB850301355E612561204633
:10F75000BDE8F081A2500108C45001080346B0F58D
:10F76000803F3ABF030410200020B3F1807F3CBFEC
:10F770001B020830B3F1805F3CBF1B010430B3F1C2
:10F78000804F3CBF9B000230002B04DB5B0001D5A7
:10F7900001307047202070470368014613F00702CC
:10F7A0000BD0DA0722D4980749BF5B089B080120D9
:10F7B0000B605CBF02200B60704798B2A0B91020AC
:10F7C0001B0CDAB20AB908301B0A1A0704BF1B095E
:10F7D00004309A0704BF9B080230DA0702D45B08A2
:10F7E00006D001300B6070471046EAE700207047F2
:10F7F0002020704710B50C460121FFF709FF024693
:10F8000028B940F24511044B0448FEF7AFFC012330
:10F810004461036110BD00BFA2500108C45001083B
:10F820002DE9F04FD1F81080D2F810900E46C8455F
:10F83000144685B004DB4B460C46C1461646984636
:10F84000A368616809EB0807BB42B8BF0131FFF745
:10F85000DFFE30B902464FF4B1714A4B4A48FEF719
:10F8600085FC00F114052B46002205EB870B5B4558
:10F8700022D306F1140101EB880304F1140C0CEB04
:10F88000890C029304F1150363458CBF0023012307
:10F890000093ACEB0403153B9B080193029B03917F
:10F8A0008B420CD8002F03DD5BF8043D002B67D0A2
:10F8B000076105B0BDE8F08F43F8042BD7E7B1F836
:10F8C00000A0BAF1000F28D0A9464FF0000E04F1B5
:10F8D000140858F8042BD9F8003096B29BB20AFBF2
:10F8E0000633D9F80060120C360C0AFB026673442A
:10F8F00006EB13469BB243EA0643C4454FEA164E55
:10F9000049F8043BE5D8009A019B002A4FEA83039B
:10F9100008BF00232B44C3F804E0039B0431B3F871
:10F9200002E0BEF1000F29D02B68A94698464FF09F
:10F93000000A04F1140632889BB20EFB02A202EB0D
:10F94000184243EA024349F8043B56F8043BD9F80D
:10F9500000804FEA134A1FFA88F30EFB0A33B445BE
:10F9600003EB12434FEA134AE5D8009E019A002E9A
:10F970004FEA820208BF00222A44536004358DE713
:10F98000013F8FE7A2500108C45001082DE9F84358
:10F99000174612F0030280460D4607D0264C013A66
:10F9A000002354F82220FFF793FE0546BF103FD0F6
:10F9B000D8F81C4094B91020FFF702FC0446C8F8A0
:10F9C0001C0030B9024640F2B3111C4B1C48FEF734
:10F9D000CDFB0023C0E901330360C360A66846B9CC
:10F9E00040F271214046FFF705FF00230646A06064
:10F9F00003602C464FF0000907F001037F1053B15C
:10FA0000294632464046FFF70BFF21460546404651
:10FA1000FFF73CFE67B1306838B9324631464046A0
:10FA2000FFF7FEFE3060C0F8009006462C46E3E784
:10FA30002846BDE8F88300BF245501084A4D010857
:10FA4000C45001082DE9F84F0C4607469146266937
:10FA5000496806EB6216A3684FEA621A06F10108CC
:10FA600043450BDB3846FFF7D3FD054648B9024650
:10FA70004FF4EF712A4B2B48FEF778FB01315B0006
:10FA8000EEE7002300F114010A461846534539DB1E
:10FA900020692AEAEA7A01EB8A0104F1140319F0D9
:10FAA0001F098C4603EB800030D04FF0000EC9F1E7
:10FAB000200AE3461A680CF1040C02FA09F242EA41
:10FAC0000E02CBF8002053F8042B984222FA0AFECB
:10FAD000EFD8031B153B23F0030304F115029042FA
:10FAE00038BF00231944C1F804E0BEF1000F00D173
:10FAF000B04638462146C5F81080FFF7C7FD2846B6
:10FB0000BDE8F88F42F8040B0133BFE753F8041B3C
:10FB10000CF1040C98424CF8041CF7D8E8E700BF3D
:10FB2000A2500108C450010803690A6930B59B1A44
:10FB30000ED11430143100EB820401EB820154F831
:10FB4000045D51F8042D954204D006D24FF0FF33E6
:10FB5000184630BDA042F2D3FAE70123F8E70000CF
:10FB60002DE9F74F8A460646114650461446FFF7E0
:10FB7000DBFF051E12D129463046FFF749FD02463C
:10FB800028B940F23721404B4048FEF7EFFA0123F5
:10FB9000C0E90435104603B0BDE8F08FBCBF534642
:10FBA000A2463046DAF80410BABF1C4601250025EB
:10FBB000FFF72EFD024618B940F24521324BE3E72C
:10FBC000C56000F11405AB464FF0000CDAF8107078
:10FBD00026690AF1140904F1140E0AF1100309EB65
:10FBE00087080EEB86060193019B5EF8040B53F821
:10FBF00004AF81B201931FFA8AF35B1A000C6344CD
:10FC0000C0EB1A4000EB23409BB243EA0043764529
:10FC10004FEA204C4BF8043BE6D8331B153B153418
:10FC200023F00303A64238BF0023E8184B441C1DF1
:10FC300026460430A5EB090546450ED308F103011D
:10FC4000091B21F003010133984538BF002101440D
:10FC500051F8043DB3B117619CE7E24606EB050E8F
:10FC600056F8041B1FFA81FCD4444FEA1149514451
:10FC700009EB2C4989B241EA09414FEA294CCEF8F7
:10FC80000010D9E7013FE3E7A2500108C450010882
:10FC90002DE97343012190469946089EFFF7B8FC71
:10FCA000054630B9024640F20F31234B2348FEF798
:10FCB0005DFAC9F30A54C9F313030CB143F480137A
:10FCC0000193B8F1000324D068460093FFF764FD68
:10FCD0000099E0B1019AC0F1200302FA03F30B434B
:10FCE000C2406B610192019B002B0CBF01220222DA
:10FCF000AB612A61ACB1A4F2334404443460C0F176
:10FD00003500099B1860284602B0BDE87083696120
:10FD1000E9E701A8FFF740FD019B01226B6120305C
:10FD2000E7E7A0F2324005EB820330601869FFF785
:10FD300015FDC0EB4210E4E7A2500108C4500108D1
:10FD40000EB44FF4017370B500259DB021AC54F88A
:10FD5000046BADF814301B9502900690FEF7FAF98B
:10FD60000B4B03900B934FF6FF7307900948ADF8C8
:10FD700016303246234602A900680F951495019467
:10FD800000F0B6FC1DB0BDE8704003B0704700BF86
:10FD9000BBFD00089C0B002010B50C46B1F90E10FD
:10FDA00000F0DAFA0028ABBF636DA3891B1823F4B7
:10FDB0008053ACBF6365A38110BD002070472DE95F
:10FDC000F0411F468B890546DB050C46164605D5D6
:10FDD00002230022B1F90E1000F0ACFAA3893246DA
:10FDE00023F48053A38128463B46B4F90E10BDE8A6
:10FDF000F04100F07DBB10B50C46B1F90E1000F0DB
:10FE000099FAB4F90C30421C0BBF23F4805343F42D
:10FE10008053A381A38118BF606510BDB1F90E1096
:10FE200000F078BBB1F90C20F8B5160705460C4672
:10FE300051D44B68002B02DC0B6C002B49DDE66AC9
:10FE4000002E46D0002312F480522F682B6031D050
:10FE5000626DA389590705D56368D21A636B0BB12C
:10FE6000236CD21A00232846E66A216AB047421C56
:10FE7000B4F90C3006D129681D2944D8264ACA4055
:10FE8000D60740D5002262602269D904226004D5D9
:10FE9000421C01D12B6803B96065616B2F60C1B151
:10FEA00004F14403994202D0284600F07DFB002370
:10FEB00063630EE001232846216AB0470246501CC6
:10FEC000C7D12B68002BC4D01D2B01D0162B19D104
:10FED0002F6000201CE00F69002FFAD0930718BF95
:10FEE00000230E6808BF4B69F61B0F608B60002E65
:10FEF000EFDD33463A462846216AD4F828C0E04769
:10FF0000002806DCA3894FF0FF3043F04003A381B3
:10FF1000F8BD0744361AEAE70100402038B50B69FE
:10FF200005460C4613B91D46284638BD18B1036A6C
:10FF30000BB9FCF759FBB4F90C30002BF3D0626E0F
:10FF4000D00704D4990502D4A06DFDF7A7FE28467A
:10FF50002146FFF767FF636E0546DA07E4D4A389FD
:10FF60009B05E1D4A06DFDF79BFEDDE70EB403B564
:10FF7000014603AB054853F8042B00680193FFF7D3
:10FF8000F5F902B05DF804EB03B070479C0B00205C
:10FF90002DE9F041074615460C4621B91146BDE84A
:10FFA000F041FFF73FB92AB900F0FEFA2C4620468F
:10FFB000BDE8F08100F0A1FE8542064602D8B5EB0F
:10FFC000500FF4D829463846FFF72CF9804608B977
:10FFD0004446ECE7B5422A46214628BF3246FEF7A2
:10FFE000ABF82146384600F0DFFAF1E7F8B50546F0
:10FFF0000F46144618B1036A0BB9FCF7F5FAA3696A
:020000040801F1
:10000000A360A3891A0701D5236943B9214628466D
:1000100000F0A4F818B14FF0FF363046F8BD236960
:100020002068C01A6369834205DC21462846FFF731
:1000300075FF0028EFD1A3680130013BA36023685E
:10004000FEB25A1C22601F706369834204D0A389E8
:10005000DB07E2D50A2EE0D121462846FFF75EFFF6
:100060000028DAD0D7E700002DE9F04386460D4698
:10007000334E284615F8014B375D17F00807F8D1C5
:100080002D2C10D101272C78851C33F0100015D1B0
:10009000302C0DD1287800F0DF00582808D16C787A
:1000A000023510230AE02B2C04BF2C78851CECE7CA
:1000B000002BF6D1302C14BF0A2308234FF0FF3851
:1000C000B8FBF3F8002603FB08F930466FEA09098C
:1000D000A4F1300CBCF1090F10D86446A3421EDD18
:1000E000B6F1FF3F07D0804516D301D1A14513DB00
:1000F000012600FB034015F8014BE9E7A4F1410C90
:10010000BCF1190F01D8373CE8E7A4F1610CBCF150
:10011000190F04D8573CE1E74FF0FF36EBE7731CAB
:1001200006D122233046CEF8003032B9BDE8F08344
:1001300007B14042002AF9D006B1691E1160F5E707
:1001400021540108FFF790BF13460A4601460248B2
:100150000068FFF789BF00BF9C0B002038B5284B13
:10016000054618680C4618B1036A0BB9FCF73CFA4F
:10017000B4F90C30190720D4DA0607D409222A6012
:1001800043F040034FF0FF30A38131E0580711D511
:10019000616B41B104F14403994202D0284600F05A
:1001A00003FA002363630022A3896260226923F0BB
:1001B0002403226043F00803A38123694BB9A38978
:1001C00003F42073B3F5007F03D02146284600F0E6
:1001D0003DF8B4F90C3013F001020AD00022A260FD
:1001E00062695242A261226942B913F08000C7D10C
:1001F00038BD990758BF6269A260F4E70020F7E7AD
:100200009C0B002070B50E46B1F90E101446002963
:100210001D4696B00ADAB28912F0800213D14FF46B
:10022000806100202A60216016B070BD6A4600F02F
:1002300081F90028EFDB019A02F47042A2F5005325
:100240005A425A41EBE700224021EAE78B8973B515
:100250009E0705460C4607D504F14703236023613A
:100260000123636102B070BD01AB6A46FFF7CAFFAC
:10027000009E28463146FEF7D5FFB4F90C3038B958
:100280009A05EFD423F0030343F00203A381E3E7CD
:1002900043F08003A381019BC4E904062060002B86
:1002A000E0D02846B4F90E1000F034F80028D9D078
:1002B000A38923F0030343F00103A381D2E788421B
:1002C00010B501EB020402D98442234607D8431E2D
:1002D000A14207D011F8012B03F8012FF8E70244DF
:1002E000824200D110BD13F8011D02F8011DF7E78D
:1002F00010B56AB101398418027811F8013F9A42A9
:1003000004D10130A04201D0002AF5D1D01A10BD8D
:100310001046FCE738B50023054C05460846236027
:1003200001F07CFE431C02D1236803B12B6038BD71
:100330001C16002038B50546084611460022054C1B
:1003400022601A4601F07AFE431C02D1236803B1F1
:100350002B6038BD1C16002038B5054608461146EE
:100360000022054C22601A4601F070FE431C02D1A7
:10037000236803B12B6038BD1C16002038B500235C
:10038000054C05460846236001F068FE431C02D177
:10039000236803B12B6038BD1C160020004870474D
:1003A000F00B00202DE9F04100230C46D0E90001BC
:1003B0004B4A01F025FC4FF46161002ABCBF02F5F5
:1003C000A83202F5C072B2FBF1F301FB13224FF029
:1003D0003C01A360B2FBF1F301FB132222604FF05A
:1003E000070200F52F20ACBF00F66C2000F66B2052
:1003F0006360C31C93FBF2F2C2EBC2029B1A394941
:1004000054D50733A361A0F50E33A3F52C7393FBEA
:10041000F1F1354B48F6AC6203FB010040F2B453F6
:10042000B0FBF2F2B0FBF3F30244D21A2F4B642676
:10043000B0FBF3F3D21A40F26D13B2FBF3F2B2FB4E
:10044000F6F5284403FB12039920A3EB920303EB78
:1004500083070237B7FBF0FC4FF0050800FB0CF0F8
:100460000230B0FBF8F003F1010EAEEB000040F2F9
:10047000F95E77458CBF6FF00907022767444FF498
:10048000C87C0CFB0121012F98BF0131B3F5997F86
:1004900012D3A3F59973E3610023A1F26C71E060BC
:1004A000C4E9047120462362BDE8F0810028A361FD
:1004B000A9DB90FBF1F1ACE712F0030F02D106FBD0
:1004C00015255DB94FF4C875B2FBF5F605FB16228C
:1004D000B2FA82F252093B331344DCE70122FAE715
:1004E00080510100B13A02004FC5FDFFB03A020051
:1004F00038B50546084611460022054C22601A46CA
:10050000FBF71AFB431C02D1236803B12B6038BDF3
:100510001C16002038B50023054C0546084623600C
:1005200001F064FD431C02D1236803B12B6038BD88
:100530001C16002038B50023064C05460846114617
:10054000236001F05BFD431C02D1236803B12B60E3
:1005500038BD00BF1C160020062008B500F042FC84
:10056000012001F089FD70B5A1FB026535B9314666
:10057000FEF758FE044628B9204670BD0C2300241F
:100580000360F9E732462946FCF71CF9F4E700005E
:100590000148FDF783BB00BFED1500200148FDF7C2
:1005A0007FBB00BFED15002037B5002942D051F8C0
:1005B000043C0C1F002BB8BFE4180190FEF7EAFFC3
:1005C0001D4A0198136833B96360146003B0BDE835
:1005D0003040FEF7E5BFA34208D9256861198B4278
:1005E00001BF19685B6849192160EDE71A465B682D
:1005F0000BB1A342FAD911685518A5420BD1246852
:1006000021445418A3421160E0D11C685B680C447B
:1006100014605360DAE702D90C230360D6E725683B
:1006200061198B4201BF19685B68491921606360D9
:100630005460CBE703B030BD1816002038B54B1C12
:10064000144603D14FF0FF35284638BD9389CDB20B
:1006500023F020039381636B52688BB1A36B9342A9
:1006600008DD23685A1E226003F8015C63680133C9
:100670006360E9E7214600F048FB0028F1D0E1E79C
:100680002169236851B1994208D213F8011CA9428B
:1006900004D1013B013223606260D5E7C4E90F3227
:1006A00004F1440363630323A363234603F8465F13
:1006B00023600123DCE710B50C46496B69B104F1F6
:1006C0004403994201D0FFF76FFF0020236C606361
:1006D000636013B1E36B236010BD23694FF0FF30FB
:1006E000236000236360A38943F02003A381F3E721
:1006F0002DE9F04F0D460021ADF5237D80466F4674
:10070000CDE9441101A94691A449DFF894B2A09122
:10071000A4490093A19192F80090B9F1000F00F064
:1007200058811BF80930561C13F008031AD06B6867
:10073000002B10DD2B681A781BF80220120701D459
:100740003246E8E7459A0133013245926A682B60E8
:10075000013A6A60EBE729464046A19B984700288A
:10076000E8D0EDE7B9F1250F40F085804193439340
:1007700053782A2B04BF1023961C4FF00A0208BF9F
:100780004193B2461AF8011BA1F13003092B1CD981
:1007900003228548FDF7C2FC38B1834B5646C01A88
:1007A0000123419A83401343419316F8013B782B70
:1007B00006D8572B10D8252B5DD057D8002B75D0D5
:1007C000032347930A23429388E0439B564602FB48
:1007D000031130394391D4E7A3F15802202AEFD80E
:1007E00001A151F822F000BFBB080108C1070108B0
:1007F000C107010817090108C1070108C10701085D
:10080000C1070108C1070108C1070108C1070108A4
:10081000C10701082D09010813090108730801081F
:100820007308010873080108C1070108CD08010811
:10083000C1070108C1070108C1070108C107010874
:100840003D090108D5080108B3080108C1070108DE
:10085000C107010839090108C10701081309010886
:10086000C1070108C1070108BB080108453B022B6D
:10087000A6D8052331E06B68002B0DDD2B681A78B4
:100880004A4540F0A68001336A682B60459B013AD7
:1008900001336A60459353E729464046A19B984738
:1008A0000028EBD04498002840F08B804FF0FF30B8
:1008B0008BE0419A42F020024192419A42F4007248
:1008C000419210226E2B429206D801E000234293FF
:1008D000032302E008234293042347936B68002B11
:1008E0003ADD419B590605D42B681A781BF8022083
:1008F000120738D4479B022B47DC3B462A4640462A
:1009000041A900F07DF8012863D002287FF418AFD8
:10091000C8E70A22D6E7314601A800F0B5F9419BA5
:10092000064643F0400341930123D6E7419B43F041
:10093000400341930023D0E70223CEE74198C3064A
:100940003FF5FEAE3B68459A191D39601B68C40728
:100950004CBF1A801A60F3E629464046A19B98478F
:100960000028BED09EE7459A013245926A68013A56
:10097000002A6A6002DD01332B60B5E72946404654
:10098000A19B98470028AFD08CE7042B0EDC3B4698
:100990002A46404641A900F08DF8B4E73D0601081B
:1009A00021540108B7060108B95001080A4B002B71
:1009B0003FF4C6AE3B462A46404641A9AFF300800D
:1009C000A1E7AB895B063FF571AF0DF5237DBDE86F
:1009D000F08F4498F9E700BF0000000082B001B931
:1009E00001A942B14BB113780B601278101E18BFE9
:1009F000012002B070471046FBE76FF00100F8E7F6
:100A00002DE9F84315468A6880460C4632B98A6952
:100A1000002A14BF4FF0FF3201228A6000272268AB
:100A2000DFF88C90D1065FBF1A68111D1960166837
:100A3000A06988B1012807D12B681A7863699B5C8B
:100A400053B9002F32D023E0022821D12B681B7824
:100A500019F803301B071BD423680137DA065EBF81
:100A60002B681B7806F8013B6B68013B6B602B68B9
:100A700001332B60A368013BA3604BB16B68002B73
:100A8000D6DC29464046D4F8803198470028CFD09C
:100A9000236813F0100305D1E2680132E260A26915
:100AA00002B13370002023693B442361BDE8F88321
:100AB000215401082DE9F04F0C4699466E4B87B042
:100AC0008246164693E8070003AB83E807006B4BAA
:100AD000A1696B4A2746032908BF1A46A3680192F9
:100AE0005A1EB2F5AE7F81BF6FF4AE7503EB0508F9
:100AF00040F25D13A36057F81C3B98BF4FF000080D
:100B00003D464FF0000B43F450632360316803AB64
:100B10000222097853F82B00FDF700FB20B3BBF14C
:100B2000010F54D162682AB908212268616042F439
:100B300000722260226822F4A0622260A268511E24
:100B4000A1608AB13268511C3160127805F8012B1E
:100B50007268013A002A726006DC31465046D4F8C9
:100B60008021904700287DD10BF1010BBBF1030FD1
:100B7000CCD1616809B90A216160424B6069591A98
:100B800000F082F84FF0000BA368002B3BD03168D7
:100B900062690878125C002A35D03028226824D196
:100BA000100522D50BF1010BB8F1000F03D0013372
:100BB00008F1FF38A3607368013B002B73601BDDF5
:100BC000336801333360A368013BA360DCE7BBF10A
:100BD000020FB3D1226802F4C061B1F5007FC8D121
:100BE000102142F480726160A7E722F41062226053
:100BF0000B7805F8013BDEE731465046D4F88031EA
:100C000098470028DFD02368DB050BD5BD4207D904
:100C100015F8011C32465046D4F87C319847013D06
:100C2000BD4227D0226812F0100212D12A70394634
:100C30006368019E5046B047D9F8003021681A1DFC
:100C4000C9F800208E061B680FD51860E3680133D1
:100C5000E36000202369ED1B5D442B44236107B052
:100C6000BDE8F08F4FF0000BCDE7CA074CBF1880EE
:100C70001860EBE70120F2E7205601084DC7000895
:100C8000450101083E51010870B50B7800F1FF05E0
:100C90005E2B13BF002201224B784C1C08BF8C1C1A
:100CA000411E01F8012FA942FBD113B9621E104663
:100CB00070BD82F001012246C154144614F8015B54
:100CC0002D2D05D05D2D16D0002DF0D02B46F2E74E
:100CD00056785D2EFAD0B342F8DC1C46023201345D
:100CE000A6420155FBDCF41A013CB342A8BF002424
:100CF00001332344E1E72246D9E751F8043C181FA9
:100D0000002BBCBF0B58C01870472DE9F0410C46B2
:100D1000496B04F1440399421BD14FF48061FEF703
:100D200081FA18B94FF0FF30BDE8F0814FF48063CD
:100D3000A36394F84630606380F8FF3394F845303D
:100D400000F2FD30437094F84430037020600020BE
:100D5000EAE7A66B77003A46FFF71AF9054600283E
:100D6000E0D000EB0608014632464046FDF7E4F9C4
:100D7000C4E90D57C4F80080E9E749B1FF2A8BBFE9
:100D80008A23012003600A7088BF4FF0FF3070474C
:100D9000084670471F2938B505460C4604D9162366
:100DA00003604FF0FF3038BDC26B12B152F82130F2
:100DB0004BB9284600F030F8224601462846BDE8E7
:100DC000384000F017B8012B0AD0591C03D1162364
:100DD00003600120E7E70021204642F824109847ED
:100DE0000020E0E7024B01461868FFF7D3BF00BFC1
:100DF0009C0B002038B50023064C054608461146DA
:100E0000236001F013F9431C02D1236803B12B6066
:100E100038BD00BF1C16002001F0F8B881F0004179
:100E200002E000BF83F0004330B54FEA41044FEACF
:100E3000430594EA050F08BF90EA020F1FBF54EA6A
:100E4000000C55EA020C7FEA645C7FEA655C00F006
:100E5000E2804FEA5454D4EB5555B8BF6D420CDDD7
:100E60002C4480EA020281EA030382EA000083EA5A
:100E7000010180EA020281EA0303362D88BF30BDFA
:100E800011F0004F4FEA01314FF4801C4CEA113150
:100E900002D0404261EB410113F0004F4FEA0333AF
:100EA0004CEA133302D0524263EB430394EA050F3A
:100EB00000F0A780A4F10104D5F1200E0DDB02FAA9
:100EC0000EFC22FA05F2801841F1000103FA0EF23D
:100ED000801843FA05F359410EE0A5F120050EF103
:100EE000200E012A03FA0EFC28BF4CF0020C43FA34
:100EF00005F3C01851EBE37101F0004507D54FF041
:100F0000000EDCF1000C7EEB00006EEB0101B1F590
:100F1000801F1BD3B1F5001F0CD349085FEA3000D6
:100F20004FEA3C0C04F101044FEA445212F5800FE1
:100F300080F09A80BCF1004F08BF5FEA500C50F17E
:100F4000000041EB045141EA050130BD5FEA4C0C61
:100F5000404141EB0101013C28BFB1F5801FE9D2BE
:100F600091F0000F04BF01460020B1FA81F308BFE1
:100F70002033A3F10B03B3F120020CDA0C3208DDAD
:100F800002F1140CC2F10C0201FA0CF021FA02F188
:100F90000CE002F11402D8BFC2F1200C01FA02F1F8
:100FA00020FA0CFCDCBF41EA0C019040E41AA2BF1D
:100FB00001EB0451294330BD6FEA04041F3C1CDAE5
:100FC0000C340EDC04F11404C4F1200220FA04F005
:100FD00001FA02F340EA030021FA04F345EA0301AF
:100FE00030BDC4F10C04C4F1200220FA02F001FA71
:100FF00004F340EA0300294630BD21FA04F02946F3
:1010000030BD94F0000F83F4801306BF81F480118B
:101010000134013D4EE77FEA645C18BF7FEA655CFE
:1010200029D094EA050F08BF90EA020F05D054EAD0
:10103000000C04BF1946104630BD91EA030F1EBFD5
:101040000021002030BD5FEA545C05D140004941D9
:1010500028BF41F0004130BD14F580043CBF01F5CC
:10106000801130BD01F0004545F0FE4141F47001B2
:101070004FF0000030BD7FEA645C1ABF194610468D
:101080007FEA655C1CBF0B46024650EA013406BF8E
:1010900052EA033591EA030F41F4002130BD00BF4D
:1010A00090F0000F04BF0021704730B54FF480640A
:1010B00004F132044FF000054FF0000150E700BF8B
:1010C00090F0000F04BF0021704730B54FF48064EA
:1010D00004F1320410F0004548BF40424FF00001D7
:1010E0003EE700BF42004FEAE2014FEA31014FEA1A
:1010F00002701FBF12F07F4393F07F4F81F0605169
:10110000704732F07F4208BF704793F07F4F04BFB3
:1011100041F40021704730B54FF4607401F0004590
:1011200021F000411CE700BF50EA010208BF7047F0
:1011300030B54FF000050AE050EA010208BF7047E1
:1011400030B511F0004502D5404261EB41014FF44A
:10115000806404F132045FEA915C3FF4D8AE4FF052
:1011600003025FEADC0C18BF03325FEADC0C18BF35
:10117000033202EBDC02C2F1200300FA03FC20FA86
:1011800002F001FA03FE40EA0E0021FA02F11444D3
:10119000BDE600BF70B54FF0FF0C4CF4E06C1CEAEC
:1011A00011541DBF1CEA135594EA0C0F95EA0C0F5D
:1011B00000F0DEF82C4481EA030621EA4C5123EAD0
:1011C0004C5350EA013518BF52EA033541F48011FF
:1011D00043F4801338D0A0FB02CE4FF00005E1FBB2
:1011E00002E506F00042E0FB03E54FF00006E1FBFC
:1011F00003569CF0000F18BF4EF0010EA4F1FF043F
:10120000B6F5007F64F5407404D25FEA4E0E6D417E
:1012100046EB060642EAC62141EA55514FEAC5208F
:1012200040EA5E504FEACE2EB4F1FD0C88BFBCF50B
:10123000E06F1ED8BEF1004F08BF5FEA500E50F1BC
:10124000000041EB045170BD06F0004646EA010182
:1012500040EA020081EA0301B4EB5C04C2BFD4EBB4
:101260000C0541EA045170BD41F480114FF0000EAD
:10127000013C00F3AB8014F1360FDEBF002001F01B
:10128000004170BDC4F10004203C35DA0C341BDC95
:1012900004F11404C4F1200500FA05F320FA04F067
:1012A00001FA05F240EA020001F0004221F000419B
:1012B00010EBD37021FA04F642EB06015EEA430E0E
:1012C00008BF20EAD37070BDC4F10C04C4F120053E
:1012D00000FA04F320FA05F001FA04F240EA0200F1
:1012E00001F0004110EBD37041F100015EEA430EC2
:1012F00008BF20EAD37070BDC4F1200500FA05F2E2
:101300004EEA020E20FA04F301FA05F243EA020360
:1013100021FA04F001F0004121FA04F220EA02006F
:1013200000EBD3705EEA430E08BF20EAD37070BDB5
:1013300094F0000F0FD101F00046400041EB010195
:1013400011F4801F08BF013CF7D041EA060195F077
:10135000000F18BF704703F00046520043EB030331
:1013600013F4801F08BF013DF7D043EA060370471E
:1013700094EA0C0F0CEA135518BF95EA0C0F0CD029
:1013800050EA410618BF52EA4306D1D181EA03016F
:1013900001F000414FF0000070BD50EA410606BF69
:1013A0001046194652EA430619D094EA0C0F02D1AE
:1013B00050EA013613D195EA0C0F05D152EA0336F3
:1013C0001CBF104619460AD181EA030101F0004111
:1013D00041F0FE4141F470014FF0000070BD41F05A
:1013E000FE4141F4780170BD70B54FF0FF0C4CF434
:1013F000E06C1CEA11541DBF1CEA135594EA0C0F53
:1014000095EA0C0F00F0A7F8A4EB050481EA030E9F
:1014100052EA03354FEA013100F088804FEA033386
:101420004FF0805545EA131343EA12634FEA022254
:1014300045EA111545EA10654FEA00260EF0004115
:101440009D4208BF964244F1FD0404F5407402D267
:101450005B084FEA3202B61A65EB03055B084FEAF8
:1014600032024FF480104FF4002CB6EB020E75EBF5
:10147000030E22BFB61A754640EA0C005B084FEA1D
:101480003202B6EB020E75EB030E22BFB61A75469A
:1014900040EA5C005B084FEA3202B6EB020E75EBE5
:1014A000030E22BFB61A754640EA9C005B084FEA5D
:1014B0003202B6EB020E75EB030E22BFB61A75466A
:1014C00040EADC0055EA060E18D04FEA051545EA59
:1014D00016754FEA06164FEAC30343EA52734FEA02
:1014E000C2025FEA1C1CC0D111F4801F0BD141EA7B
:1014F00000014FF000004FF0004CB6E711F4801FE0
:1015000004BF01430020B4F1FD0C88BFBCF5E06FBF
:101510003FF6AFAEB5EB030C04BFB6EB020C5FEACF
:10152000500C50F1000041EB045170BD0EF0004E24
:101530004EEA113114EB5C04C2BFD4EB0C0541EA56
:10154000045170BD41F480114FF0000E013C90E653
:1015500045EA060E8DE60CEA135594EA0C0F08BF17
:1015600095EA0C0F3FF43BAF94EA0C0F0AD150EA16
:1015700001347FF434AF95EA0C0F7FF425AF1046A9
:1015800019462CE795EA0C0F06D152EA03353FF4D1
:10159000FDAE1046194622E750EA410618BF52EA4E
:1015A00043067FF4C5AE50EA41047FF40DAF52EA22
:1015B00043057FF4EBAE12E74FF0FF3C06E000BFBF
:1015C0004FF0010C02E000BF4FF0010C4DF804CDCC
:1015D0004FEA410C7FEA6C5C4FEA430C18BF7FEA8C
:1015E0006C5C1BD001B050EA410C0CBF52EA430CBA
:1015F00091EA030F02BF90EA020F0020704710F13A
:10160000000F91EA030F58BF994208BF90422CBFC8
:10161000D8176FEAE37040F0010070474FEA410CC1
:101620007FEA6C5C02D150EA013C07D14FEA430CDF
:101630007FEA6C5CD6D152EA033CD3D05DF8040B50
:10164000704700BF8446104662468C461946634682
:1016500000E000BF01B5FFF7B7FF002848BF10F159
:10166000000F01BD4DF808EDFFF7F4FF0CBF01209E
:1016700000205DF808FB00BF4DF808EDFFF7EAFF1A
:1016800034BF012000205DF808FB00BF4DF808EDD5
:10169000FFF7E0FF94BF012000205DF808FB00BFCA
:1016A0004DF808EDFFF7CEFF94BF012000205DF854
:1016B00008FB00BF4DF808EDFFF7C4FF34BF012061
:1016C00000205DF808FB00BF4FEA410C7FEA6C5C2C
:1016D00002D150EA013C0AD14FEA430C7FEA6C5C2C
:1016E00002D152EA033C02D14FF0000070474FF0A4
:1016F000010070474FEA410212F5001215D211D5D0
:101700006FF47873B3EB625212D94FEAC12343F0FE
:10171000004343EA505311F0004F23FA02F018BF80
:10172000404270474FF00000704750EA013005D149
:1017300011F0004008BF6FF0004070474FF000000C
:10174000704700BF80F0004002E000BF81F0004120
:1017500042001FBF5FEA410392EA030F7FEA226C57
:101760007FEA236C6AD04FEA1262D2EB1363C1BFE7
:10177000D218414048404140B8BF5B42192B88BF56
:10178000704710F0004F40F4000020F07F4018BF79
:10179000404211F0004F41F4000121F07F4118BF99
:1017A000494292EA030F3FD0A2F1010241FA03FC41
:1017B00010EB0C00C3F1200301FA03F100F0004329
:1017C00002D5494260EB4000B0F5000F13D3B0F1F1
:1017D000807F06D340084FEA310102F10102FE2A60
:1017E00051D2B1F1004F40EBC25008BF20F00100D0
:1017F00040EA03007047490040EB0000013A28BF6F
:10180000B0F5000FEDD2B0FA80FCACF1080CB2EBF1
:101810000C0200FA0CF0AABF00EBC250524218436F
:10182000BCBFD0401843704792F0000F81F4000114
:1018300006BF80F400000132013BB5E74FEA4103E7
:101840007FEA226C18BF7FEA236C21D092EA030F53
:1018500004D092F0000F08BF0846704790EA010FCD
:101860001CBF0020704712F07F4F04D1400028BFFA
:1018700040F00040704712F100723CBF00F50000DC
:10188000704700F0004343F0FE4040F40000704712
:101890007FEA226216BF08467FEA236301464202BE
:1018A00006BF5FEA412390EA010F40F480007047D1
:1018B0004FF0000304E000BF10F0004348BF404277
:1018C0005FEA000C08BF704743F0964301464FF0B3
:1018D00000001CE050EA010208BF70474FF000030F
:1018E0000AE000BF50EA010208BF704711F0004350
:1018F00002D5404261EB41015FEA010C02BF844620
:101900000146002043F0B64308BFA3F18053A3F57E
:101910000003BCFA8CF2083AA3EBC25310DB01FAC5
:1019200002FC634400FA02FCC2F12002BCF1004F49
:1019300020FA02F243EB020008BF20F001007047DA
:1019400002F1200201FA02FCC2F1200250EA4C002E
:1019500021FA02F243EB020008BF20EADC70704774
:101960004FF0FF0C1CEAD0521EBF1CEAD15392EA82
:101970000C0F93EA0C0F6FD01A4480EA010C40025E
:1019800018BF5FEA41211ED04FF0006343EA5010B8
:1019900043EA5111A0FB01310CF00040B1F5000FFA
:1019A0003EBF490041EAD3715B0040EA010062F1A9
:1019B0007F02FD2A1DD8B3F1004F40EBC25008BF93
:1019C00020F00100704790F0000F0CF0004C08BFB1
:1019D00049024CEA502040EA51207F3AC2BFD2F17E
:1019E000FF0340EAC250704740F400004FF000038C
:1019F000013A5DDC12F1190FDCBF00F000407047C6
:101A0000C2F10002410021FA02F1C2F1200200FA03
:101A100002FC5FEA310040F1000053EA4C0308BFCA
:101A200020EADC70704792F0000F00F0004C02BF1B
:101A3000400010F4000F013AF9D040EA0C0093F096
:101A4000000F01F0004C02BF490011F4000F013BF0
:101A5000F9D041EA0C018FE70CEAD15392EA0C0F5E
:101A600018BF93EA0C0F0AD030F0004C18BF31F0C9
:101A7000004CD8D180EA010000F00040704790F09F
:101A8000000F17BF90F0004F084691F0000F91F043
:101A9000004F14D092EA0C0F01D142020FD193EA09
:101AA0000C0F03D14B0218BF084608D180EA010091
:101AB00000F0004040F0FE4040F40000704740F06D
:101AC000FE4040F4400070474FF0FF0C1CEAD0523B
:101AD0001EBF1CEAD15392EA0C0F93EA0C0F69D097
:101AE000A2EB030280EA010C49024FEA402037D002
:101AF0004FF0805343EA111143EA10130CF00040F9
:101B00008B4238BF5B0042F17D024FF4000C8B42E8
:101B100024BF5B1A40EA0C00B3EB510F24BFA3EBC8
:101B2000510340EA5C00B3EB910F24BFA3EB910398
:101B300040EA9C00B3EBD10F24BFA3EBD10340EAF2
:101B4000DC001B0118BF5FEA1C1CE0D1FD2A3FF638
:101B500050AF8B4240EBC25008BF20F001007047ED
:101B60000CF0004C4CEA50207F32C2BFD2F1FF0390
:101B700040EAC250704740F400004FF00003013AC1
:101B800037E792F0000F00F0004C02BF400010F465
:101B9000000F013AF9D040EA0C0093F0000F01F079
:101BA000004C02BF490011F4000F013BF9D041EA9B
:101BB0000C0195E70CEAD15392EA0C0F08D14202CE
:101BC0007FF47DAF93EA0C0F7FF470AF084676E7A1
:101BD00093EA0C0F04D14B023FF44CAF08466EE77A
:101BE00030F0004C18BF31F0004CCAD130F0004248
:101BF0007FF45CAF31F000437FF43CAF5FE700BFA0
